:020000040000FA
:100000000002040000000000E0800000E08000002A
:10001000E0800000E0800000E0800000E080000060
:10002000E0800000E0800000E0800000E080000050
:10003000E0800000E0800000E0800000E080000040
:10004000E0800000E0800000E0800000E080000030
:10005000E0800000FE63000020640000E0800000FB
:10006000E0800000E0800000E0800000E080000010
:10007000E0800000E0800000E0800000E080000000
:10008000E0800000E0800000E0800000E0800000F0
:10009000E0800000E0800000E0800000E0800000E0
:1000A000E0800000E0800000E0800000E0800000D0
:1000B000E0800000E0800000E0800000E0800000C0
:1000C000E0800000E0800000E0800000E0800000B0
:1000D000E0800000E0800000E0800000E0800000A0
:1000E000E0800000E0800000E0800000E080000090
:1000F000E0800000E0800000E0800000E080000080
:10010000E0800000E0800000E0800000E08000006F
:10011000E0800000E0800000E0800000E08000005F
:10012000E0800000E0800000E0800000E08000004F
:10013000E0800000E0800000E0800000E08000003F
:10014000E0800000E0800000E0800000E08000002F
:10015000E0800000E0800000E0800000E08000001F
:10016000E0800000E0800000E0800000E08000000F
:10017000E0800000E0800000E0800000E0800000FF
:10018000E0800000E0800000E0800000E0800000EF
:10019000E0800000E0800000E0800000E0800000DF
:1001A000E0800000E0800000E0800000E0800000CF
:1001B000E0800000E0800000E0800000E0800000BF
:1001C000E0800000E0800000E0800000E0800000AF
:1001D000E0800000E0800000E0800000E08000009F
:1001E000E0800000E0800000E0800000E08000008F
:1001F000E0800000E0800000E0800000E08000007F
:10020000FFFFFF00FFFFFF00E0800000E080000034
:10021000E0800000E0800000E0800000E08000005E
:10022000E0800000E0800000E0800000E08000004E
:10023000E0800000E0800000E0800000E08000003E
:10024000E0800000E0800000E0800000E08000002E
:10025000E0800000FE63000020640000E0800000F9
:10026000E0800000E0800000E0800000E08000000E
:10027000E0800000E0800000E0800000E0800000FE
:10028000E0800000E0800000E0800000E0800000EE
:10029000E0800000E0800000E0800000E0800000DE
:1002A000E0800000E0800000E0800000E0800000CE
:1002B000E0800000E0800000E0800000E0800000BE
:1002C000E0800000E0800000E0800000E0800000AE
:1002D000E0800000E0800000E0800000E08000009E
:1002E000E0800000E0800000E0800000E08000008E
:1002F000E0800000E0800000E0800000E08000007E
:10030000E0800000E0800000E0800000E08000006D
:10031000E0800000E0800000E0800000E08000005D
:10032000E0800000E0800000E0800000E08000004D
:10033000E0800000E0800000E0800000E08000003D
:10034000E0800000E0800000E0800000E08000002D
:10035000E0800000E0800000E0800000E08000001D
:10036000E0800000E0800000E0800000E08000000D
:10037000E0800000E0800000E0800000E0800000FD
:10038000E0800000E0800000E0800000E0800000ED
:10039000E0800000E0800000E0800000E0800000DD
:1003A000E0800000E0800000E0800000E0800000CD
:1003B000E0800000E0800000E0800000E0800000BD
:1003C000E0800000E0800000E0800000E0800000AD
:1003D000E0800000E0800000E0800000E08000009D
:1003E000E0800000E0800000E0800000E08000008D
:1003F000E0800000E0800000E0800000E08000007D
:100400004FD921000E7F22000E018800000000005D
:100410000C00070080CD260001002000110007001D
:10042000000020000000E000020032000000020096
:1004300000000000A07D0200000000000040DA0083
:100440000000FE004440A900802520000000E000DC
:100450000300320000002000A00188004440A800F2
:100460000000060091018800800078000000EB0089
:1004700015003700E280400032A0B4009101BA00BC
:10048000E280400032A0B4009102BA00E280400055
:1004900032A0B4000002EB00472BDE00F507B200EB
:1004A000602CE10004003A000059EB008301E900F0
:1004B000FDFF3E00040037006128E100010032002A
:1004C0000082EB00040007001101BA000200E00006
:1004D000E8FF3A00000006003159BA008301E90044
:1004E0000C0032002159BA008301E90008003200F3
:1004F0000400E00003003A00E280400032A0B400B3
:10050000F5FF370011D9BA008301E900FAFF3A007C
:100510008100E800E180400032A0B4000000060045
:1005200000000000000000000000000000000000CB
:1005300000000000000000000000000000000000BB
:1005400000000000000000000000000000000000AB
:10055000000000000000000000000000000000009B
:10080000889FBE008A9FBE00010578000100E000BD
:100810000400350008003C000000E0002000320029
:100820000500370060001000E080180002003B0067
:1008300001F02C001A0037000004BE006011B8005F
:100840006B0920000982CF00020039000882CF0026
:100850000441B000694252000E00320008003B0023
:1008600082817100610164008904D1000884D30091
:100870008B05E8000442E800F9FF3A000500370064
:100880000804440089844C008B05E9000442E90017
:10089000FBFF3A00730207000AF0A70001F0A00076
:1008A0004F05BE004F04BE0000000600F4FF2F00FD
:1008B000920237001400200090023700889FBE008B
:1008C0008A9FBE008C1F7800A7020700AE0233008B
:1008D00003866C006450E1002E0032006420E100C9
:1008E000330032006150E1002F0032006120E1004E
:1008F0003100320085855500EB07B000090020006B
:1009000008042000050037000804440089844C00D6
:100910000A0031000603430087834B0000015300A7
:1009200081815B00F8FF33000203BE000800A000D5
:100930000804440089844C00F6FF3900C639DD0004
:100940008301730001003200130020008904D100EC
:100950000884D3000998A300050032000800A7000E
:100960000300A0008904D1000884D3008B05E800AF
:100970008904D1000884D3000001EB000281D20079
:100980003802070001F0A1000CF0A70001F0A00060
:10099000860237006420E100880232000801BE00B0
:1009A0000200BE00F7FF37006120E1008302320041
:1009B0006000B800F3FF37000000200001F82700B6
:1009C000F0FF370003F0A200889FBE008A9FBE00A0
:1009D0008C1F7800640207006B0233006450E10052
:1009E0004F0032006420E1005200320003826C00AC
:1009F00007003B000905D0000306D000820F540019
:100A00000C065D0002003900020032008901780006
:100A1000030678008582550004003D000003FD00B8
:100A20008103FD008502EA008B854200840F72007D
:100A300002003B0060001000E08018006011B80068
:100A40000005EB007A28E1000A0039000600780072
:100A5000C75DDD00F707B200878075002D00370005
:100A6000828171000A017800610560008180D100F7
:100A70000080D3008502E900F9FF3B000604400036
:100A80008784480002003B0060041400E0841C00DE
:100A90000988A300070032008A81710082817100F9
:100AA000610164008904D1000884D3008B05E8004B
:100AB000170037000978A30013003A000B00E0008C
:100AC000130034008B05E9000804440089844C00BD
:100AD0000A4474000978A3000D003A000B00E000FE
:100AE000070034008B05E9000804440089844C00A9
:100AF00001003A000B0020000978A300F7FF320044
:100B00000001EB0002003700828171000A017800C9
:100B1000D40107000CF0A70001F0A0002302370069
:100B20006420E10002003A00838F6C00230233004E
:100B30000801BE000200BE001C023700889FBE00F4
:100B40008A9FBE008C1F7800070207000E02330048
:100B500003866C006450E100240032006420E10050
:100B6000270032006150E100220032006120E100E4
:100B7000210032008B854200EB07B1000134B80040
:100B8000003AB8000804420089844A00013AB800DB
:100B90000030B8008880400009014A00040033009A
:100BA0000000400081804800020149008B05E900F7
:100BB000C909DD008301700001003200130020002C
:100BC000C814DE004814DD004709DE001200B20040
:100BD000C808DE0008847000A201070001F0A1002F
:100BE0000CF0A70001F0A000F00137006120E10047
:100BF000F20132000801BE000200BE00F7FF37001C
:100C00006150E100FCFF3A00EC0137000001BE003A
:100C1000ED0107000470A70003F0A10003F8A30092
:100C200013003A006509B1001000320009003500D8
:100C30006928E100020035000100280000000500DD
:100C400000004000818048008502E900FCFF3A0076
:100C500000000600F88F4200050035008100D10039
:100C60000080D3008502E800FCFF3A000000060087
:100C70008000EB0000000500889FBE008A9FBE0038
:100C8000030578000300E000050035000B003C0080
:100C9000008270000402710030003200070037004B
:100CA00060001000E080180060011900E081190068
:100CB00002003B0001F02D00280037000004BE00B8
:100CC0000200BE006011B8006B09200095022000F0
:100CD0000182CF000A0039000541B1000082CF0037
:100CE000070039000541B1000982CF000400390036
:100CF0000541B1000882CF00010039000541B10073
:100D000005425200120032000A003B00828171004D
:100D1000610164008100D1000080D3008984D30088
:100D20000884D3008B05E8000442E800F7FF3A008E
:100D3000070037000804440089844C000000480084
:100D4000818048008B05E9000442E900F9FF3A0080
:100D5000440107000AF0A70001F0A0004F05BE0003
:100D60004F04BE00000006000003BE00960107000D
:100D70006011B8000470A70007F0A10007F8A300F5
:100D800017003A006509B1000D0032000D00350072
:100D9000860220000628E100030035000300280039
:100DA0006000B8000200050000004000818048009B
:100DB00002014900838149008502E900FAFF3A00F7
:100DC00000000600F88F4200050034008100D100C9
:100DD0000080D3008502E800FCFF3A000000060016
:100DE0006011B8008000EB0000000500881F78004B
:100DF000000478005001BE004000BE000400400026
:100E0000858048000601490087814900009CBE009A
:100E10000294BE000400E1000588E1000690E100B4
:100E20000798E10002003100680044001008E80063
:100E30004F04780000000600F4874700889FBE003A
:100E40008A9FBE008C9FBE008E1F78000205BE00E8
:100E50000004BE00D4B79F00E5B79F00F6B79F001F
:100E600087BF9F000000EB00C0B79F00B0B79F0096
:100E7000A0B79F0090B79F0080B79F000D0420008F
:100E8000BFB097004FB09700000140000000E000A5
:100E90000F003D004F08DE0000007100C0B79F004A
:100EA0009E00070001003D0012002000A100070085
:100EB00001003D0012002000A6000700B10007005D
:100EC000B60007000F004000C8FF070022003700EF
:100ED0004F08DE0000067100CCB79F008F000700AE
:100EE00001003D00120020009200070001003D00BB
:100EF0001200200097000700A20007000FB2970021
:100F00009FB297002FB39700BFB39700A9000700C7
:100F10000000520081805A0002015B0083815B0067
:100F200080B79F0091B79F00A2B79F00B3B79F0003
:100F30000007EB009F0007000020E10001A8E1008E
:100F400002B0E10003B8E100010031001E00200002
:100F50000E005600C0B79F004FB297000400E0009B
:100F60000700350010002000010020006011B800CB
:100F700008047000898470000A0571008B85710077
:100F80008D06E900BEFF3A000400E00003003D00CA
:100F9000820007000F00400094FF07004FA8970051
:100FA0000000E00004003A000FB497009FB49700DF
:100FB0002FB59700BFB59700940007004F07780042
:100FC0004F06BE004F05BE004F04BE004F01B100EA
:100FD00000000600881F780018002000881F780095
:100FE00095FF07008F87E9004F0478000000060096
:100FF000801FEB0090FF07008F87E90000000600CC
:10100000889FBE008A9FBE008C1F78006E0007007C
:1010100007003D0073000700E00F5B00E08F5B00FE
:1010200007003D00320007000006EB000400370017
:101030003400070002003D002A0007001C002000C9
:1010400072000700E3FF07000203BE000002BE00BB
:101050000C00E00001003200220007000400BE0086
:101060000601BE004F0678004F05BE004F04BE00CB
:1010700000000600889FBE008A9FBE008C1F78007B
:101080005100070005003D0056000700E00F5B001F
:10109000E08F5B0006003D000400370019000700E8
:1010A00003003D006000B8006011B80010000700A8
:1010B00056000700CEFF07000203BE000002BE007C
:1010C0000C00E00001003200060007000400BE0032
:1010D0000601BE004F0678004F05BE004F04BE005B
:1010E000000006006000B8006011B8000000370082
:1010F0000402500085825800060359008783590076
:10110000000006000006EB00E00F5200E08F5A00DE
:10111000E00F5B00E08F5B000000060001804000F4
:1011200090B79F000001EB008FB097000100E00036
:10113000000006000200700090B79F000180400090
:1011400080B79F000001EB00FFA897000100E000BE
:10115000000006000200700080B79F000180400080
:101160006FAA9700CF20DE0001007000F0AF9F0053
:1011700004024200250007004F18DE000002720042
:1011800000000600E4AF9F000804440089844C007E
:101190000A054D008B854D00000006003FB2970008
:1011A000CFB297005FB39700EFB3970000FE2F0018
:1011B000000006003FB09700CFB097005FB19700E6
:1011C000EFB19700000006000205BE000004BE005B
:1011D000E00F5000E08F5800E00F5900E08F5900F9
:1011E000000006006000B8006011B800080450005C
:1011F000898458000A0559008B8559001C0020007D
:10120000E00F5200E08F5A00000006000800BE0008
:101210000A01BE00000006006022B800060220009D
:101220000000D0008180D2000482D2008582D200EA
:101230000000A0000202520083825A000300310025
:101240000202420083824A000000A1000603E90076
:10125000F3FF3A0000000600EFFF07000400BE00A5
:101260000000060081002000618055000B003D0059
:101270000B00200061FE2F000100E1001D00340082
:1012800082817100610164008904D1000884D30067
:101290000000E800FAFF3A007100200061006400DD
:1012A0000300700002006000090032006104440085
:1012B000E0844C000988A500050032008B05E80099
:1012C0006808E10002003A008904D1000884D300D4
:1012D000F20F20000258E10005003D00C75DDD006F
:1012E000F907B20089807500080078000000060048
:1012F0000BF827008B00780000000500889FBE00D7
:101300008A9FBE00841F7800170007004F007800F6
:1013100011003300F0FF2F00838F6C0006003B00AC
:10132000040565000A00A7000800370009F0A600C0
:101330001000200008003700820F5400838F5C00EB
:10134000030039001000200001003E0000002000D2
:1013500009F0A7000000EA004F05BE004F04BE00E0
:101360000000E000000006000004BE0016000700B8
:101370000003BE000405BE000200BE00120007000C
:10138000844F7500000006000200BE006450E100BA
:10139000050036006420E100020036000968A30061
:1013A00001003A000800BE000160A0004F0678006E
:1013B0004F05BE004F04BE0000000600F0FF2F00E6
:1013C000F1FF2700F9FF3700C70ADE00F107B2007E
:1013D000F50FB20008003200E1CF420002003200F7
:1013E0000170A00024000500810F70000100320090
:1013F0000408050044000500810F700002003A0057
:10140000140005008502E9000000400081C048008A
:10141000FCFF3B000170A000240005003E0000001E
:1014200008200000080000001B5B000044000000D2
:101430001B5B000000440000001B00005B43000039
:10144000001B00005B3200004B0D00000043000059
:10145000000000001B5B0000324400000057000049
:10146000617200006E6900006E6700003A200000A3
:101470006E6F0000207600006F6C00007461000049
:1014800067650000206F00006E20000056700000AD
:10149000756C00006C750000702000007069000021
:1014A0006E000000203D000020000000436C0000A2
:1014B0007574000063680000206500006E6700001E
:1014C0006167000065640000212100002100000028
:1014D0005652000045470000207400006F6F000066
:1014E000206C00006F7700002C2000006973000062
:1014F0002074000068650000726500002061000033
:1015000020730000686F0000727400003F0000004C
:10151000436C0000757400006368000020640000E4
:1015200069730000656E0000676100006765000078
:101530006421000021210000002E0000203C00005A
:10154000002E000020000000546F00002066000004
:10155000696E000069730000682000007365000078
:1015600074750000702C000020730000746100008E
:101570007274000020750000702000007468000084
:1015800065200000706F0000776500007220000089
:1015900073750000707000006C69000065730000D6
:1015A000207700006974000068200000636F00006D
:1015B0006D6D0000616E0000642000002757000080
:1015C000270D00000A0000000D0A0000280000009E
:1015D00078000000293E0000004200007573000002
:1015E0002050000069720000617400006520000056
:1015F0007633000000200000636C00006F6E000076
:1016000065200000772F0000646900006666000016
:1016100065720000656E00007420000050490000F3
:101620004300000046690000726D00007761000011
:101630007265000020760000362E0000332D000079
:101640006265000074610000312000007232000009
:101650003038000038200000002000002832000050
:10166000344600004A360000344700004130000094
:101670003000000034200000003200002000000094
:1016800041330000004200003400000042350000F9
:101690000042000038000000554E00004B000000E2
:1016A0002900000049090000004F00000900000067
:1016B00048090000004C000009000000456E0000D1
:1016C0007465000072200000726100007720000045
:1016D000766100006C75000065200000666F0000F8
:1016E000722000004252000047000000000000008D
:1016F00000000000000000002C01000000000000BD
:101700005802000000000000B004000000000000CB
:101710006009000000000000C0120000000000008E
:10172000802500000000000040380000000000009C
:10173000004B00000000000080700000000000006E
:101740000096000000000000C0DA00000000000069
:1017500000E100000000000000C2000001000000E5
:1017600000F400000100000000E800000300000099
:1017700041520000543100000000000020480000E9
:101780007A00000046720000657100007565000077
:101790006E63000069650000732000003C200000BB
:1017A000314800007A2000006172000065200000CE
:1017B0006E6F0000742000007375000070700000F0
:1017C0006F72000074650000642E000000000000CD
:1017D0003062000000300000303000002C000000BB
:1017E000303000000030000031320000333400009F
:1017F0003536000037380000394100004243000010
:10180000444500004630000078000000436F0000AF
:10181000756C0000646E000027740000206B0000EF
:101820006565000070200000757000000000000079
:101830005350000049310000000000000029000062
:101840000020000057000000205200000049000066
:1018500032430000310000003A2000000000000088
:101860002E00000031570000303100000000000061
:10187000314100004C53000000420000507600004F
:1018800033000000080800000808000008000000FD
:101890000000000042420000494F000031000000FB
:1018A0005241000057310000000000004F4300008B
:1018B00044310000000000000000000000000000B3
:1018C000290000000000000000000000EE87470033
:1018D000889FBE008A9FBE008C9FBE008E1F78002E
:1018E0000000EB005065880040658800A04088003B
:1018F0006065880000017800E3CA20000042EB0028
:10190000050220004510DD00030040008000EB00D0
:10191000045878008100E800858F5000FCFF3A00F1
:101920000201E800E50F5100F6FF3A000000EB006D
:10193000706A880080067800D0B79F00C0B79F000B
:10194000ACAF2000A1408000000320000089B90056
:1019500040952000000041002860020000000000C7
:10196000A18120000020200011006000040032004E
:1019700071002000E0562000827C02000000000080
:10198000E0A0280028600200000000000001EB0039
:10199000B2B79F0001003700BEB79F00706A800099
:1019A0000000E000440032000000E900706A880096
:1019B0004500DD00E1CA2000E0C078000104E0003D
:1019C000130032000004EB0089BA2000EACA2000AC
:1019D0004065800001F07C0001407800B4630200A3
:1019E00000000000406580000000E8000804E800F6
:1019F000F00FB20040658800706A80004500DD008D
:101A000008004000E0407D000104E000F0FF3A00E3
:101A10000000EB00706A8800270037009C407800C7
:101A200064C06000240032004A8120001A0078005F
:101A3000090320000980B9007A004000C892200004
:101A400060007C00000001000000E0001A0032008D
:101A50001A0078000980B9008002B0000800400038
:101A60002860020000000000E0A0280028600200BA
:101A7000000000005065800041658000810F50002B
:101A80000D00320000047800808F50000A00320000
:101A900089BA200068C07C00B46302000000000026
:101AA00008007800F00FB2000004E80040658000F4
:101AB000800F5400F7FF3A001A6302000000000094
:101AC0000004E000D5FF3200D063020000000000F7
:101AD0000004E00003003200D863020000000000B0
:101AE000AEFF3700A0630200000000000045780050
:101AF0000080FB0001002000F2072000820F500050
:101B0000E08F580083023E00006001007902370038
:101B10003F023700130137007E023700BD00370057
:101B20004E023700250137007A0237007700370070
:101B3000780237005C023700760237007502370002
:101B40005902370099013700720237002901370026
:101B5000700237006F0237006E0237006D023700E7
:101B60006C0237006B0237006A02370069023700E7
:101B70006802370067023700D3003700650237007C
:101B800064023700630237006202370061023700E7
:101B9000600237005F0237005E0237005D023700E7
:101BA0005C0237005B0237005A02370059023700E7
:101BB00058023700570237005602370055023700E7
:101BC00054023700530237005202370051023700E7
:101BD000500237004F0237004E0237004D023700E7
:101BE0004C0237004B0237004A02370049023700E7
:101BF00048023700470237004602370045023700E7
:101C000044023700430237004202370041023700E6
:101C1000400237003F0237003E0237003D023700E6
:101C20003C0237003B0237003A02370039023700E6
:101C300038023700370237003602370035023700E6
:101C400034023700330237003202370031023700E6
:101C5000300237002F0237002E0237002D023700E6
:101C60002C0237002B0237002A02370029023700E6
:101C700028023700270237002602370025023700E6
:101C800024023700230237002202370021023700E6
:101C9000200237001F0237001E0237001D023700E6
:101CA0001C0237001B0237001A02370019023700E6
:101CB00018023700170237001602370015023700E6
:101CC00014023700130237001202370011023700E6
:101CD000100237000F0237000E0237000D023700E6
:101CE0000C0237000B0237000A02370009023700E6
:101CF00008023700070237000602370005023700E6
:101D000004023700030237004200370050658000AC
:101D1000808F56003B00320040658000808F560067
:101D20000B003A000D00E90080067800FD0FB200BC
:101D30004D6588000040EB0083BA200080F67900F2
:101D400000A12800286002000000000013FF3700F7
:101D50000D00E90080067800FD0FB20040A12800C8
:101D600028600200000000000D0178008D0078005E
:101D70008004EB00406580008D0F5000140032009D
:101D80008004EB008ABA20000204E80068407D006D
:101D900000717D000004E00003003200B463020023
:101DA000000000000300370000C2B300B46302006B
:101DB000000000008904E80008017800F20FB2007A
:101DC0008200780040658000820F5000EEFF3A00EC
:101DD0000100E900F00FB2004065880080A12800F2
:101DE0002860020000000000094078000462020040
:101DF00000000000B0A128002860020000000000E0
:101E0000E6FE370070C0B300B463020000000000BB
:101E1000E2FE370040658000808F560026003200C9
:101E20008D0078000D0178000005EB008D0F50004B
:101E3000140032000005EB0089BA20000104E8001C
:101E400068C07C0080F07C000004E00003003200E9
:101E5000B4630200000000000300370000C2B300BA
:101E6000B4630200000000000A05E8008800780062
:101E7000F10FB2000101780040658000810F500031
:101E8000EEFF3A000200E900F00FB2004065880062
:101E900080A1280028600200000000000A407800AD
:101EA0000462020000000000B0A1280028600200C7
:101EB00000000000B9FE370070C0B300B463020038
:101EC00000000000B5FE3700A06302000000000023
:101ED000B1C5B300814F5000B0FE3A00A0630200CC
:101EE000000000008040780010C4B30080CF500094
:101EF0004000320007003E007040500080CF50008C
:101F00000C0032006340400080CF5000A3FE3A0036
:101F10000E00370030C4B30080CF500027003200DD
:101F2000A20039000040E80080CF50009BFE3A003C
:101F30000C003700A063020000000000E1C7B300FE
:101F4000814F500095FE3A0031013700A063020036
:101F500000000000E1C7B300814F50008FFE3A003F
:101F60003E0137004FB09700E40F500005003400E9
:101F70005A6F0200000000008000EB00C1B79F0014
:101F800086FE370050658000808F560007003200C3
:101F90000D00E90080067800FD0FB20040A1280086
:101FA00028600200000000007CFE370070C0B30013
:101FB000B46302000000000078FE37004065800036
:101FC000808F5600070032000D00E8008006780080
:101FD000FD0FB200D0A12800286002000000000020
:101FE0006EFE370070C0B300B46302000000000052
:101FF0006AFE3700546580000400E90000047800A0
:10200000F80FB2000805780041658000810F540088
:10201000620032008002EB0083BA200068C07900C1
:102020000004E00057003A000800E90000017800D1
:10203000F20FB20062C079000004E00051003200EB
:102040008502E800BFB19700858F51004D00310037
:102050008301E800B3B79F00810F52000A003200ED
:1020600083BA20008042EB00F60F200085F0790053
:102070000100E90086006000810F5200FBFF3A007A
:102080004165880085F0790041658000828F5000AD
:10209000CF053A000D00370083BA200062C07900F6
:1020A0000004E00004003A000200E800F00FB20073
:1020B000D0B79F00050037000200E900000178005A
:1020C000F20FB200828F5000F3FF3A0010A22800F6
:1020D0002860020000000000A140800000032000F2
:1020E0000089B900409520000000410028600200EE
:1020F00000000000A18120000020200011006000ED
:102100000400320071002000E0562000827C0200B2
:1021100000000000E0A0280028600200000000008D
:102120005FB09700880F50000F00320080047800E5
:102130008BBA2000FD0F200069C07D00B46302004F
:10214000000000004065800069F07D000000E800AC
:102150000D006000406588000900E8008D04600003
:10216000888F5400F4FF3A004D6580000040EB007A
:1021700082BA2000807679008A8F560007FE3A00E6
:10218000060037000800E90000047800F80FB200EC
:1021900008057800888F50009FFF3A0070C0B30098
:1021A000B463020000000000FCFD370054658000AD
:1021B0000400E90080047800F90FB20009057800F6
:1021C00041658000818F5400620032000007EB00FF
:1021D00083BA200069C079000004E00057003A008B
:1021E0000900E90000017800F20FB20062C0790036
:1021F0000004E000510032000E07E800BFB1970074
:102200000300E9008E0F50004C003A00810F52008D
:102210000A00320083BA20008042EB00F60F200053
:1022200085F079000100E90086006000810F52000E
:10223000FBFF3A004165880085F079004165800028
:10224000828F500067053A000D00370083BA2000E6
:1022500062C079000004E00004003A000200E800D7
:10226000F00FB200D0B79F00050037000200E90070
:1022700000017800F20FB200828F5000F3FF3A00A5
:1022800010A228002860020000000000A140800089
:10229000000320000089B9004095200000004100A3
:1022A0002860020000000000A18120000020200022
:1022B000110060000400320071002000E056200090
:1022C000827C020000000000E0A0280028600200DC
:1022D000000000005FB09700890F50000F0032002F
:1022E000000478008BBA2000FD0F200068C07D003C
:1022F000B4630200000000004065800068F07D00CB
:102300000000E8000D006000406588000800E8005B
:102310000D046000890F5400F4FF3A004D65800001
:102320000040EB0082BA2000807679008A8F560048
:1023300099FD3A00BEB79F00060037000900E9008A
:1023400080047800F90FB20009057800898F5000E9
:102350009FFF3A003FB09700E10F500028003A007D
:1023600010A228002860020000000000A1408000A8
:10237000000320000089B9004095200000004100C2
:102380002860020000000000A18120000020200041
:10239000110060000400320071002000E0562000AF
:1023A000827C020000000000E0A0280028600200FB
:1023B000000000004D65800051658000818F56004F
:1023C0000900320082BA20008041EB00F40F2000A7
:1023D000837679000D00E90084066000818F560045
:1023E000FBFF3A004D6588000040EB0081BA2000F9
:1023F00080F678000001EB00B2B79F0067FD370060
:1024000070C0B300B46302000000000063FD370039
:1024100058658000888F56000C00320080A128008B
:10242000286002000000000008805600F00FB20093
:102430000462020000000000B0A128002860020031
:10244000000000005D65800054FD370070C0B300DF
:10245000B46302000000000050FD370048658000B2
:10246000888F56000C00320080A1280028600200EE
:10247000000000000D005400F00FB20004620200E2
:102480000000000070A22800286002000000000088
:102490004D65800041FD370070C0B300B463020099
:1024A000000000003DFD3700406580008040EB00EB
:1024B00083BA200001F079000000E800800678006F
:1024C000FD0FB2004D65880090A228004060020018
:1024D0000000000040658000F0B79F00516580005B
:1024E000E1B79F000000EB006065880000477800BE
:1024F000530037004FB197000201E800C2B79F00B8
:10250000F40F510025FD3A0048640200000000006D
:1025100022FD3700486580000800E800F90F200020
:102520000900600051658000810F500040003200BA
:10253000FF4F55003E003600E0C7B300804F550006
:102540003B003E008D0F54000C003A000A4078001A
:10255000B4630200000000004065800083BA2000E0
:102560000AF079000000E800890660004D658800E7
:102570000040EB0080F6790008FD370080A12800BC
:1025800028600200000000000D005400F80F200039
:1025900008006000046202000000000070A2280031
:1025A0002860020000000000496580000D00E9007D
:1025B00088056000898F55001000320088BA20001D
:1025C0000900E80069707C0069407C000004E000BC
:1025D00005003200B463020000000000A0A2280041
:1025E00028600200000000000900E9008004780073
:1025F000F90FB200898F5500F1FF3A000A407800C8
:10260000B46302000000000082BA20008A767900DC
:102610000D00E800F10F2000810660004065800099
:102620000000E8000100600040658800DBFC370026
:1026300070C0B300B463020000000000D7FC370094
:102640005265800083BA200062C079000080FB00E0
:1026500001002000E3072000830F5000E08F5800A6
:1026600030043E0000600100300437002D043700C4
:102670002C0437002B0437002A04370029043700C4
:1026800028043700270437002604370025043700C4
:1026900026043700230437002204370023043700C0
:1026A000200437001F0437001E0437001D043700C4
:1026B0001C0437001B0437001A04370019043700C4
:1026C00018043700170437001604370015043700C4
:1026D00014043700130437001204370011043700C4
:1026E000100437000F04370010043700F0033700E0
:1026F00072023700120137001B013700CF0137008B
:10270000BD013700070437004F02370005043700CA
:10271000040437000504370004043700A40337001D
:10272000BB0337008A033700D5023700D4023700D5
:10273000D3023700D2023700D1023700D00237006F
:10274000CF023700CE023700CD023700CC0237006F
:10275000F4033700F3033700D4013700B800370023
:10276000F00337003F003700290137001D01370013
:10277000EC033700610037009C013700E9033700A4
:10278000E8033700E7033700E6033700E5033700C7
:10279000E4033700E303370061003700E10337004B
:1027A000E0033700DF03370081003700DD03370027
:1027B000DC033700B2013700DA033700D9033700F2
:1027C000D803370026013700D6033700D50337007A
:1027D000D40337008B0237006903370098023700B3
:1027E000990337007E033700CE033700F20037002D
:1027F000270037003A0037006E013700C903370061
:10280000290037002B003700C803370018003700B5
:10281000C4033700C30337004A0037001A003700EB
:10282000C00337001C0037004F003700BD033700DE
:10283000F6023700BB033700BA033700B90337008D
:102840001700370040013700B6033700B5033700E3
:10285000B40337007202370091003700800237005E
:10286000AA003700E67C020000000000AF0337003A
:10287000E0050700408120001000E000AB033200BB
:1028800051060700A9033700D8040700A703370043
:102890006F070700A50337004E070700A3033700A3
:1028A000CE060700A103370012340200000000002A
:1028B0009E033700408120001000E00005003A0030
:1028C000D1012000505A2000DC7C020000000000F2
:1028D00096033700C0320200000000009303370067
:1028E000C0CFB3001C4E600061012000A057200043
:1028F000DC7C0200000000008C0337001C407800E4
:102900000014A1000004A000004E78005101200036
:1029100000592000DC7C0200000000008303370027
:102920001C34A000C1012000E07E2000827C020057
:102930000000000090A2280040600200000000009B
:102940007A0337001C34A100B1012000307D200043
:10295000827C02000000000090A22800406002007B
:102960000000000071033700408120001000E000EB
:1029700005003A00D1012000505A2000DC7C020002
:102980000000000069033700CB62A900C962A900FA
:1029900051012000205C2000827C02000000000029
:1029A00090A2280040600200000000005F03370092
:1029B000408120001000E00005003A00D101200015
:1029C000505A2000DC7C0200000000005703370052
:1029D0009C40780070C0600004003A002102200092
:1029E000F0E92000DC7C020000000000C962A800C1
:1029F000CB62A90041012000705D2000827C0200B2
:102A00000000000090A228004060020000000000CA
:102A100021E3A800B0C0B300FE7A0200000000006D
:102A2000F1042000810F500003003E00F0A22800B6
:102A3000406002000000000021E3A9003B033700D2
:102A40000200E800F00FB20050658800570407004C
:102A500072030700000478004A62020000000000D0
:102A600020A528002860020000000000084078002F
:102A7000046202000000000020A528002860020077
:102A800000000000084078006060020000000000C4
:102A900090A22800406002000000000023033700DD
:102AA0000200E800F00FB200506588003F04070004
:102AB0005A0307000080FB005A7C0200000000005F
:102AC000000478004A6202000000000020A52800EF
:102AD0002860020000000000084078000462020044
:102AE0000000000020A5280028600200000000006F
:102AF00008407800606002000000000090A22800FA
:102B00004060020000000000080337004081200000
:102B10001000E00005003A0011C0B3000140780049
:102B2000327402000000000000033700A101200001
:102B3000B05E2000DC7C020000000000FB023700D9
:102B40005100200050602000DC7C020000000000EA
:102B500012630200000000000004E000FCFF3200ED
:102B60000000FE00F1023700727D0200000000004C
:102B70000000E000ED023200A1002000A060200073
:102B8000DC7C02000000000040062000087C0200FF
:102B900000000000C07A0200000000001263020082
:102BA000000000000004E000FCFF320081BF2A00AA
:102BB00001400100DD023700B50307008004780002
:102BC0000000E000D90232000004EB00F8390200F6
:102BD000000000000804E800888F5400D30232008F
:102BE000FAFF3700AA030700800478000000E00025
:102BF000CE0232000004EB00DC39020000000000CD
:102C00000804E800888F5400C8023200FAFF370039
:102C10009F030700800478000000E000C302320038
:102C20000004EB006101200040612000827C020072
:102C300000000000143A02000000000018600200CA
:102C40000000000090A22800406002000000000088
:102C50000804E800888F5400B4023200F1FF370006
:102C6000408120001000E00005003A00D101200062
:102C7000505A2000DC7C020000000000AB0237004C
:102C8000C002A900C202A80021E3A8002000200081
:102C9000087C020000000000A0C0B300FE7A020021
:102CA00000000000011B2000810F500018003600BA
:102CB00090C0B300FE7A020000000000712B2000DB
:102CC000810F50001200360011012000A062200088
:102CD000827C02000000000090A2280040600200F8
:102CE00000000000A0408000020320000280B90024
:102CF0000002B000C29220006000790000000100D4
:102D000060A5280040600200000000000C003700B1
:102D1000C002A900C202A90080A6280040600200EB
:102D20000000000021012000B0632000827C02002E
:102D30000000000090A22800406002000000000097
:102D400021E3A90079023700A14080000100E000E2
:102D500005003A00D1012000505A2000DC7C02001E
:102D60000000000071023700000320000088B90055
:102D70002002B000C2922000600079000000010033
:102D800080A828004060020000000000C002A900E6
:102D9000C202A90021012000B0632000827C020051
:102DA0000000000090A22800406002000000000027
:102DB0005E023700F1002000C0362000827C020055
:102DC00000000000107B0200000000001100200045
:102DD000B0372000827C02000000000090A2280092
:102DE0004060020000000000500237001E7B02001D
:102DF000000000004D0237002503070000047800A2
:102E00006100200090652000827C0200000000002C
:102E100008007800BA6102000000000021002000D4
:102E2000F0652000DC7C0200000000000800780053
:102E30002C7C0200000000003C0237001403070055
:102E4000000478006100200090652000827C020070
:102E50000000000008007800BA61020000000000D5
:102E60002100200030EE2000DC7C02000000000089
:102E700008007800087C0200000000002B023700E8
:102E8000408120001000E00005003A00D101200040
:102E9000505A2000DC7C02000000000023023700B2
:102EA0003A3A020000000000200237001100200022
:102EB000616588000200E8008081FB0080BA200084
:102EC000634078000004E000130032000102780043
:102ED000E6C3B300F70F200085BA2000864F5000EC
:102EE00001003A000002EB008100E800010041000F
:102EF0000700600060C07A000004E000F7FF3A00BD
:102F00006465880020022000808F50000200340099
:102F10001000200060658800696580000900E000FD
:102F200002023A00536588003C0207000004780062
:102F300052658000F30F20008300610080BA2000FA
:102F4000E1407800D0C3B30080CF50001E003A00AB
:102F50000802E900E40F520018003E000200E800F9
:102F60008301600053658800C520DD00E0CA2000B1
:102F700080804000090078000041EB00050220003D
:102F8000825878000000E800850F50001A023200D5
:102F9000FBFF3700825878000300E8008081FB00C7
:102FA00080BA200063417800E0C3B300804F510035
:102FB000F8FF3A0053658800DC013700100020005C
:102FC00060658800D90137000800E00013003A006E
:102FD000E9CA2000180020000840780004620200BE
:102FE00000000000D0A928002860020000000000B6
:102FF000090078002860020000000000E0A028001E
:1030000040600200000000000804E8000902B0006F
:10301000E60F5400C5013200EFFF37000800E90059
:10302000E40F500005003E0090A22800406002001E
:1030300000000000786A8800BC0137001000200002
:1030400060658800B90137000200E800F80F200031
:103050000800600050658800F001070080047800D7
:10306000D2020700506580000800600081BA20008D
:10307000E0C0780090C2B30080CF50000C003A004E
:10308000A0408000020320000280B9007C004000C4
:10309000C2922000E00079000900780001000100E0
:1030A00090A2280040600200000000009F0137004D
:1030B00010002000606588009C013700130020008C
:1030C000636588000200E8000080FB0081BA2000F0
:1030D00060C078000004E0000E0032008280E8004A
:1030E0000301780025C2B300F30F200084BA20004A
:1030F000854F500001003A000001EB0003806000A2
:1031000060407A008100E8000004E000F8FF3A0027
:1031100062658800606580000000E00083013A007D
:103120007100200010662000827C02000000000078
:1031300020C2B300B46302000000000050658000AC
:103140000000E800506588000081FB0080BA200084
:10315000E240780020C2B30080CF5000210032004E
:1031600088BA20005265880001407800B4630200EC
:10317000000000005065800060407C008001FB0082
:10318000A0AF2000104078006840600004003200CA
:10319000030078005A7C02000000000080017800E3
:1031A000A0408000020320000280B90068004000B7
:1031B000C2922000E00079000300780001000100C5
:1031C000506580000000E80050658800000178002C
:1031D000F20FB200E2407C0020C2B30080CF50006A
:1031E000E0FF3A005265880020C2B300B4630200D9
:1031F0000000000090A228004060020000000000D3
:103200004A013700A0408000020320000280B9007C
:10321000C2922000620078000000010043013700E4
:10322000A0408000020320000280B9000080E80076
:10323000C292200060007900000001003B013700CD
:10324000A0408000020320000280B900640040001A
:10325000C2922000600079000000010033013700B5
:10326000A0408000020320000280B90066004000F8
:10327000C292200060007900000001002B0137009D
:103280007100200010662000827C02000000000017
:103290006201070080047800506580000000E900AA
:1032A0000080FB0050658800F901070080BF9F0087
:1032B0000E020700800078000000E00009003200E4
:1032C00090AE200001487800E88F500003003400E1
:1032D000A0AF20001054A00002003700A0AF2000D3
:1032E0001054A1008005EB00410037000900780070
:1032F0007C7B02000000000003C2B300A2AF2000EC
:1033000012C0610005003A0081C0B30090AE2000F9
:1033100090CF100005003A000B00370003C1B30046
:1033200092AE200092CF110007003200B0C3B3006C
:10333000B46302000000000091AE2000114078004C
:103340000462020000000000A2AF200012417800D9
:103350006840610004003200090078005A7C0200D5
:103360000000000080047800A040800002032000DC
:103370000280B90068004000C2922000E00079009D
:1033800009007800010001000004780000C2B300C9
:10339000B463020000000000AAAF200003C4B30021
:1033A0001AC0610011003200610020008066200018
:1033B000827C0200000000001A4578006840650029
:1033C00004003200080078005A7C0200000000006F
:1033D00000047800080078007C7B020000000000F8
:1033E00000C2B300B4630200000000008B05E800D7
:1033F0000FB89700808F5500BCFF3A0090A22800BC
:103400004060020000000000C8003700610020009A
:1034100080662000827C020000000000CA010700D4
:10342000804478009A01070080057800AF0107000A
:10343000800078000000E0000900320090AE20001B
:1034400001487800E88F500003003400A0AF20004E
:103450001054A00002003700A0AF20001054A100BB
:103460000904E000040032002181200011477800A7
:103470000980FB008008E9000B00E0002C0032000E
:103480000004EB009AAE2000A04080000203200060
:103490000280B9006A004000C292200060007900FA
:1034A0000000010080007800A2AF200012417800E7
:1034B0006840610004003200010078005A7C02007C
:1034C0000000000080007800010078007C7B020092
:1034D0000000000001C2B300A3AF200013C06000D1
:1034E00004003A0082C0B3009A4F110004003A0071
:1034F0000900370003C1B3009ACF11000600320063
:10350000B0C3B300B4630200000000001A407800AA
:10351000046202000000000000C2B300B4630200B5
:10352000000000000804E800888F5500D6FF3A002C
:103530000904E000020032000E80FB009040880089
:1035400090A22800406002000000000077003700D1
:1035500081002000E0662000DC7C0200000000000A
:10356000A0408000020320000280B9006C004000EF
:10357000C292200060007900000001006B0037005B
:103580008100200060672000DC7C02000000000059
:10359000A0408000020320000280B9006E004000BD
:1035A000C292200060007900000001005F00370037
:1035B000E1002000E0672000DC7C02000000000049
:1035C000A0408000020320000280B900700040008B
:1035D000C292200060007900000001005300370013
:1035E000E1002000C0682000DC7C02000000000038
:1035F000A0408000020320000280B9007200400059
:10360000C2922000600079000000010047003700EE
:10361000C1002000D0642000827C02000000000075
:10362000A0408000020320000280B9007400400026
:10363000C2922000600079000000010018600200C2
:103640000000000039003700110107000004780075
:10365000D1002000A06A2000827C0200000000004F
:10366000080078007C7B0200000000000800E000F9
:103670000B0032008004EB000A032000CB922000F4
:10368000A04080000A80B9007600400060807D0084
:10369000000001008904E800890F5400F8FF3A0097
:1036A00090A2280040600200000000001F003700C8
:1036B000F700070080047800A1002000706B200054
:1036C000827C0200000000000900E00010003200CF
:1036D0000004EB000A032000CB922000A0408000F1
:1036E0000A80B9007800400060807D000000010081
:1036F000186002000000000000C2B300B4630200C2
:10370000000000000804E800888F5400F3FF3A002E
:1037100001012000A0692000DC7C02000000000004
:1037200002003700100020006065880050658000AE
:103730000000E8000080FB005065880060658000A4
:103740000000E00002003A00000178001600370097
:1037500051012000106C2000827C0200000000005B
:1037600050658000EFB09700808F5000040031005A
:103770000140500004620200000000000400370015
:103780004FE9970002405000046202000000000070
:103790000000EB006065880090A2280040600200F5
:1037A000000000001200200051658000406580008C
:1037B000808F5000020032000200E000A0FB3200C7
:1037C000FFB1970053658800436588005DF83700B6
:1037D00080BA2000624078000004E00032FA320033
:1037E00035FA370080BA2000624078000004E0001B
:1037F0009AFA32009DFA370080BA200063417800BF
:10380000E0C3B300804F5100C8FF3200C520DD0087
:10381000E0CA200080804000DEFD3700881F78006D
:1038200055658000F40F20000480620083BA2000F8
:10383000E0C07900F0CCB30000C04000E84F500079
:103840001A003E000100FB0001FD2F0001014000B5
:103850000500E8000400600060C279008140420079
:1038600016002000E9CF500077003E00160020002F
:1038700001FD2F00F80F200087BA20006A11B9005F
:103880000400FB0002004000010140000603E800C4
:10389000068042000800600060C27B0001404200D8
:1038A000E94F500068003E00F4FF370000C3B3004A
:1038B00080CF500060003A000500E8000080FB0067
:1038C00081BA200060C2780020C6B300804F520049
:1038D0006100320020C4B300804F520012003A0051
:1038E0005D003700260020000001EB0003FD2F00E3
:1038F000F70F200084BA2000020041008100FB0085
:1039000001004000030140000603E8000680420079
:1039100007006000E0407A0003C04000E14F500023
:1039200049003E00F4FF370080C7B300804F5200CB
:103930001600320080C5B300804F520026003A00C6
:10394000120037004411DD00E9CF510005003E00B0
:103950000100FB000000410001FD2F0001014000BB
:1039600008003700014078000054A00081BA200010
:1039700000F278000000FB000000410091FA2F00E7
:10398000010140000603E800020037002600200085
:103990000001EB00068042000082FB0080BA20009C
:1039A000E440780000CDB30080C14000E9CF510071
:1039B000E4FF36007140500000C04000E54F500069
:1039C000E0FF3600F0C9B30000C04000E54F5000F2
:1039D000DCFF36001C00370000CDB3000040420081
:1039E000160020000001EB00E94F500016003E00D9
:1039F0008400FB0000FD2F00008140008000780063
:103A0000F80F200087BA20006A11B9000400FB00FB
:103A100002004000010140000603E80005004300E9
:103A20000800600060C27B0001404200E94F500086
:103A300005003E00F4FF370010002000606588009C
:103A40000001EB000F003700068042000080FB0001
:103A5000506588000B0037000580E8000080FB00FF
:103A600081BA2000E0C0780000CDB30000C0400063
:103A7000260020000001EB00E14F5000F2FF3E0065
:103A800098FF3700020078004F047800000006001D
:103A9000881F7800526580000200E8000080FB006B
:103AA00081BA2000E0C0780013002000A0C3B3005A
:103AB00080CF50000A003A000280E800F80F200092
:103AC000080060005065880054FF070080017800FE
:103AD000506580000000E900080060005065880023
:103AE000030078004F04780000000600881F78006B
:103AF000526580000200E8000080FB0081BA2000CF
:103B0000E0C078008001EB00B0C3B30080CF50006C
:103B10000A003A000280E800F80F20000800600068
:103B2000506588003DFF07008001780050658000E7
:103B30000000E9000800600050658800030078007C
:103B40004F04780000000600506580000000E80087
:103B50000081FB0080BA2000E240780080C7B300FB
:103B600080CF500003003A00526588001300200007
:103B70000C00370040C6B30080CF500003003A006D
:103B80005265880023002000060037008001EB000A
:103B900020C6B30080CF500002003A005265880072
:103BA000330020000300780000000600526580000A
:103BB00080BA2000E240780000C2B30080CF5000FD
:103BC00009003A00F40F200083BA200080407800FA
:103BD0000200E8000401600062C07900814F5000DB
:103BE000FBFF32005265880000000600889FBE007F
:103BF0008A9FBE008C1F7800506580000000E8009E
:103C00000080FB0050658800E8FF070003FF070005
:103C10000000E00042003A00180020000B032000E2
:103C2000CA922000084078000462020000000000F0
:103C300010AA280028600200000000000BC0B90094
:103C4000680050000A0040004060020000000000D0
:103C50000804E800E90F5400F2FF3A007101200067
:103C6000606D2000DC7C0200000000000000EB0022
:103C70006065880013002000820020008300780027
:103C8000030078004C0007000006E9000000E8008F
:103C9000E10F500005003E00E1002000D06E200042
:103CA000DC7C0200000000003B0037004B8120005C
:103CB0001B007800080320000880B9002002B00033
:103CC000CA92200060007D0000000100C07A02005E
:103CD000000000008C0D780008E4B9007E04440068
:103CE00068007D000000010080A8280040600200FC
:103CF000000000000C00E00004003200C222A80016
:103D000040AA28004060020000000000510020008E
:103D100050572000DC7C0200000000001E0037002D
:103D20000006E900E70F560017003C004B81200019
:103D30001B007800080320000880B9002002B000B2
:103D4000CA92200060007D0000000100C07A0200DD
:103D5000000000008C0D780008E4B9007E044400E7
:103D600068007D00000001000C00E000010032004E
:103D7000C222A8005100200050572000DC7C020025
:103D8000000000000400370051012000C072200034
:103D9000DC7C020000000000406580000000E900BB
:103DA0000080FB00506588004F0678004F05BE007C
:103DB0004F04BE0000000600E8874700889FBE0051
:103DC0008A9FBE008C9FBE008E1F78000005BE003B
:103DD000820678000307780040AE280028600200C1
:103DE000000000000A00E00004003D0080AE280052
:103DF0002860020000000000030037000A4078003D
:103E00000462020000000000A0AE2800286002004A
:103E1000000000008004EB0009067800360037003F
:103E20000900E000050032008904E90000A1280033
:103E300028600200000000002F0037000C00E000A6
:103E40000600320000A128002860020000000000E7
:103E50008004EB00090678002700370070C0B3002B
:103E6000B4630200000000008004EB002200370071
:103E70000900E00005003A00D0C2B300B4630200BC
:103E8000000000001C0020001B00370070C0B300C1
:103E9000B463020000000000170037000E00E000CD
:103EA00046003A0000CDB30000404400E94F500006
:103EB0000E003E00E38F54000500340070C0B300D4
:103EC000B463020000000000490020000A0037002F
:103ED00008407800B46302000000000074805400C1
:103EE00008F07F008904E8000300370070C0B300C9
:103EF000B463020000000000A063020000000000A4
:103F000000447800ED4F50002E00320005003C00C8
:103F1000E84F5000C2FF3200EA4F5000E1FF3A0084
:103F200028003700D0C2B300804F5400D0FF3200C9
:103F300080C7B300804F5400DAFF3A00D7FF370044
:103F40000901E9000000EB000D0033000000EB0068
:103F50008000780005FD2F000202E8006A01B90028
:103F60007483570066C078000000FB000200400028
:103F7000050040008100E800848F5000F7FF3A0000
:103F8000808F550008003C00808F560006003500E9
:103F90000C00E00002003A00000578000E00370037
:103FA0000005EA000C003700B101200080EC200081
:103FB000DC7C02000000000087FF37000085EB007A
:103FC0000500370090A228004060020000000000B9
:103FD0000900E000DAFF3A000A0078004F07780095
:103FE0004F06BE004F05BE004F04BE008F00B1005B
:103FF00000000600881F7800D0AE2800286002006C
:1040000000000000E0C2B300B46302000000000042
:10401000A081200010407800B4630200000000007E
:1040200061812000F0442000910F100003003A004D
:10403000B0AF2800286002000000000090A2280015
:10404000406002000000000020B12800286002004B
:1040500000000000D1002000A0802000827C02002F
:1040600000000000A1BF2A000000EB00DA6202009D
:1040700000000000000478004800DE000462020036
:1040800000000000E0C2B300B463020000000000C2
:1040900008407800046202000000000090A228009E
:1040A0004060020000000000610020003076200027
:1040B000827C020000000000688120001800780067
:1040C00086620200000000007100200010EC200059
:1040D000827C020000000000C04080008662020076
:1040E00000000000D0B2280028600200000000009C
:1040F000F0442000980F100004003A00A0B32800FC
:10410000286002000000000003003700D0B3280040
:104110002860020000000000C1408000200423004D
:10412000808F50001000320004003E003000230059
:10413000808F500018003A00070037003004230039
:10414000808F50000C00320063004000808F5000D0
:1041500011003A000C00370000B42800286002006B
:10416000000000000F00370030B428002860020073
:10417000000000000B00370060B428002860020037
:10418000000000000700370090B4280028600200FB
:104190000000000003003700C0B4280028600200BF
:1041A0000000000000B52800406002000000000090
:1041B000E101200090762000DC7C0200000000007D
:1041C0004F047800000006005100200050922000AB
:1041D000827C020000000000C1BF2A000000EB004A
:1041E000DA620200000000008662020000000000A7
:1041F00061002000A0922000827C020000000000EC
:10420000E1BF2A000000EB00DA62020000000000BB
:10421000866202000000000090A2280040600200B8
:1042200000000000C100200070782000DC7C02004B
:104230000000000069000700C2C2BF000008A30020
:104240000500320011012000A0622000827C0200E3
:10425000000000000400370021012000B0632000AE
:10426000827C020000000000C0C2B300B463020000
:104270000000000000C2B300B463020000000000B0
:10428000CBC2BF000038A30005003200410120006E
:10429000705D2000827C02000000000004003700F6
:1042A00051012000205C2000827C02000000000000
:1042B000C0C2B300B46302000000000000C2B3003B
:1042C000B463020000000000A0AF2000104078009E
:1042D000704060000500320021022000307920008B
:1042E000DC7C02000000000004003700E101200037
:1042F000507B2000DC7C020000000000A0AF20000A
:10430000104078006840600005003A00B1012000CC
:10431000307D2000827C0200000000000400370095
:10432000C1012000E07E2000827C0200000000002D
:10433000C0C2B300B46302000000000000C2B300BA
:10434000B463020000000000B1012000B01A210097
:10435000827C02000000000090AE20001040780037
:10436000046202000000000090A2280040600200E9
:1043700000000000A0AF2000104078006340600003
:10438000E14F500005003A00510120000059200083
:10439000DC7C020000000000040037006101200006
:1043A000A0572000DC7C020000000000A04080003C
:1043B000020320000280B9006002B000C292200017
:1043C0006000790000000100C1002000707820002A
:1043D000DC7C02000000000000000600A1002000BC
:1043E00040072100DC7C0200000000006104200086
:1043F000C00C2100DC7C020000000000A1012000B4
:10440000E0072100827C020000000000A040800044
:10441000020320000280B9004002B000C2922000D6
:104420006000790000000100A10020008009210047
:10443000827C020000000000004020004F000700C6
:10444000001020004D000700002020004B00070056
:104450000004200049000700000820004700070072
:1044600090A22800406002000000000041002000EF
:1044700020112100827C02000000000021E3A8003E
:10448000A0C0B300FE7A020000000000B06202008B
:104490000000000011002000B0372000827C0200E4
:1044A0000000000090C0B300B463020000000000F0
:1044B00090C0B300FE7A020000000000B06202006B
:1044C0000000000011002000B0372000827C0200B4
:1044D0000000000090C0B300B463020000000000C0
:1044E000C0C0B300FE7A020000000000B06202000B
:1044F0000000000011002000B0372000827C020084
:104500000000000090C0B300B4630200000000008F
:10451000B0C0B300FE7A020000000000B0620200EA
:104520000000000011002000B0372000827C020053
:104530000000000090C0B300B4630200000000005F
:1045400021E3A90000402000170007000010200010
:1045500015000700002020001300070000042000C1
:1045600011000700000820000F00070090A228009B
:1045700040600200000000000000060041168000BC
:10458000808060000400320020B52800286002000E
:10459000000000000300370050B52800286002002A
:1045A00000000000000006005116800080806000BE
:1045B0000400320080B528002860020000000000DE
:1045C00003003700B0B5280028600200000000009A
:1045D00000000600881F7800506580000000E80099
:1045E0000080FB005065880070FD07008BFC070011
:1045F0000000E900E30F500002003E0090408800F8
:104600000D0037000004EB006865880021022000DF
:1046100070812000DC7C020000000000880178002E
:10462000420020001100200010002000E2FD0700E1
:104630000000E900904088002101200090832000C4
:10464000DC7C0200000000004F047800000006003F
:10465000881F7800506580000000E8000080FB00A3
:104660005065880051FD07006CFC07008040E900A0
:10467000E9CF500003003E0000812000014878008F
:104680000D0037000004EB0068658800D1082000A9
:1046900060872000DC7C02000000000088017800B8
:1046A000A20020001100200090002000C2FD0700A1
:1046B000018120008048E9000044EB0000812000D7
:1046C00091C0B30090CF100010003A0037FD0700F2
:1046D00052FC0700004478000004E0000B003A00A0
:1046E0000004EB0068658800E0B528004060020027
:1046F0000000000088017800F2FF270088007800A1
:1047000020022000ACFD0700004478004101200099
:1047100030902000DC7C020000000000110120002D
:10472000A0192100DC7C02000000000012630200DE
:10473000000000000004E000FCFF320000812000C7
:1047400091C0B30090CF100003003A0008407800F9
:10475000CA63020000000000F062020000000000D6
:1047600008C2B300A063020000000000884F5000A0
:10477000FCFF3A004F047800000006005752490041
:1047800054452000424954003A2020002A6E65001A
:1047900078742000636C6F00636B2000285E290032
:1047A000207769006C6C20007573650020746800C8
:1047B0006973200076616C0075654E006F2064009F
:1047C0006576690063652C002074720079202800EA
:1047D000414C4100524D29002053450041524300B5
:1047E00048206D00616372006F206600697273007B
:1047F0007441440044524500535320004D4143004E
:10480000524F200020302E004D616300726F200057
:104810006D656E00754D610063726F002020200091
:104820002020310057495200452061006464720025
:10483000657373000D0A200020202A0031574900BB
:1048400052452000524F4D0020434F004D4D410036
:104850004E4420004D414300524F73003A0D0A0070
:10486000203531002E52450041442000524F4D006A
:10487000202830007833330029202A00666F720028
:10488000207369006E676C006520640065766900BE
:1048900063652000627573000D0A200038352E0014
:1048A0004D41540043482000524F4D002028300015
:1048B0007835350029202A00666F6C006C6F770010
:1048C000656420006279200036346200697420003B
:1048D0006164640072657300730D0A002032300059
:1048E000342E53004B49500020524F004D202800D9
:1048F00030784300432920002A666F006C6C6F00FB
:10490000776564002062790020636F006D6D61003F
:104910006E640D000A20320033362E00414C4100F7
:10492000524D20005345410052434800202830009A
:1049300078454300290D0A0020323400302E530000
:104940004541520043482000524F4D00202830007E
:104950007846300029414C0041524D00205345001B
:104960004152430048202800307845004329530035
:104970004541520043482000283078004630290045
:104980004465760069636500204944007320610036
:104990007265200061766100696C6100626C65007F
:1049A00020627900204D410043524F002C207300BB
:1049B00065652000283029002E5245004144200022
:1049C000524F4D002028300078333300293A200020
:1049D0004D41540043482000524F4D0020283000E4
:1049E0007835350029534B0049502000524F4D0077
:1049F000202830007843430029556E006B6E6F000D
:104A0000776E20006D616300726F2C00207472005D
:104A100079203F00206F7200202830002920660096
:104A20006F72200068656C00704255005320520080
:104A3000455345005420570061726E00696E67004F
:104A40003A202A0053686F00727420006F722000B1
:104A50006E6F200070756C006C2D750070202A0040
:104A60004E6F200064657600696365002064650010
:104A7000746563007465640020445300313853004A
:104A8000323020004869670068205000726573006A
:104A90002044690067205400686572006D4453002B
:104AA000313842003230200050726F0067205200CF
:104AB00065732000446967002054680065726D00CA
:104AC0004453310038323200204563006F6E2000BD
:104AD000446967002054680065726D0044533200D9
:104AE00034303400204563006F6E7200616D200029
:104AF00074696D006520430068697000445332009A
:104B00003433310020314B002045450050524F00D6
:104B10004D556E006B6E6F00776E200064657600F9
:104B20006963650050574D0020646900736162003D
:104B30006C656400314B48007A2D34002C30300015
:104B4000304B48007A205000574D46007265710086
:104B500075656E0063792000696E20004B487A000D
:104B60002050720065736300616C65003A5052001A
:104B7000323A44007574790020637900636C6500F3
:104B800020696E002025200050574D0020616300F1
:104B90007469760065455200524F52003A20500029
:104BA000574D200061637400697665002C20670012
:104BB00020746F0020646900736162006C654100BD
:104BC0005558200046726500717565006E63790066
:104BD0003A20410055582000494E500055542F00AE
:104BE00048492D005A41550058204800494748007F
:104BF00041555800204C4F0057564F004C544D0023
:104C00004554450052204D004F444500564F4C003E
:104C10005441470045205000524F4200453A200081
:104C200056457200726F720028292000406C69009E
:104C30006E653A0020407000676D7300706163001C
:104C4000653A20006279740065732E00546F6F001E
:104C5000206C6F006E67210053796E0074617800DC
:104C600020657200726F72004E6F20004545500043
:104C7000524F4D004572610073696E0067646F00AA
:104C80006E655300617669006E672000746F2000C6
:104C9000736C6F00742049006E7661006C6964006B
:104CA00020736C006F744C006F616400696E670064
:104CB000206672006F6D2000736C6F0074204500D9
:104CC00052524F00523A2000636F6D006D616E00CA
:104CD00064206800617320006E6F200065666600C6
:104CE000656374002068650072654100434B4E00A7
:104CF00041434B0049324300205354004152540079
:104D0000204249005449320043205300544F500080
:104D1000204249005449320043206D006F64650011
:104D20003A0D0A0020312E0020536F006674770080
:104D3000617265000D0A2000322E20004861720069
:104D400064776100726553006574200073706500BC
:104D500065643A000D0A2000312E20007E354B009C
:104D6000487A0D000A2032002E207E0035304B009C
:104D7000487A0D000A2033002E207E0031303000AA
:104D80004B487A000D0A2000342E20007E3430007B
:104D9000304B48007A574100524E49004E473A0086
:104DA00020484100524457004152450020493200FA
:104DB0004320690073206200726F6B00656E2000F3
:104DC0006F6E200074686900732050004943210011
:104DD00020285200455620004133290053657400B5
:104DE00020737000656564003A0D0A0020312E00C2
:104DF00020313000304B48007A0D0A0020322E005E
:104E000020343000304B48007A0D0A0020332E0049
:104E100020314D00487A490032432000286D6F0050
:104E200064207300706429003D28200020302E008B
:104E30004D616300726F20006D656E00750D0A0094
:104E400020312E00376269007420610064647200B2
:104E5000657373002073650061726300680D0A005A
:104E600020322E004932430020736E0069666600CE
:104E70006572530065617200636869006E672000A7
:104E8000493243002061640064726500737320003E
:104E90007370610063652E0020466F00756E6400BC
:104EA00020646500766963006573200061743A00D0
:104EB000536E6900666665007228420041534900DE
:104EC000432952006561640079612F00412F400041
:104ED00020636F006E7472006F6C73002041550088
:104EE00058207000696E61002F412F004020630040
:104EF0006F6E7400726F6C0073204300532070005B
:104F0000696E43006F6D6D00616E6400206E6F000E
:104F1000742075007365640020696E002074680059
:104F2000697320006D6F6400655075006C6C2D0016
:104F30007570200072657300697374006F7273007E
:104F4000204F4600465075006C6C2D007570200097
:104F500072657300697374006F727300204F4E00A6
:104F600053656C00662D74006573740020696E00D3
:104F7000204869005A206D006F646500206F6E0044
:104F80006C7952004553450054424F004F544C0039
:104F90004F4144004552410055582000494E5000B1
:104FA00055542F0048492D005A2C200052454100ED
:104FB000443A2000504F57004552200053555000AE
:104FC000504C4900455320004F4E50004F5745006C
:104FD00052205300555050004C49450053204F007B
:104FE000464644004154410020535400415445007A
:104FF0003A204400454C4100592075007357520037
:10500000495445003A205200454144003A204300AB
:105010004C4F43004B2C200031434C004F434B007E
:105020002C2030004441540041204F005554500082
:1050300055542C002031440041544100204F55006C
:1050400054505500542C200030202A0070696E0006
:1050500020697300206E6F0077204800695A430072
:105060004C4F43004B20540049434B00533A20001F
:10507000524541004420420049543A0020537900EF
:105080006E7461007820650072726F00722061009A
:10509000742063006861720020782E00206578001B
:1050A0006974280077697400686F75007420630064
:1050B00068616E00676529006E6F20006D6F640087
:1050C0006520630068616E00676523003A204E002A
:1050D0006F2073006F667400776172006520720044
:1050E0006573650074206F006E207600342C2000FC
:1050F0007573650020746800652072006573650033
:1051000074206200757474006F6E2E004E6F6E0016
:1051100065786900737465006E74200070726F00AA
:10512000746F63006F6C2100782E20006578690031
:10513000740D0A00496E7600616C6900642063009A
:10514000686F690063652C0020747200792061002B
:10515000676169006E444500564944003A6874002E
:1051600074703A002F2F6400616E670065726F00E3
:1051700075737000726F74006F74790070657300DE
:105180002E636F006D2A2D002D2D2D002D2D2D004D
:105190002D2D2D002A4F7000656E20006472610075
:1051A000696E20006F75740070757400732028009C
:1051B000483D4800692D5A002C204C003D474E00C8
:1051C00044294E006F726D00616C20006F75740091
:1051D0007075740073202800483D33002E3376002C
:1051E0002C204C003D474E0044294D0053422000E6
:1051F000736574003A204D004F53540020736900CA
:1052000067206200697420006669720073744C0044
:1052100053422000736574003A204C00454153000E
:105220005420730069672000626974002066690079
:105230007273740020426F006F746C006F616400C1
:1052400065722000762031002E20480045580D0060
:105250000A2032002E20440045430D000A2033006E
:105260002E204200494E0D000A2034002E2052000C
:1052700041574400697370006C61790020666F00CB
:10528000726D610074207300657456006F6C740059
:1052900061676500206D6F006E6974006F72730046
:1052A0003A203500563A2000207C2000332E33006F
:1052B000563A2000207C2000565055004C4C55009A
:1052C000503A2000536574002073650072696100D4
:1052D0006C2070006F72740020737000656564004C
:1052E0003A20280062707300290D0A0020312E0038
:1052F00020333000300D0A0020322E0020313200E1
:1053000030300D000A2033002E20320034303000BF
:105310000D0A2000342E200034383000300D0A00F1
:1053200020352E002039360030300D000A2036009E
:105330002E20310039323000300D0A0020372E0087
:1053400020333800343030000D0A2000382E200081
:105350003537360030300D000A2039002E2031005C
:105360003135320030300D000A3130002E2042003D
:105370005247200072617700207661006C756500ED
:1053800041646A007573740020796F0075722000A3
:10539000746572006D696E00616C41007265200079
:1053A000796F75002073750072653F0020434600D9
:1053B00047313A002043460047323A00285C2D002E
:1053C0002F5F5C002D2928005C5F2F002D295300E2
:1053D000656C6500637420006F75740070757400EF
:1053E0002074790070653A000D0A2000312E2000EB
:1053F0004F7065006E206400726169006E202800A5
:10540000483D4800692D5A002C204C003D474E0075
:1054100044290D000A2032002E204E006F726D00CC
:10542000616C200028483D00332E3300562C2000AC
:105430004C3D47004E44290052325700202873004B
:105440007064200068697A00293D2800202030001F
:105450002E4D610063726F00206D65006E750D004A
:105460000A2031002E4953004F37380031362D00C5
:105470003320410054520D000A2032002E495300BF
:105480004F37380031362D003320700061727300C1
:1054900065206F006E6C790049534F00203738004B
:1054A00031362D003320410054522000285245004F
:1054B00053455400206F6E0020435300290D0A000D
:1054C000524553004554200048494700482C2000CD
:1054D000434C4F00434B2000544943004B2C2000C9
:1054E00052455300455420004C4F570049534F003C
:1054F0002037380031362D003320720065706C0083
:10550000792028007573650073206300757272003E
:10551000656E7400204C5300422073006574740063
:10552000696E6700293A200050726F00746F630043
:105530006F6C3A0020736500726961006C33200063
:105540007769720065322000776972006552460003
:1055500055756E006B6E6F00776E5200656164006A
:105560002074790070653A0020746F0020656E0029
:105570006476610072696100626C6500206C650090
:105580006E6774006844610074612000756E690084
:1055900074733A00206E6F0020696E0064696300C6
:1055A000617469006F6E44006174610020756E0063
:1055B000697420006C656E006774680020286200C2
:1055C00069747300293A200043532000454E41007E
:1055D000424C45004443530020444900534142009B
:1055E0004C4544005233570020287300706420005B
:1055F00063736C00206869007A293D002820290027
:105600000D0A4400697363006F6E6E006563740079
:1056100020616E007920640065766900636573001F
:105620000D0A43006F6E6E006563740020285600FB
:1056300070752000746F20002B3556002920610002
:105640006E64200028414400432074006F202B002A
:10565000332E33005629430074726C0041555800B4
:105660004D4F440045204C0045445000554C4C00E3
:1056700055502000485055004C4C550050204C00CF
:105680005652450047414400432061006E642000AB
:1056900073757000706C79003556560050553300A4
:1056A0002E33560041444300427573002068690060
:1056B000676842007573200048692D005A20300049
:1056C00042757300204869002D5A2000314D4F006B
:1056D00044452000616E640020565200454720007A
:1056E0004C45440073207300686F75006C642000A3
:1056F000626520006F6E2100466F75006E642000A9
:1057000020657200726F7200732E4D004F53490076
:10571000434C4B004D4953004F435300204F4B0027
:1057200020464100494C53006574200073706500A9
:1057300065643A000D0A2000312E200033304B0002
:10574000487A0D000A2032002E20310032354B00FD
:10575000487A0D000A2033002E20320035304B00ED
:10576000487A0D000A2034002E2031004D487A007E
:10577000436C6F00636B2000706F6C006172690096
:1057800074793A000D0A2000312E200049646C0023
:1057900065206C006F7720002A64650066617500E3
:1057A0006C740D000A2032002E204900646C6500E4
:1057B0002068690067684F00757470007574200078
:1057C000636C6F00636B200065646700653A0D00D1
:1057D0000A2031002E204900646C650020746F009F
:1057E0002061630074697600650D0A0020322E0086
:1057F0002041630074697600652074006F206900A1
:10580000646C6500202A640065666100756C740034
:10581000496E70007574200073616D00706C6500D6
:1058200020706800617365003A0D0A0020312E0077
:10583000204D690064646C0065202A006465660080
:1058400061756C00740D0A0020322E0020456E0038
:1058500064535000492028007370640020636B007B
:10586000702073006B652000736D700020637300FF
:105870006C206800697A29003D28200020302E0025
:105880004D616300726F20006D656E00750D0A003A
:1058900020312E00536E69006666200043532000BD
:1058A0006C6F77000D0A2000322E53006E6966007F
:1058B000662061006C6C200074726100666669008D
:1058C000632D7000202D6600202A42007974650047
:1058D00073206400726F7000706564002A46410096
:1058E000494C4500442C20004E4F200044415400B8
:1058F000414461007461200062697400732061009A
:105900006E64200070617200697479003A0D0A00BB
:1059100020312E0020382C00204E4F004E45200014
:105920002A646500666175006C7420000D0A200011
:10593000322E2000382C2000455645004E200D0008
:105940000A2033002E2038002C204F004444200031
:105950000D0A2000342E2000392C20004E4F4E001E
:10596000455374006F70200062697400733A0D0033
:105970000A2031002E203100202A64006566610073
:10598000756C74000D0A2000322E20003252650022
:105990006365690076652000706F6C006172690054
:1059A00074793A000D0A2000312E200049646C0001
:1059B00065203100202A640065666100756C740002
:1059C0000D0A2000322E200049646C006520300052
:1059D0005541520054202800737064002062720008
:1059E000672064006270200073622000727870008B
:1059F000206869007A293D0028202000302E4D00C3
:105A0000616372006F206D00656E75000D0A2000E5
:105A1000312E540072616E007370610072656E0009
:105A2000742062007269640067650D000A2032000C
:105A30002E4C6900766520006D6F6E0069746F00F2
:105A4000720D0A0020332E004272690064676500FF
:105A50002077690074682000666C6F00772063000F
:105A60006F6E7400726F6C000A0D2000342E4100BE
:105A700075746F00204261007564200044657400F5
:105A800065637400696F6E005541520054206200D6
:105A90007269640067655200657365007420740064
:105AA0006F206500786974005261770020554100CD
:105AB00052542000696E70007574550041525400B4
:105AC000204C49005645200044495300504C4100A9
:105AD000592C20007D2054004F205300544F50007B
:105AE0004C49560045204400495350004C41590050
:105AF000205354004F5050004544570041524E002F
:105B0000494E47003A207000696E7300206E6F00A6
:105B100074206F0070656E002064720061696E0011
:105B200020284800695A290020524500564944005F
:105B30003A0D0A00496E7600616C690064206300CA
:105B4000686F690063652C00207472007920610021
:105B5000676169006E6D7300525320004C4F57000F
:105B60002C2043004F4D4D00414E4400204D4F002E
:105B70004445520053204800494748002C20440027
:105B800041544100204D4F0044454100646472007F
:105B900065737300206F660020504300463835005F
:105BA00037343F005468690073206D006F646500EE
:105BB00020726500717569007265730020616E0066
:105BC000206164006170740065724C0043442000E1
:105BD00074797000653A0D000A2031002E204800CB
:105BE00044343400373830002028750073696E0063
:105BF00067205000434638003537340020494F00B5
:105C00002065780070616E0064657200294C430065
:105C100044202800747970002061640064722900B7
:105C2000203D200028202000302E4D0061637200AE
:105C30006F206D00656E75000D0A2000312E4C003E
:105C4000434420005265730065740D000A20320041
:105C50002E496E00697420004C4344000D0A200058
:105C6000332E43006C65610072204C0043440D00EC
:105C70000A2034002E43750072736F00722070008A
:105C80006F73690074696F006E206500783A2800B0
:105C900034292000300D0A0020362E00577269008A
:105CA000746520007465730074206E00756D620069
:105CB00065727300206578003A2836002920380084
:105CC000300D0A0020372E005772690074652000DD
:105CD000746573007420630068617200616374000E
:105CE00065727300206578003A2837002920380053
:105CF0003044690073706C00617920006C696E003B
:105D000065733A000D0A2000312E200031200D006D
:105D10000A2032002E204D00756C740069706C00F2
:105D200065494E00495443004C45410052435500DB
:105D300052534F005220530045544E006F204100F3
:105D4000434B2C002063680065636B002061640096
:105D500061707400657243004C4B09004D4F530055
:105D60004909430053094D0049534F0050696E00E3
:105D700073746100746573003A474E004409330040
:105D80002E33560009352E00305609004144430099
:105D90000956500055094100555809005009500056
:105DA0000950090049094900092D09004F574400CD
:105DB000092D09002D2D090054784400092D0900F2
:105DC0005278440053434C000953440041092D00CC
:105DD000092D50004743090050474400092D090090
:105DE0002D312E0028425200290932002E2852005F
:105DF00044290900332E28004F52290009342E006F
:105E000028595700290935002E2847004E29090036
:105E1000362E2800424C290009372E002850550004
:105E2000290938002E28470052290900392E280058
:105E30005754290009302E0028426C006B29470076
:105E40004E440900474E44000941440043093500CF
:105E50002E30560009332E00335609005650550097
:105E6000094155005809650078656300757465003F
:105E7000203A200020617500746F7200616E670027
:105E800065202B004D487A00292B6B00487A2900A9
:105E900052617700207661006C75650020666F00A6
:105EA0007220420052472000284D490044493D00DD
:105EB0003132370029574100524E49004E473A00CF
:105EC00020506F0073736900626C6500206275007A
:105ED00066666500726F7600657266006C6F7700AB
:105EE000416E7900206B6500792074006F20650099
:105EF000786974005370610063652000746F20003E
:105F0000636F6E0074696E0075654E00756D62009A
:105F1000657220006F662000626974007320720051
:105F2000656164002F777200697465003A20430050
:105F3000533A0D000A2031002E204300530D0A0071
:105F400020322E00202F430053202A006465660073
:105F500061756C0074506F0073697400696F6E0036
:105F600020696E00206465006772650065735300E8
:105F7000657276006F206100637469007665570072
:105F800061697400696E670020616300746976005E
:105F9000697479002E2E2E002A2A20004561720095
:105FA0006C7920004578690074212A002A4261003A
:105FB00075643E0031366D003A20420050204300A7
:105FC000616E6E006F7420006D6561007375720004
:105FD00065203E0020313600303030003030300057
:105FE0002C2044006F6E65002E0A0D0043616C008A
:105FF00063756C0061746500643A2000090A0D0045
:1060000045737400696D6100746564003A20200076
:10601000092062007073200047656E0065726100A0
:106020006C0909000909090050726F00746F630060
:106030006F6C2000696E74006572610063746900A2
:106040006F6E20002D2D2D002D2D2D002D2D2D00BE
:106050002D2D2D002D2D2D002D2D2D002D2D2D0024
:106060002D2D2D002D2D2D002D2D2D002D2D2D0014
:106070002D2D2D002D2D2D002D2D2D002D2D2D0004
:106080002D2D2D002D2D2D002D2D2D002D2D2D00F4
:106090002D2D2D002D2D2D002D2D2D002D2D2D00E4
:1060A0002D2D2D002D2D2D00203F09005468690055
:1060B00073206800656C7000090909002830290008
:1060C000094C6900737420006375720072656E007C
:1060D00074206D00616372006F7320003D582F00C3
:1060E0007C580900436F6E0076657200747320005F
:1060F000582F72006576650072736500205809009C
:106100000928780029094D00616372006F2078002A
:10611000207E090053656C00667465007374090085
:1061200009095B000953740061727400202309009F
:106130005265730065742000746865002042500049
:1061400020202000090909005D095300746F7000C8
:10615000202409004A756D00702074006F206200D1
:106160006F6F74006C6F61006465720009097B00D9
:10617000095374006172740020776900746820000C
:1061800072656100642026002F25090044656C00BB
:106190006179200031207500732F6D0073090900AB
:1061A000097D090053746F00702061002F412F009A
:1061B0004009410055585000494E2000286C6F009E
:1061C000772F4800492F5200454144002909090012
:1061D000226162006322090053656E00642073002F
:1061E000747269006E6720006209530065742000B4
:1061F000626175006472610074650900090931000B
:1062000032332000632F43000941550058206100BC
:1062100073736900676E6D00656E740020286100FD
:1062200075782F0043532900090930007831320076
:10623000332064002F4409004D65610073757200BE
:106240006520410044432000286F6E0063652F00E5
:10625000434F4E00542E2900093062003131300086
:10626000095365006E64200076616C00756520003E
:1062700066094D00656173007572650020667200E5
:1062800065717500656E6300790909007209520035
:106290006561640020672F0053094700656E650043
:1062A0007261740065205000574D2F0053657200D5
:1062B000766F0900092F0900434C4B0020686900E4
:1062C00020680900436F6D006D616E0064686900AD
:1062D00073746F007279090009095C0009434C006E
:1062E0004B206C006F2069000956650072736900CD
:1062F0006F6E69006E666F002F73740061747500B5
:1063000073696E00666F0900095E0900434C4B001B
:1063100020746900636B20006C2F4C0009426900F7
:10632000746F72006465720020286D0073622F0024
:106330004C534200290909002D0944004154200012
:10634000686920006D09430068616E006765200080
:106350006D6F640065090900095F0900444154003C
:10636000206C6F00206F090053657400206F75006A
:106370007470750074207400797065000909090053
:106380002E094400415420007265610064207000B1
:106390002F50090050756C006C75700020726500FC
:1063A00073697300746F7200732028006F66660053
:1063B0002F4F4E0029092100094269007420720004
:1063C0006561640020730900536372006970740092
:1063D00020656E0067696E0065090900093A0900C9
:1063E000526570006561740020652E00672E2000E4
:1063F000723A310030207600095368006F77200030
:10640000766F6C0074732F00737461007465730091
:1064100009093B000942690074732000746F200071
:1064200072656100642F77007269740065206500F1
:106430002E672E002030780035353B003220770063
:106440002F5709005053550020286F0066662F0013
:106450004F4E290009093C00783E2F003C783D0052
:10646000203E2F003C303E000955730065726D00E0
:10647000616372006F2078002F6173007369670099
:106480006E2078002F6C690073742000616C6C00C2
:106490000000EB0080088800F0088800E00C88000D
:1064A000225D80000200E00006003A00CAC6BF007C
:1064B00001CEB30001406000CAE6B700125C88005C
:1064C0002E003700E30F510004003C0010A1A8008B
:1064D0001081A800E003200010003700FE0F5100DB
:1064E00004003C0010A1A8001081A900A00F20000A
:1064F0000A003700400F2000800F510004003C00CC
:1065000010A1A9001081A800007D20000300370021
:1065100010A1A9001081A90000E8230011000900C2
:106520000280D8000000E90060088800325D800029
:106530000280B90042062000110009000280D80044
:10654000A26C20001241780003CEB3000341610029
:106550006241B3000001FD00CAE6B7000001FD0082
:10656000D00C8800C00C880060002000E00C88007F
:1065700011E1A80020002000105C88000000060047
:10658000889FBE008A9FBE008C1F78000004EB002D
:1065900088088800F8088800E80C8800105C8000F3
:1065A000E20F500010003A00CAC6BF0001CEB3008F
:1065B00001406000CAE6B700C1002000E02B2000C7
:1065C000DC7C020000000000185C88005065800040
:1065D0000000E8000080FB0081BA200060C0780065
:1065E0000004E0008B003200506580000000E800ED
:1065F0000080FB0050658800D61D020000000000EE
:106600000E1C02000000000000047800D61D0200ED
:10661000000000000E1C020000000000CF80DE0021
:1066200000040200000000000005BE000001EB00B5
:106630008800E900E0F92000808F500001003E0052
:1066400012002000820478006011B8000A00BE0029
:1066500056040200000000000000E00008003400C2
:1066600002002000832C24000A00BE005A0402000D
:10667000000000000000E00001003D008904E80087
:10668000E28F5400110032000004EB0068658800BE
:1066900011012000A02C2000DC7C02000000000082
:1066A00011012000B02D2000827C020000000000BB
:1066B0008801780002FA2000110020002003200049
:1066C000DC1E02000000000000047800E30F54000C
:1066D00004003E0010A1A8001081A800E0032000E3
:1066E00010003700FE0F540004003E0010A1A80067
:1066F0001081A900A00F20000A003700400F2000E1
:10670000800F540004003E0010A1A9001081A800D1
:10671000007D20000300370010A1A9001081A9000E
:1067200000E82300110009000880D8000006E900F5
:10673000E28F54000E00320001012000902F200053
:10674000827C0200000000008001EB003206200085
:106750008300780020032000DC1E020000000000FF
:10676000CF80DE0000040200000000000005BE0033
:1067700002002000832C24000A00BE005E040200F8
:10678000000000000004BE006160B90000040200C7
:10679000000000000C00E00004003D0002002000AA
:1067A00003782400E4040200000000000001BE00A1
:1067B0000800BE009E050200000000000606020060
:1067C00000000000A26C20001241780003CEB3004C
:1067D000034161006241B3000001FD00CAE6B70059
:1067E0000001FD00D00C8800C00C88006000200073
:1067F000E00C88006C08880011E1A800A1002000CE
:1068000090302000DC7C020000000000200020000E
:10681000105C88004F0678004F05BE004F04BE0094
:1068200000000600889FBE008A9FBE00105C8000AA
:10683000E20F500005003A00F10120003031200045
:10684000DC7C02000000000019023700F10020008B
:1068500020332000827C0200000000000004EB00D6
:10686000F808880088088800C942A80086C6BF00CA
:1068700001CEB30001406000A040B30086E6B7003F
:10688000A0032000800888002C0207000002BE0040
:106890000803780088037800F0FF2300010020003F
:1068A0006011B8000020E10001A8E10002B0E100A1
:1068B00003B8E1000D0036000605BE000404BE006A
:1068C000C85DDD004850DE008B0570004855DD00D6
:1068D0004848DE000A057000C84CDD004840DE0074
:1068E000890470004844DD0009003700B100200031
:1068F000A0132100827C020000000000A000200004
:10690000800888000D0207000004BE006055B80032
:10691000F0F92000010020006011B8000040E10003
:1069200001C8E10002D0E10003D8E1000700360011
:106930000800BE00F060020000000000E0BB28007C
:106940004060020000000000D4013700E00F540056
:10695000E08F5C00E00F5D00E08F5D00CC01320055
:10696000B1002000A0132100827C02000000000082
:1069700008007800120207000002BE006033B80071
:1069800000A82100610020006011B8000020E10093
:1069900001A8E10002B0E10003B8E1006A0036009E
:1069A000E00F5200E08F5A00E00F5B00E08F5B00C9
:1069B000050035000400BE000601BE003C060200D2
:1069C000000000001400370010002000010020002B
:1069D0006011B8000400600085806000060161005D
:1069E000878161008703D1000683D3008582D300AD
:1069F0000482D300000072008180720002017300E3
:106A0000838173003C060200000000000001BE000C
:106A1000E4040200000000000001BE00703B2400FE
:106A2000A13B25005E04020000000000B406020045
:106A3000000000000205BE000004BE00046A280039
:106A4000150020006033B800EA07020000000000D3
:106A5000F060020000000000E0C2B300B463020076
:106A600000000000046A2800150020006033B80010
:106A70000800BE000A01BE00F80702000000000086
:106A80000205BE000004BE00F070220001002000DC
:106A90006011B8000040E10001C8E10002D0E1004F
:106AA00003D8E10003003E0000C3B300B46302005A
:106AB00000000000703E2000010020006011B800BE
:106AC0000040E10001C8E10002D0E10003D8E1008C
:106AD00003003E0000C3B300B463020000000000E6
:106AE00030062000010020006011B8000040E100E5
:106AF00001C8E10002D0E10003D8E10003003E003C
:106B000000C3B300B4630200000000009000200046
:106B1000010020006011B8000040E10001C8E10060
:106B200002D0E10003D8E10003003E0000C3B3003F
:106B3000B4630200000000000800BE008A6002008A
:106B4000000000004E013700B0E12E0011002000CF
:106B50006011B8000020E10001A8E10002B0E100EE
:106B600003B8E1005F003600E00F5200E08F5A00EA
:106B7000E00F5B00E08F5B00050035000400BE0005
:106B80000601BE003C0602000000000014003700B1
:106B900010002000010020006011B8000400600017
:106BA0008580600006016100878161008703D10054
:106BB0000683D3008582D3000482D30000007200D4
:106BC0008180720002017300838173003C06020021
:106BD000000000000001BE00E4040200000000000C
:106BE0000001BE00902F2000512125005E0402000C
:106BF00000000000B4060200000000000205BE0014
:106C00000004BE0004712200050020006033B800BB
:106C1000EA07020000000000F0600200000000002F
:106C2000E0C2B300B463020000000000047122005F
:106C3000050020006033B8000800BE000A01BE0055
:106C4000F8070200000000000205BE000004BE00BC
:106C5000703E2000010020006011B8000040E100FB
:106C600001C8E10002D0E10003D8E10003003E00CA
:106C700000C3B300B463020000000000300620002F
:106C8000010020006011B8000040E10001C8E100EF
:106C900002D0E10003D8E10003003E0000C3B300CE
:106CA000B4630200000000009000200001002000FA
:106CB0006011B8000040E10001C8E10002D0E1002D
:106CC00003D8E10003003E0000C3B300B463020038
:106CD0000000000008007800BA6102000000000017
:106CE000E700370000C42900010020006011B8004F
:106CF0000020E10001A8E10002B0E10003B8E100DA
:106D000054003600E00F5200E08F5A00E00F5B00A5
:106D1000E08F5B00050035000400BE000601BE00E8
:106D20003C060200000000001400370010002000A4
:106D3000010020006011B800040060008580600040
:106D400006016100878161008703D1000683D300BB
:106D50008582D3000482D30000007200818072001B
:106D600002017300838173003C06020000000000F2
:106D70000001BE00E4040200000000000001BE00AB
:106D800080B22600E10625005E040200000000003B
:106D9000B4060200000000000205BE000004BE00B0
:106DA000843E2000050020006033B800EA0702009E
:106DB00000000000F060020000000000E0C2B3002C
:106DC000B463020000000000843E200005002000A3
:106DD0006033B8000800BE000A01BE00F8070200D8
:106DE000000000000205BE000004BE0030062000C6
:106DF000010020006011B8000040E10001C8E1007E
:106E000002D0E10003D8E10003003E0000C3B3005C
:106E1000B463020000000000900020000100200088
:106E20006011B8000040E10001C8E10002D0E100BB
:106E300003D8E10003003E0000C3B300B4630200C6
:106E40000000000008007800BA61020000000000A5
:106E50008B00370090162300010020006011B8005D
:106E60000020E10001A8E10002B0E10003B8E10068
:106E700049003600E00F5200E08F5A00E00F5B003F
:106E8000E08F5B00050035000400BE000601BE0077
:106E90003C06020000000000140037001000200033
:106EA000010020006011B8000400600085806000CF
:106EB00006016100878161008703D1000683D3004A
:106EC0008582D3000482D3000000720081807200AA
:106ED00002017300838173003C0602000000000081
:106EE0000001BE00E4040200000000000001BE003A
:106EF00000C22B00E1EB24005E0402000000000051
:106F0000B4060200000000000205BE000004BE003E
:106F100044062000050020006033B800EA070200A4
:106F200000000000F060020000000000E0C2B300BA
:106F3000B4630200000000004406200005002000A9
:106F40006033B8000800BE000A01BE00F807020066
:106F5000000000000205BE000004BE0090002000FA
:106F6000010020006011B8000040E10001C8E1000C
:106F700002D0E10003D8E10003003E0000C3B300EB
:106F8000B4630200000000000840780004620200C0
:106F9000000000003A003700E00F5200E08F5A0076
:106FA000E00F5B00E08F5B00050035000400BE00D1
:106FB0000601BE003C06020000000000140037007D
:106FC00010002000010020006011B80004006000E3
:106FD0008580600006016100878161008703D10020
:106FE0000683D3008582D3000482D30000007200A0
:106FF0008180720002017300838173003C060200ED
:10700000000000000001BE00E404020000000000D7
:107010000001BE000068290081D124005E04020046
:1070200000000000B4060200000000000205BE00DF
:107030000004BE00A4002000050020006033B8005A
:10704000EA07020000000000F060020000000000FB
:10705000E0C2B300B463020000000000A4002000FE
:10706000050020006033B8000800BE000A01BE0021
:10707000F8070200000000000462020000000000A7
:10708000E0BB280040600200000000000300370061
:1070900020BC28004060020000000000F0C1B300E6
:1070A0008666B7000000EB00F008880080088800C2
:1070B0004F05BE004F04BE00000006000000EB00BC
:1070C000F008880080088800C942A80086C6BF0072
:1070D00001CEB30001406000A040B30086E6B700D7
:1070E000A00320008008880014000700F20F200091
:1070F000820F5000E08F5800050036004809DD007F
:10710000C801DE00830171004801DD000400370082
:10711000A000200080088800080007000001BE00D1
:10712000F0C1B3008666B7000000EB00F0088800ED
:10713000800888000200BE00000006000080EB000E
:1071400070088800600888000000EB004008880094
:1071500030088800B0088800A0088800800020005F
:10716000F0088800400F2000E0088800004022005E
:10717000D00888008780A9001FE1A80011E1A800BD
:1071800087C0BF000048A300FDFF320011E1A90045
:107190001FE1A90030088000405C880042088000A0
:1071A00003002000C011DD000200200000004100AB
:1071B000E0804900205C8800315C88000000060007
:1071C000889FBE008A9FBE008C9FBE00800678000C
:1071D00084A0A9008420A9008FC6BF0001CEB300FF
:1071E00001406000A040B3008FE6B7008EC6BF002C
:1071F00001406000A040B3008EE6B7000000EB0045
:10720000400888003008880080002000800888003E
:1072100011E1A80030002000300A8800300820006A
:10722000100A880042C1BF000038A30007003200E6
:10723000000A80006101B80042C1BF000038A3000D
:10724000FBFF3A00F25C8800035D880046C1BF0086
:107250000038A30007003200200A80006101B80056
:1072600046C1BF000038A300FBFF3A00D25C880093
:10727000E35C880042C1BF000038A300FDFF32007C
:10728000000A80006104B800D85C8800E95C8800CE
:10729000200A80006101B800925C8800A35C88002D
:1072A0006000B800505C8800615C88000002EB0060
:1072B000145D88000D00E00026003200040678000E
:1072C0000005BE0042C1BF000038A300FDFF320030
:1072D000000A80006103B800200A80006102B80043
:1072E0000200520083805A00C000DD000000200030
:1072F0000801530089815B00000041008180490042
:107300000A0540008B8548000C06E8008C8F56006B
:10731000030032000401BE000604BE00E9FF37008E
:10732000705C8800815C8800B45C8800C55C880063
:107330001D5D88005A5C88006B5C8800945C880046
:10734000A55C8800D65C8800E75C8800F65C880055
:10735000075D88000000EB00100A8800100A880012
:1073600011E1A9006169B800505C8000615C800097
:107370000C090200000000004F06BE004F05BE00D1
:107380004F04BE0000000600A0AF200010407800AF
:107390006340600002003A00C942A80001003700C3
:1073A000C8C2A800E100200010342000827C020046
:1073B0000000000000000600A0AF20001040780090
:1073C0006340600003003A00C942A900CB42A80014
:1073D00002003700C8C2A900CAC2A800810020006C
:1073E000F0342000DC7C02000000000000000600F9
:1073F000A0AF2000104078006340600003003A0016
:10740000C942A900CB42A90002003700C8C2A900A6
:10741000CAC2A9007100200070352000DC7C020087
:107420000000000000000600A0AF2000104078001F
:107430006340600007003A00C942A8000000000055
:1074400000000000CBC2BF004200DE0061406000CF
:1074500006003700C8C2A8000000000000000000BD
:10746000CAC2BF004600DE00614060000080FB0031
:1074700000000600889FBE008A1F78000004EB0011
:1074800088088800F8088800E80C8800105C8000F4
:10749000E20F500011003A00506580000000E80043
:1074A0000080FB0081BA200060C078000004E0008A
:1074B0000A003A00CAC6BF0001CEB3000140600016
:1074C000CAE6B700C1002000E02B2000DC7C0200EF
:1074D00000000000185C88006000370050658000E4
:1074E0000000E8000080FB0050658800D61D020007
:1074F000000000000E1C020000000000CF80DE0033
:1075000000040200000000000004BE006A65800064
:107510000A00E00006003A00020020004333240085
:1075200056040200000000000000E00011003400DA
:107530000004EB006865880031012000301E210046
:10754000DC7C02000000000088017800420B200073
:1075500088007800A0052000DC1E0200000000006A
:10756000CF80DE0000040200000000000004BE0026
:107570001AC0B30010A1A8001081A80002002C00BE
:10758000A35524000800BE005E04020000000000B5
:1075900002002400C34924009E05020000000000F0
:1075A0000200200083272400E40402000000000001
:1075B0000606020000000000A26C200012417800C4
:1075C00003CEB300034161006241B3000001FD003E
:1075D000CAE6B7000001FD00D00C8800C00C88008E
:1075E00060002000E00C8800204E20006008880029
:1075F00011E1A800C1002000601F2100DC7C020016
:107600000000000020002000105C8800E14F5500C1
:1076100012003A0013002000420B20008000EB0013
:107620000080EB00DC1E020000000000CF80DE00C6
:1076300000040200000000000004BE006011B80059
:107640005A040200000000000000E000C9FF3D00F5
:1076500070BE280040600200000000004F05780066
:107660004F04BE0000000600A0AF20001064A00080
:1076700080B02000104078006840600005003200B3
:10768000CAC2A900F0C2B300B46302000000000047
:1076900001003700CAC2A800A100200090AB200062
:1076A000DC7C02000000000000000600A0AF20000B
:1076B0001064A10080B02000104078006840600095
:1076C00005003200CAC2A900F0C2B300B4630200D0
:1076D0000000000001003700CAC2A800A10020007D
:1076E00090AB2000DC7C02000000000000000600DF
:1076F00080B0200010407800684060000500320033
:10770000CAC2A800F0C2B300B463020000000000C7
:1077100001003700CAC2A900B100200030AC20002F
:10772000DC7C0200000000000000060000C0EB004E
:10773000CA0107000080FB0000000600C701070027
:1077400000417800A0AF200001C4B30010C0600069
:107750008000EB00010032008280FB000100780015
:1077600000000600881F78000102200000CA2000E7
:10777000827C02000000000080AE20001040E80083
:10778000046202000000000000C2B300B463020003
:107790000000000088B020009840780061C06000C0
:1077A000046202000000000000C2B300B4630200E3
:1077B000000000001880FB000000D1006140600064
:1077C000046202000000000000C2B300B4630200C3
:1077D000000000001880FB004200DE0061406000F5
:1077E000046202000000000000C2B300B4630200A3
:1077F000000000001880FB004300DE0061406000D4
:10780000046202000000000000C2B300B463020082
:1078100000000000A0AF20001080FB004400DE004C
:1078200061406000046202000000000000C2B3007A
:10783000B4630200000000003100200020AE2000F0
:10784000827C0200000000004F0478000000060067
:10785000889FBE008A9FBE008C1F7800D61D020044
:10786000000000000E1C0200000000000004780070
:10787000D61D0200000000000E1C020000000000E7
:1078800080047800D61D0200000000000E1C0200DB
:107890000000000000057800D61D02000000000076
:1078A0000E1C02000000000080057800D61D0200BA
:1078B000000000000E1C020000000000000678001E
:1078C000D61D0200000000000E1C02000000000097
:1078D000000178000800E900E30F500002003600C4
:1078E0000004EB000200370080AE20000848E900E9
:1078F0000900E900E10F5000020036000004EB002F
:107900000500370081B020000940E90061406000B7
:107910001104A100914870000A00E900E10F500035
:10792000020036000004EB000600370081B02000A2
:107930000A40E90061406000004040001114A100CD
:10794000914870000B00E900E10F50000200360082
:107950000004EB000600370081B020000B40E90076
:10796000614060004200DD001124A10091487000D8
:107970000C00E900E10F5000020036000004EB00AB
:107980000600370081B020000C40E9006140600033
:107990004300DD001134A100914870000200E900AD
:1079A000E10F500008003E00A0AF2000E140610060
:1079B000C408DD00104178000244A10001487100B4
:1079C0000800E0005B003A008004EB006965880075
:1079D0007103200000BC2000DC7C020000000000DD
:1079E00089017800420020001100200010002000D2
:1079F000DC1E02000000000081AE20008048E9008B
:107A00005103200070BF2000DC7C02000000000059
:107A100089017800220020001100200010002000C1
:107A2000DC1E02000000000088B020000040E900D9
:107A3000614060001804A100184C7000310420005F
:107A4000C0C22000DC7C0200000000008901780038
:107A5000220020001100200020002000DC1E020077
:107A6000000000000040E90061406000004040006C
:107A70001814A100184C700011032000F0C620005B
:107A8000DC7C020000000000890178002200200058
:107A90001100200010002000DC1E02000000000089
:107AA0000040E900614060004200DD001824A100B0
:107AB000184C7000D1012000601C2100DC7C020009
:107AC0000000000089017800220020001100200041
:107AD00020002000DC1E0200000000000040E90041
:107AE000614060004300DD001834A100184C7000B4
:107AF000F1042000E0932000DC7C02000000000084
:107B000089017800220020001100200010002000D0
:107B1000DC1E020000000000A2AF200061406000F7
:107B20004400DD00924078000144A10000C97000CB
:107B3000010037000BFF0700A0AF20001064A10078
:107B40004F0678004F05BE004F04BE00000006003F
:107B500080AE20009080FB00E08120006140780032
:107B60007300070080B020001080FB004300DE009F
:107B7000614060004600DD00A12C200091407800AB
:107B80000164A10080C0700001007800CAE2B70063
:107B900000000600A300070000000600010020000E
:107BA000EF0F5000E08F580057003E0000600100CA
:107BB0000F003700130037001E0037005600370053
:107BC00051003700500037004F0037004E0037009B
:107BD0004D0037004C0037002200370024003700EA
:107BE00026003700280037002A0037002C00370015
:107BF0004103200000CC2000DC7C020000000000DB
:107C0000450037007100200070562000DC7C020027
:107C100000000000F1002000B0182100DC7C020010
:107C20000000000011C0B3000040EB00940007000A
:107C3000390037007100200070562000DC7C020003
:107C400000000000F1002000B0182100DC7C0200E0
:107C50000000000011C0B300014078008800070058
:107C60002D00370080B020001004A1000E00370066
:107C700080B020001004A0000B00370080B020006E
:107C80001014A1000800370080B020001014A000DC
:107C90000500370080B020001024A100020037004A
:107CA00080B020001024A00082B020001240780094
:107CB000E1406000C608DD0042C2BF000064A100D0
:107CC0000140700042E2B7009280FB000101D10048
:107CD0006141610043C2BF000004A1000240700086
:107CE00043E2B700C208DE00E1C0600081C040008E
:107CF00043C2BF000014A1000140700043E2B7007E
:107D000098FE07000400370041022000E01D20001B
:107D1000DC7C0200000000000000060001012000E1
:107D200040062100DC7C020000000000000006008C
:107D30000041780041E2A900A0AF20001040780087
:107D40007040600004003200CEE2A800CF02A8001C
:107D5000CEC2A80003003700CEE2A900CF02A900DE
:107D6000CEC2A900A8C6BF0001CEB300014060008A
:107D70007040B300A8E6B700C9C6BF00014060006C
:107D80007040B300C9E6B700C8C6BF00014060003C
:107D90000034A000C8E6B700CAC2A800C8C2A90043
:107DA000C902A900C8E2A800C922A9000280FB00FC
:107DB0001012880042A2A80082B020001240780071
:107DC000E1406000C608DD0042C2BF000064A100BF
:107DD0000140700042E2B7009280FB000101D10037
:107DE0006141610043C2BF000004A1000240700075
:107DF00043E2B700C208DE00E1C0600081C040007D
:107E000043C2BF000014A1000140700043E2B7006C
:107E10000000EB00201288000012880041E2A80058
:107E20000000060041E2A900F0C1B300A866B70057
:107E3000C9C6BF0001CEB30001406000C9E6B7006B
:107E4000C8C6BF0001406000C8E6B700CEE2A90086
:107E5000CF02A900CEC2A900000006000080FB00EE
:107E60004012880085C0BF000028A300FDFF32003B
:107E7000401280008540A9000080FB000000060041
:107E8000889FBE008A9FBE008C9FBE0080467800FF
:107E900081457800AC8120002063020000000000D2
:107EA000E0FF0700710007000D04E00007003A0042
:107EB00042E2A80062E2A8000600370060C0280085
:107EC0004060020000000000F3FF3700E1CF5600E1
:107ED00064003E0041E2A80061E2A80061003700B2
:107EE0000A04E00007003A00CAC2BF000068A3000D
:107EF00004003200D0C5B300786302000000000027
:107F00001AC0B30040C2BF000058A30028003A00C6
:107F100060C2BF0001C2B3000144600024003A0007
:107F20004012800080447800E14F550004003A0080
:107F3000B0C5B30078630200000000000845780077
:107F40000B04E000040032000980FB0066620200BE
:107F50000000000006003700C0C5B30078630200CF
:107F60000000000009407800786302000000000073
:107F700040138000004478000B04E0000A00320047
:107F800080C2B30078630200000000000880FB009C
:107F9000666202000000000090C2B3007863020035
:107FA00000000000020037007863020000000000BB
:107FB00040C2BF000068A30007003A0060C2BF00D3
:107FC0000068A30004003A00004020001C0060008C
:107FD0000D00320005003700004020001C0060004A
:107FE00002003A0052630200000000000000EB00B3
:107FF00000128800001388000B04E000AFFF3A0075
:10800000C222A9000D0037002E630200000000000C
:108010001A63020000000000E14F5000B0FF3A0078
:10802000A0630200000000000B04E0000300320027
:1080300070C1280040600200000000005A000700E4
:1080400080AE20009080FB00E0812000614078003D
:1080500037FF07004F06BE004F05BE004F04BE00AD
:10806000000006001AC0B300A6FF3700C8C2A8006F
:10807000C902A800C8E2A800C922A800AAC6BF0079
:1080800001CEB300014060006040B300AAE6B70033
:10809000AEC6BF00014060006040B300AEE6B7006E
:1080A000A8C6BF00014060009040B300A8E6B7003A
:1080B000A9C6BF00014060000034A000A9E6B700D7
:1080C000ACC6BF00014060007040B300ACE6B70032
:1080D000ADC6BF00014060000034A000ADE6B700AF
:1080E00080AE20009080FB00E0812000614278009B
:1080F0000482FB001412880081B020001140780037
:10810000E1416000C619DD0042C2BF00F6CBB300FA
:10811000064060000340700042E2B7001181FB009E
:108120000201D1006141610043C2BF00E5CFB3004D
:10813000054060000240700043E2B7008000EB00A1
:1081400021128800011288001413880062C2BF0047
:10815000064060000340700062E2B70063C2BF00E7
:10816000054060000240700063E2B7002113880000
:108170000113880041128800411388004322A9009E
:108180006322A9004362A80042A2A9006362A8007A
:1081900062A2A90040C2A90060C2A9004402A800CE
:1081A0006402A8000000060041E2A9004362A900A1
:1081B00061E2A9006362A900F0C1B300AA66B7003A
:1081C000AE66B700A866B700A966B700AC66B70090
:1081D000AD66B7000000060080C1280028600200DC
:1081E0000000000000000600889FBE008A9FBE00BD
:1081F0008C9FBE0011C0B30080AE20000148780003
:1082000080B020001004A1001014A0001024A100D0
:10821000A0AF20001044A000208220001040900059
:10822000C3FE0700ECFF07006CB02000A063020053
:108230000000000080417800004E78000080FB00C4
:10824000C400DE0050B0200001487800E4CF5000A8
:108250001D01320005003E000104E000080032006C
:10826000E1CF50004A013A0002013700E6CF50004A
:108270001C013200E8CF500045013A0025013700CB
:10828000E5CF51000A003E00E4CF51002E0031003E
:10829000E1CF5100120032000C003900E2CF510052
:1082A00011003200E3CF5100EE003A001300370016
:1082B000EDCF510016003200EECF51001B0032000E
:1082C000E6CF5100E7003A006C003700D5FE07000A
:1082D0004F06BE004F05BE004F04BE000000060062
:1082E000BDFF0700D1FF3700CCC2A90010C0B3000A
:1082F000B463020000000000CCFF3700CCC2A8002D
:1083000010C0B300B463020000000000C7FF3700D4
:1083100010C0B300B4630200000000008040EB0016
:1083200010C0B300D6FE0700C0FF370010C0B30076
:10833000B4630200000000008040EB0001407800C0
:10834000CFFE0700B9FF3700A06302000000000065
:108350004804DD00A0630200000000000080FB0074
:1083600000057400A0630200000000004804DD0066
:10837000A0630200000000000080FB008005740084
:1083800000002100800F550002003E00808F550044
:10839000030136000040EB00B4630200000000005F
:1083A000A2FF37008004EB00ED8020001D84440014
:1083B000A063020000000000004C78008904E8007F
:1083C000890F5500F9FF3A0040C0B3009C4F1000E0
:1083D00001003A00CAC2A9000A00E000070032000A
:1083E0000004EB0070408000684078009BFE0700AE
:1083F0000804E800880F5500FAFF3A00100020003A
:108400002C7C0200000000000B00E000090032009C
:108410008004EB00EA8020001A84440000C0EB00D6
:108420008EFE0700004C78008904E800898F550013
:10843000F9FF3A0040C0B3009C4F100001003A0021
:10844000CAC2A80010C0B300B4630200000000005C
:108450000B00E00075FF32000004EB00704080006C
:1084600068407800B4630200000000000804E800DF
:10847000888F55006DFF3200F8FF370010C0B30041
:10848000B46302000000000022C2BF000008A30085
:10849000FDFF320030118000004E7800E14F5000A7
:1084A0000A003200050039008002EB006055B80078
:1084B000E24F50000F0032006600370010C0B300DA
:1084C000B46302000000000058FF370010C0B30082
:1084D000B4630200000000000040EB00B46302003F
:1084E0000000000010C0B300B463020000000000F0
:1084F0004EFF370022C2BF000008A300FDFF32007C
:10850000341180004859DD00C851DE00830171003C
:108510004851DD000480FB000100200000057100CF
:10852000818571008502E800E38F5200F1FF36007B
:10853000044E78008002EB006044B80022C2BF0005
:108540000008A300FDFF3200341180004849DD001F
:10855000C841DE00830171004841DD000480FB005A
:108560000100200000047100818471008502E80090
:10857000E38F5200F1FF3600044E7800F2FF2F0027
:1085800003002000820F5500838F5D0008003E002D
:10859000820F5400838F5C0005003E000A004400F7
:1085A0008B804C00820F5000838F580004003600EF
:1085B0000040EB00B4630200000000001BFF370026
:1085C00010C0B300B463020000000000E00F5400CC
:1085D000E08F5C0015FF320000C2B3001FFE0700F1
:1085E000C855DE000B4078001CFE07000A407800EA
:1085F0001AFE07000040EB0018FE0700B4630200FB
:1086000000000000E10F5400E08F5C0007FF320023
:1086100080C2B30011FE07000B4078000FFE070078
:108620000A4078000DFE07000040EB000BFE07003B
:10863000B46302000000000062045400E0845C00A7
:108640000A05E800E00F5400E08F5C00F7FE3200FE
:10865000E1FF37000040EB00B463020000000000BF
:10866000F2FE37000040EB00B4630200000000009F
:10867000EEFE37006FC06100004EE80010C0B3008E
:10868000B46302000000000040B020000048EB008E
:108690001C04E000E5FE32000004780069B0200010
:1086A000A063020000000000ECFD0700B4630200BC
:1086B000000000001840E800004C7800994F50007E
:1086C000DAFE3100F6FF37000340780096800200A2
:1086D0000000000010C0B300B463020000000000FE
:1086E000D2FE370067C06100004E780081AE2000E6
:1086F000804878000080FB002182200060C0780064
:108700008BFD070010C0B300B4630200000000003E
:10871000C6FE370081B020001104A1001114A10091
:108720001124A100A0AF20001044A1000381FB0090
:108730000228A300010032001104A0000218A300C7
:108740000200320080B020001014A0000308A30033
:108750000200320080B020001024A0000238A300E4
:1087600002003A00A0AF20001044A00080AE20001C
:108770009080FB0020822000614078006CFD0700A3
:1087800010C0B300B463020000000000A7FE370071
:108790000040EB00B463020000000000A3FE3700BD
:1087A0000A00E00008FF3200FEFE3700881F780054
:1087B000A67F0200000000000004E0001A00320062
:1087C00032C2BF000038A300040032003100200094
:1087D00040CF2000827C02000000000032C2BF00B7
:1087E0000028A300040032003100200070CF2000D8
:1087F000827C0200000000009C7F0200000000005C
:108800000004780032C2BF000018A3000B00320041
:10881000F1002000A0CF2000827C020000000000B8
:108820003222A90005003700F100200090D020007E
:10883000827C0200000000000004EB0008007800C9
:108840004F04780000000600907F02000000000046
:108850000000EB0000000600881F780001022000E5
:10886000F0DB2000827C02000000000088AE2000C7
:1088700018407800046202000000000000C2B3004B
:10888000B46302000000000018407800E94F500077
:1088900007003A00C0118000BA6102000000000029
:1088A00000C2B300B46302000000000009003700FA
:1088B0000080FB0000004000E1AB200060807800F9
:1088C000BA6102000000000000C2B300B4630200FD
:1088D00000000000A8D520009840780063C0600028
:1088E000046202000000000000C2B300B463020092
:1088F000000000001880FB004200DE0061406000C4
:10890000046202000000000000C2B300B463020071
:10891000000000001880FB004300DE0061406000A2
:10892000046202000000000000C2B300B463020051
:1089300000000000A0AF20001080FB004400DE001B
:1089400061406000046202000000000000C2B30049
:10895000B4630200000000003100200020AE2000BF
:10896000827C0200000000004F0478000000060036
:10897000889FBE008A9FBE008C1F7800D61D020013
:10898000000000000E1C020000000000000478003F
:108990000006EB00EA0F500005003A00D61D020069
:1089A000000000000E1C020000000000000678001D
:1089B000D61D0200000000000E1C02000000000096
:1089C00080047800D61D0200000000000E1C02008A
:1089D0000000000000057800D61D02000000000025
:1089E0000E1C02000000000080057800D61D020069
:1089F000000000000E1C0200000000008001780052
:108A00000800E900E90F5000020036000004EB0006
:108A10000200370080AE20000848E9000900E900A4
:108A2000E30F5000020036000004EB0006003700A0
:108A3000A0D520008940E900E3C06000C2CFB300A8
:108A40001048610010C870000A00E900E10F5000F2
:108A5000020036000004EB0006003700A1D520001C
:108A60000A40E900614060004200DD001124A100DD
:108A7000914870000B00E900E10F50000200360041
:108A80000004EB0006003700A1D520000B40E900F0
:108A9000614060004300DD001134A1009148700086
:108AA0000300E900E10F500008003E00A0AF2000E5
:108AB000E1C06100C408DD00104178000244A1005B
:108AC000014871000800E0005B003A000004EB0080
:108AD00068658800D108200060872000DC7C0200E7
:108AE0000000000088017800A20020001100200092
:108AF00010002000DC1E0200000000000040E90021
:108B000081AE200080487800E94F50000B003A0009
:108B1000C1012000F0142100DC7C020000000000F4
:108B200088017800F2FF27001100200020022000B9
:108B3000DC1E020000000000C0118800410520007A
:108B400080D12000827C0200000000008001EB0048
:108B5000420020001100200010002000DC1E020056
:108B600000000000A8D520000040E900634060003C
:108B7000C1CFB30018CC6000184C70001102200067
:108B8000C0D62000827C0200000000008001EB00C3
:108B9000220020001100200010002000DC1E020036
:108BA000000000000040E900614060004200DD007C
:108BB0001824A100184C700021032000D0D82000F8
:108BC000827C0200000000008001EB0022002000F7
:108BD0001100200010002000DC1E02000000000038
:108BE0000040E900614060004300DD001834A1004E
:108BF000184C7000F1042000E0932000DC7C02009F
:108C0000000000008001EB00220020001100200085
:108C100010002000DC1E020000000000A2AF2000B7
:108C2000614060004400DD00924078000144A100F2
:108C300000C970000D00370080AE200091C0B30065
:108C400090CF100008003A006161B9000090200048
:108C5000D10320000C090200000000006100500058
:108C6000E0805800C0118800FBFE07004F06780026
:108C70004F05BE004F04BE000000060080AE20007D
:108C800090417800E9CF510010003A00C0118000F7
:108C9000A3D520001381FB004212DE004311DE0049
:108CA00061416100A1AF20009180FB00C408DE009B
:108CB000E1C060006142620093417800E3C161005D
:108CC000067F02000000000012003700A5D520003A
:108CD0001581FB004212DE004311DE00614161009C
:108CE000A0AF20009080FB00C408DE00E1C060005F
:108CF0000380FB0000004000E3AB200060807900AF
:108D00006142620095427800E3C16200067F020082
:108D100000000000A0D520001040780063406000F3
:108D2000E34F500003003A0091C0B30090AE200022
:108D300001487800707F020000000000C11180002F
:108D400040118000808F500004003100010220009B
:108D5000B0162100DC7C02000000000000000600CC
:108D60007A7F02000000000000000600889FBE001D
:108D700000047800E20F50005700320005003E006A
:108D80000000E00008003200E10F500079003A00D6
:108D90000E003700E30F500008003200E40F5000CF
:108DA00074003A0064003700A1062000F0DD2000C6
:108DB000827C02000000000072003700C062A9003F
:108DC000C082A800C8C2A800C902A900B100200042
:108DD00090E42000DC7C020000000000D1002000B4
:108DE00040E52000DC7C020000000000727D0200F3
:108DF000000000000000E000620032003222A90002
:108E0000D9FF2F0032C2BF000008A30005003200C6
:108E100023C2BF000018A30002003A00B011800076
:108E2000201188001A63020000000000E14F50008A
:108E300007003A0033C2BF000018A30004003A0044
:108E4000A0630200000000000080FB00A011880069
:108E500032C2BF000018A30003003A0022C2BF00C4
:108E60000018A300070032008004FD003222B60083
:108E70008004FD008004FD002222B6008004FD0075
:108E8000C222A900E30F5400DEFF3A00212C20008B
:108E900091407800C408DE00E1806000CBC2BF00D2
:108EA0000004A10001407000CBE2B700CAC2BF00BD
:108EB0004600DE00610060004300DD00212C200040
:108EC000914078000134A10080C07000010078005A
:108ED000C2E2B700CBFF3700E100200010E620001F
:108EE000DC7C020000000000F1002000B01821002E
:108EF000DC7C0200000000003222A90032C2BF0068
:108F00000008A3000500320023C2BF000018A30020
:108F100002003A00B0118000201188001A6302009C
:108F200000000000E14F5000F4FF3A00A06302008F
:108F300000000000130037007A7F020000000000EC
:108F40000000EB0092000700707F020000000000AC
:108F5000C111800040118000808F50000900310055
:108F600001022000B0162100DC7C0200000000009D
:108F70000400370041022000E01D2000DC7C0200DC
:108F8000000000004F04BE00000006003222A900CD
:108F9000A0D520001044A000A0AF20001024A00005
:108FA000C1012000F0E62000DC7C0200000000008F
:108FB00000000600A0D520001044A100A0AF2000B2
:108FC0001024A10041012000B0E82000DC7C020058
:108FD0000000000000000600881F78000004EB007D
:108FE0002C003700A0D520001040780070406000B1
:108FF0002500320060B72800406002000000000039
:109000006100200080662000827C020000000000D9
:1090100032C2BF000038A30004003200310020003B
:1090200040CF2000827C02000000000032C2BF005E
:109030000028A300040032003100200070CF20007F
:10904000827C0200000000009C7F02000000000003
:109050007C7B02000000000032C2BF000018A300A9
:1090600005003200F1002000A0CF2000827C020029
:10907000000000003222A90060B728004060020012
:1090800000000000020037009C7F0200000000008A
:1090900018002000A67F0200000000000004E0008D
:1090A000D0FF3A00080078004F0478000000060066
:1090B000B1002000B00A2100DC7C020000000000AA
:1090C000000006000000EB00F0088800800888001F
:1090D000810020008108880040088800300888004E
:1090E000B0088800A0088800F10888000000060089
:1090F00011E1A9001FE1A900F0C1B3008666B70025
:109100000000EB00F0088800800888003008880024
:1091100040088800000006000002BE001100200088
:10912000C0B728001001BE00840F5100858F590080
:1091300010003600C208DD0080B7280080804000A3
:1091400061BB9700F1BB9700060051008780590072
:109150008100D1000080D3000600400087804800D5
:10916000800F5200818F5A0007003E000601BE00AA
:10917000050037008100E80064004000EF8F5000D8
:10918000E8FF3A006011B8000200BE0000000600CF
:10919000889FBE008A9FBE008C9FBE00800678001C
:1091A000CAE2A900C8E2A8000000E00004003A00FA
:1091B0003101200020202100DC7C020000000000A2
:1091C000CA42E20007003D006300370000000000D3
:1091D000CA42E20003003D0022C2BF000008A30013
:1091E000FAFF320022C2BF000008A30008003200CC
:1091F00030118000BEFF0700E10020005021210057
:10920000DC7C0200000000006044B800560037001B
:109210008004EB006055B80008C8B3000006EB00FE
:10922000A8FF0700CAC2BF0008406000FDFF32006F
:109230001FE1A80011E1A80001C8B300CAC2BF0025
:1092400001406000FDFF3A0011E1A9001FE1A90003
:10925000F0C1B3008666B700FC0888008C0888005F
:109260004008800001002000C000DD000000200058
:109270003208800002004000E08048000900E00061
:1092800007003200E00F5500E08F5D000300320060
:109290008A0F50008B8F5800010031000005BE007E
:1092A0008904E800F98F5400DDFF3A0090FF0700C1
:1092B0000A01BE0000402200410F20000C090200FC
:1092C000000000000004BE000D00E00026003A008F
:1092D000009F240021002000800F5400818F5C003B
:1092E00005003600F102200030222100DC7C020063
:1092F000000000001C003700F100200020252100A4
:10930000827C0200000000000800BE008A600200AB
:10931000000000004100200000272100DC7C02004A
:1093200000000000F100200010262100827C0200D5
:10933000000000000800BE0077FF07008A600200FE
:10934000000000004100200000272100DC7C02001A
:10935000000000000400370022C2BF000008A30084
:109360009AFF32009FFF37000800BE004F06BE0084
:109370004F05BE004F04BE000000060080BB280061
:10938000286002000000000000000600889FBE0068
:109390008A9FBE008C1F7800A1D52000C0CFB300EB
:1093A000914860001124A1001134A100A0AF200059
:1093B0001044A00090568000A06A88001144A100CB
:1093C0001181FB004212DE004311DE0061416100A9
:1093D0006142620091407800E3C1600011C0B300B7
:1093E000067F020000000000707F02000000000005
:1093F000E2FF0700A8D520008AD52000ABAF2000EF
:10940000A67F0200000000000004E0000A00320015
:109410009840780070C06000050032009C7F020018
:1094200000000000B46302000000000002003700EA
:109430009C7F02000000000032C2BF000018A300A1
:10944000010032003222A9001A630200000000006D
:10945000E14F5000EAFF3A00A06302000000000064
:1094600080417800004D78000080FB00C400DE00E1
:1094700070D5200001487800E4CF50008A00320007
:1094800005003E000104E0000A003200E1CF500078
:10949000E1003A006C003700E6CF5000890032004E
:1094A000DD00390068C05000E14F5000DA003E0096
:1094B000A5003700E2CF51001500320005003E0044
:1094C0000304E0000A003200E1CF51005A003A00E4
:1094D0000D003700E7CF51001B003200EFCF5100E5
:1094E0003D003200E3CF510053003A001100370035
:1094F0007A7F0200000000004F0678004F05BE0092
:109500004F04BE00000006009CFF0700BCFF3700B0
:1095100010C0B300B46302000000000032C2BF00FC
:109520000018A300010032003222A9001844A00054
:10953000B3FF37001844A10010C0B300B4630200A9
:1095400000000000AEFF370010C0B300B46302009B
:10955000000000007A7F020000000000A06302000B
:10956000000000004800DD00A06A880010C0B300C1
:10957000B463020000000000A063020000000000CD
:109580000080FB00A16A800001007000A06A8800D2
:109590001881FB004212DE004311DE0061416100D0
:1095A0009B80FB00C408DE00E1C0600061426200F5
:1095B00098427800E3C16200067F020000000000CC
:1095C000707F02000000000010C0B300B46302000E
:1095D000000000008AFF370010C0B300B46302002F
:1095E000000000003222A90032C2BF000008A30020
:1095F0000500320023C2BF000018A30002003A0099
:10960000B0118000201188001A63020000000000E1
:10961000E14F5000F4FF3A0033C2BF000018A3002E
:10962000F1FF3A00A0630200000000000080FB0090
:10963000A0118800ECFF37000040EB00B46302008B
:10964000000000006EFF37006FC06100004DE800B1
:1096500010C0B300B46302000000000060D5200019
:109660000048EB001A04E00065FF32008004780037
:109670008CD52000A0630200000000000080FB00E9
:10968000907F02000000000010C0B300B46302002D
:10969000000000001940E800804C78009C4F50000A
:1096A00057FF3100F3FF3700034078009680020037
:1096B0000000000010C0B300B4630200000000000E
:1096C0004FFF37006FC0610081D5200080487800CF
:1096D000EA4F500002003600A0C0B3008048780076
:1096E0001A80FB000000400021AD2000608078005F
:1096F000A06A88007A7F0200000000001881FB0049
:109700004212DE004311DE00614161009B80FB00DC
:10971000C408DE00E1C06000A06A8000614262000F
:1097200098427800E3C16200067F0200000000005A
:10973000707F02000000000010C0B300B46302009C
:10974000000000002EFF3700A1D52000C4CFB300D9
:10975000914862001124A1001134A1001B44A10012
:109760000381FB000238A30005003200914278001B
:1097700063C062000014A00084C8620091487000B9
:109780000228A300060032009840780063C0600001
:109790000004A000C1CFB30018CC6000184C7000CA
:1097A0000218A300010032001824A0000308A3003F
:1097B000010032001834A0000248A30001003A0062
:1097C0001B44A0007A7F0200000000001881FB000B
:1097D0004212DE004311DE00614161009B80FB000C
:1097E000C408DE00E1C06000A06A8000614262003F
:1097F00098427800E3C16200067F0200000000008A
:10980000707F02000000000010C0B300B4630200CB
:1098100000000000FAFE37000040EB00B4630200D5
:1098200000000000F6FE370000C528002860020096
:109830000000000000000600889FBE008A9FBE0056
:109840008C1F7800A1AF2000114078000034A100E7
:109850000044A0008048780018C0B30080AE20000B
:109860000848780081C0B30090AE2000014878001D
:1098700020C0B30041D720008048780080C0EB00B2
:109880008267020000000000C922A900C902A900E5
:10989000C8E2A80008407800AE690200000000009D
:1098A000E1FF07008AD720006CD72000A0630200E8
:1098B0000000000080417800004D78000080FB002F
:1098C0004400DE0071D7200080487800E34F50004C
:1098D000C700320004003E00E14F50008600320015
:1098E000BA003E000B003700E64F50007202320013
:1098F00003003E00E44F5000A3023A006702370025
:10990000E84F50007B023200EA4F50009E023A00BE
:10991000D80037000380FB0001002000ED0F50004D
:10992000E08F580070003E00006001009A0237008E
:109930000C0037000D003700120037001700370009
:109940001D003700230037003A0037003E00370083
:1099500042003700480037004E00370054003700FF
:109960005A003700B0FF0700D0FF3700F46702004D
:109970000000000010C0B300B4630200000000004B
:10998000CAFF3700286802000000000010C0B300C2
:10999000B463020000000000C4FF37000040EB0089
:1099A000AE6902000000000010C0B300B463020002
:1099B00000000000BDFF370010C0B300AE69020018
:1099C0000000000010C0B300B463020000000000FB
:1099D000B6FF370040D7200021C0B30090CF100061
:1099E00004003A00EC68020000000000004E78001D
:1099F00004003700F00F200044680200000000005F
:109A0000004E7800A0AF2000104078006840600051
:109A1000040032001C80FB005A7C020000000000A1
:109A2000004E78001C407800B46302000000000083
:109A30009EFF37002E69020000000000B4630200A0
:109A40000000000099FF3700BA6902000000000022
:109A5000B46302000000000094FF370010C0B300A0
:109A6000706902000000000010C0B300B46302007F
:109A7000000000008DFF37000040EB00A2690200EB
:109A80000000000010C0B300B4630200000000003A
:109A900086FF370010C0B300A2690200000000007A
:109AA00010C0B300B4630200000000007FFF370065
:109AB0000040EB00966902000000000010C0B300F7
:109AC000B46302000000000078FF370010C0B3004C
:109AD000966902000000000010C0B300B4630200E9
:109AE0000000000071FF37000040EB00B46302008B
:109AF000000000006DFF37006FC06100004DE800FE
:109B000010C0B300B463020000000000004EEB0080
:109B10001A04E00065FF320059D72000ABAF2000E7
:109B2000A06302000000000080407800804C7800B4
:109B30001B41780068406100040032000180FB0096
:109B40005A7C020000000000804C780040D72000C2
:109B500021C0B30090CF100007003A001980FB002D
:109B6000A46802000000000010C0B300B46302004B
:109B7000000000001000370058D720001880FB00BC
:109B8000446802000000000080407800004C78002B
:109B90001B41780068406100040032000180FB0036
:109BA0005A7C020000000000004C78001940780048
:109BB000B4630200000000001C40E800004E780082
:109BC0009A4F500039FF3100D5FF37006FC0610058
:109BD0000040E800004D78007069020000000000BD
:109BE00010C0B300B4630200000000002FFF370074
:109BF0006FC06100004DE80010C0B300B463020004
:109C000000000000A06302000000000071D72000E7
:109C100080487800004EEB001A04E000110032008A
:109C20000104780069D720001804E00004003D001A
:109C300010C0B300526902000000000003003700AA
:109C40000040EB005269020000000000184078005C
:109C5000004C40001940E800804C78009A4F5000BA
:109C6000F1FF390010C0B300B4630200000000002F
:109C70000EFF370040CAB30080CF510014003200FD
:109C800004003E006440500080CF51007F013A0044
:109C90000700370050CAB30080CF5100980032004F
:109CA00000C0E80080CF510078013A00ED00370095
:109CB000A06302000000000061AE20008048780030
:109CC00010C0B300B463020000000000F7FE3700CC
:109CD00060AE200010407800E14F500003003200D9
:109CE000E24F500082003A002A003700A0630200D1
:109CF000000000000080FB006300B900906B88004A
:109D00000001EB00626B88000000E0000C003200F4
:109D100082007800E980200019844000A0630200DE
:109D200000000000004C7800606B80008000E800BC
:109D3000616B8800906B8000808F5000F6FF3900C7
:109D40008000EB00616B8800906B80000000E000F9
:109D50000C00320070408000010040002041900063
:109D60009040900010407800D7010700606B8000A1
:109D7000E3004000616B8800906B8000808F500092
:109D8000F4FF390010C0B300B4630200000000000B
:109D9000C6FE3700A0630200000000000080FB0048
:109DA0004200DD00906B88008000EB00616B880052
:109DB0000B003200E980200019844000A0630200FB
:109DC00000000000004C7800606B80008000E8001C
:109DD000616B8800906B8000808F5000F6FF390027
:109DE0000000EB00606B8800906B80000000E000DA
:109DF0003B0032000040EB0052690200000000000E
:109E00000040EB0052690200000000000040EB003F
:109E100052690200000000000040EB00526902009D
:109E200000000000616B800070408000614078009D
:109E30000080FB00A4680200000000007040800069
:109E4000616B800001004000104090000080FB002A
:109E5000A46802000000000070408000616B800078
:109E600001004000204090000080FB00A468020038
:109E700000000000626B8000E080200010004100C4
:109E800063004000904078006FC86000004EEB0017
:109E90007040800000004100304090000004E0006D
:109EA0000A00320068D72000B80107001840E80017
:109EB000004C7800626B800071408000828040001E
:109EC000B1409000814F5000F7FF3900E40041009D
:109ED000616B8800906B8000808F5000C5FF390057
:109EE00010C0B300B4630200000000006FFE370032
:109EF0000040EB00B4630200000000006BFE37007E
:109F000060AE200010407800E14F500003003200A6
:109F1000E24F500065FE3A0030003700A0630200B7
:109F2000000000000080FB00906B8800A06302002E
:109F30000000000071D72000804878000000EB008E
:109F4000606B8800906B80000000E00057FE3200DC
:109F500058D7200069D7200070D72000104C780017
:109F6000804CEB001880FB000008A30004003200C6
:109F700010C0B30052690200000000000300370067
:109F80000040EB0052690200000000001880FB0056
:109F90000000D100004C78001940E800804C7800A7
:109FA000E34F5000EFFF3600EC68020000000000B5
:109FB000EC68020000000000B46302000000000032
:109FC000606B80000000E800606B8800916B80008F
:109FD000810F500035FE3100DFFF3700A063020023
:109FE000000000008080FB00916B88008000EB0087
:109FF000616B88000004E0002CFE320022C0B30038
:10A0000060B92000A10B20009F010700CB010700D1
:10A0100022C0B30060BB2D00A10B20009A010700F5
:10A0200022C0B300603D2D00A10B20009601070067
:10A03000C201070022C0B30060BB2000A10B2000BA
:10A0400091010700BD010700606B80000000E8007F
:10A05000606B8800916B8000810F500013FE31000F
:10A06000E6FF3700A0630200000000000080FB0054
:10A07000806B8800A0630200000000000081FB00EC
:10A08000726B880060AE200010407800E24F5000F4
:10A0900005003A00806B80006500B90000004100B7
:10A0A000906B880014003700E14F500006003A0022
:10A0B000806B800000004000000041000000400074
:10A0C000906B88000C003700E34F500006003A0008
:10A0D000806B800000004000000041000000400054
:10A0E000906B8800040037000040EB00B46302006E
:10A0F00000000000EDFD37008000EB00616B880080
:10A10000906B80000000E0000B003200E98020002E
:10A1100019844000A063020000000000004C780099
:10A12000606B80008000E800616B8800906B8000AD
:10A13000808F5000F6FF3900706B80000000E00057
:10A140000300320010C0B300B4630200000000003E
:10A150000000EB00606B880068AE20004000370014
:10A1600070408000E2407800E1CF500021003A00CA
:10A1700098407800E3CF500009003A000200400008
:10A1800030419000A0409000104090009A000700DD
:10A19000606B800064004000606B88003000370016
:10A1A000E1CF500009003A00020040003041900029
:10A1B000A040900010409000C3000700606B80003A
:10A1C00064004000606B880025003700E2CF50003B
:10A1D00023003A0002004000C04090000000E80068
:10A1E00000010700606B800065004000606B880024
:10A1F0001B003700E2CF500019003A009840780069
:10A20000E3CF500007003A000200400010409000E9
:10A2100065000700606B80000080E800606B8800CC
:10A220000F003700E1CF500007003A000200400065
:10A23000104090008C000700606B80000080E800F8
:10A24000606B880006003700E2CF500004003A003F
:10A250003A010700606B80000000E800606B880036
:10A26000626B8000906B8000800F5100BCFF390052
:10A27000706B80000000E0008CFD3A0010C0B3005D
:10A28000B46302000000000088FD37000040EB00CE
:10A29000B46302000000000084FD37000340780032
:10A2A000968002000000000010C0B300B4630200FA
:10A2B000000000007DFD3700E3C06100014D780023
:10A2C00080AE20000148780040D720001040780080
:10A2D000826702000000000010C0B300AE690200F7
:10A2E0000000000010C0B300B463020000000000D2
:10A2F0006EFD3700A2AF2000124078000040A100A0
:10A30000004978008380FB000138A30002003A0076
:10A310000044A0000049780042D7200020C0B300CC
:10A32000004978000128A3000200320030C0B300C9
:10A3300000497800A2AF2000124078000030A10050
:10A34000004978000118A300020032000034A00088
:10A350000049780080AE20009040780040D720006F
:10A3600010407800826702000000000010C0B300B7
:10A37000AE6902000000000010C0B300B463020028
:10A380000000000049FD37000040EB00B46302000C
:10A390000000000045FD37004F0678004F05BE0065
:10A3A0004F04BE0000000600889FBE0000447800F5
:10A3B00069C0B300614064005269020000000000FF
:10A3C0000880FB000004D1008944E900F9FF3A004D
:10A3D000EC68020000000000B4630200000000000E
:10A3E000EC68020000000000B463020000000000FE
:10A3F0004F04BE0000000600889FBE008A9FBE007A
:10A400008C1F78000044780081457800024678006F
:10A4100000C8B3000045640069C0B3006140640037
:10A4200052690200000000000880FB000004D10017
:10A430008944E900F9FF3A000A04E00006003A0006
:10A440000B80FB00A4680200000000000C80FB00F1
:10A45000A4680200000000004F0678004F05BE000F
:10A460004F04BE0000000600889FBE000044780034
:10A4700049C0B3000808A3000400320010C0B300B4
:10A480005269020000000000030037000040EB00AA
:10A4900052690200000000000880FB000004D100A7
:10A4A0008944E900F3FF3A00EC6802000000000074
:10A4B000EC68020000000000B4630200000000002D
:10A4C0004F04BE0000000600889FBE008A9FBE00A9
:10A4D0008C1F78000044780081457800024678009F
:10A4E0000080FB004605DE008044EB000F003700D3
:10A4F000E3CF54000D003A000A04E0000A003200E5
:10A5000010C0B300A2690200000000000A80FB0036
:10A51000087C0200000000000040EB00A26902007D
:10A52000000000000C00370039C0B3000808A30089
:10A530000400320010C0B3005269020000000000A5
:10A54000030037000040EB005269020000000000E9
:10A550000880FB000004D1008944E800E3CF5400E8
:10A56000E3FF36000B80FB00A4680200000000003F
:10A570000C80FB00A4680200000000004F06780079
:10A580004F05BE004F04BE00000006000040EB0077
:10A5900052690200000000000040EB005269020016
:10A5A000000000000040EB005269020000000000C3
:10A5B0000040EB0052690200000000000000EB00C8
:10A5C000A4680200000000000000EB00A468020084
:10A5D000000000000000EB00A46802000000000082
:10A5E00000000600889FBE000004780081447800C7
:10A5F0000040EB0052690200000000000040EB0048
:10A6000052690200000000000040EB0052690200A5
:10A61000000000000040EB00526902000000000052
:10A620001880FB00A46802000000000018409000A1
:10A630000080FB00A4680200000000002840900099
:10A640000080FB00A4680200000000006FC06400EE
:10A650000041E900E14F4100090032000244780066
:10A660000080EB000090B900004041008044E90008
:10A67000C6FF07000844E90088CF5400FCFF3A00F9
:10A680004F04BE0000000600889FBE008A1F7800AD
:10A690000004BE00024578000040EB005269020051
:10A6A000000000000040EB005269020000000000C2
:10A6B0000040EB0052690200000000000040EB0087
:10A6C0005269020000000000080078005A7C020075
:10A6D00000000000A4680200000000004849DD00FE
:10A6E0004840DE0000007100C848DE005A7C0200CD
:10A6F00000000000A468020000000000404CDE00E2
:10A70000080078005A7C020000000000A4680200E3
:10A71000000000006F456500050032000044EB00BA
:10A720009AFF07000844E800884F5500FCFF3A00F4
:10A730004F0578004F04BE0000000600881F780017
:10A7400010C0B30052690200000000000040EB009E
:10A7500052690200000000000040EB005269020054
:10A76000000000000040EB00526902000000000001
:10A770000000EB00A468020000000000EC6802008A
:10A780000000000000047800EC68020000000000F7
:10A79000B46302000000000008407800B4630200C7
:10A7A0000000000079FF070078FF07004F047800E1
:10A7B00000000600805880000000E0001100320018
:10A7C00000C2B300B46302000000000031002000AA
:10A7D00030412000827C02000000000000C2B30073
:10A7E000B463020000000000705880000000E00028
:10A7F00002003A0052690200000000000000EB0075
:10A80000805888008040EB00705880000000E00015
:10A8100003003A00EC68020000000000804078006D
:10A8200010002000805888000180FB000000060016
:10A83000881F780000047800805880000000E00045
:10A840001100320000C2B300B46302000000000037
:10A850003100200030412000827C02000000000016
:10A8600000C2B300B4630200000000007058800012
:10A870000000E00002003A005269020000000000FF
:10A880000000EB0080588800705880000000E00055
:10A8900006003A0008007800A468020000000000EA
:10A8A0002E690200000000000084FB0000C2B3001B
:10A8B000B4630200000000000800E00006003A0057
:10A8C0003100200030412000827C020000000000A6
:10A8D00000302000050037004100200060412000CA
:10A8E000827C020000000000001020004F0478006D
:10A8F00000000600805880000000E0000F003200D9
:10A900004100200060412000827C02000000000025
:10A91000E0C1280040600200000000007058800084
:10A920000000E00003003A0010C0B30052690200CA
:10A93000000000000000EB00805888007058800084
:10A940000000E0000F003A00F46702000000000081
:10A950000000E0000B00320091002000C020200029
:10A96000827C0200000000005101200050212000E4
:10A97000827C020000000000E0C12800406002006C
:10A9800000000000D1002000A0412000DC7C02007B
:10A990000000000000000600805880000000E00079
:10A9A0000F0032004100200060412000827C020044
:10A9B00000000000E0C1280040600200000000002C
:10A9C000705880000000E00003003A0010C0B3009F
:10A9D00052690200000000000000EB00805888006F
:10A9E000705880000000E00002003A002868020071
:10A9F00000000000C100200070422000DC7C02004A
:10AA0000000000000000060001012000404F20006F
:10AA1000827C0200000000000040EB0004620200A3
:10AA20000000000000C2B300B46302000000000098
:10AA300080AE200010407800046202000000000098
:10AA400000C2B300B463020000000000F0C128009F
:10AA5000406002000000000000000600881F78002F
:10AA60000000EB0070588800D61D020000000000B6
:10AA70000E1C020000000000800078000000E900C9
:10AA8000E30F500004003E0080AE20000148E900C2
:10AA90000100E00010003A000004EB006865880047
:10AAA00078588800B103200080452000DC7C02003B
:10AAB0000000000088017800420020001100200002
:10AAC00010002000DC1E02000000000081AE20000B
:10AAD0008048E9000B00370081812000300023000E
:10AAE000910F100004003E00510320003049200067
:10AAF000827C020000000000C3FF07000000EB00A2
:10AB000080588800A0AF20001044A0004F047800B7
:10AB100000000600705880000000E00009003A00C4
:10AB2000C922A800C902A800CB02A900CB22A90013
:10AB300080AE20009040780020C0B3008267020001
:10AB400000000000000006000000EB0080588800B4
:10AB500070588000E10F500001003A0007E2A900A0
:10AB600000000600889FBE00E10F5000090032007F
:10AB700003003900E20F50006B003A005B00370021
:10AB80005103200040502000827C020000000000A1
:10AB9000690037008040EB0000302000C2690200ED
:10ABA00000000000E102200090532000DC7C020045
:10ABB00000000000CBC2BF000008A3000500320067
:10ABC000CBC2BF00190020000004EB000018A30056
:10ABD0000C003A0091002000C0202000827C02007E
:10ABE000000000005101200050212000827C020062
:10ABF00000000000E0C128004060020000000000EA
:10AC00004D003700705880000000E00008003A0056
:10AC1000F46702000000000008007800A468020049
:10AC2000000000002E690200000000008084FB008C
:10AC30000900E00020003A00080078007C7B020058
:10AC40000000000080C2B300B463020000000000F6
:10AC50000880D1007C7B0200000000000808A300EF
:10AC600004003A0010C22800286002000000000022
:10AC70000B003700705880000000E00005003A002B
:10AC8000EC6802000000000010C0B300526902002E
:10AC90000000000040C22800286002000000000000
:10ACA000F0C12800286002000000000000C2B300CC
:10ACB000B463020000000000705880000000E00053
:10ACC00002003A0028680200000000000804E800C2
:10ACD00000102000800F5400CAFF3A00E0C1280095
:10ACE0004060020000000000130037007058800030
:10ACF000E10F500001003A0007E2A90071002000B6
:10AD000070562000DC7C020000000000F1002000F2
:10AD1000B0182100DC7C02000000000010C0B3006D
:10AD20000C0007000400370041022000E01D200055
:10AD3000DC7C0200000000004F04BE0000000600A2
:10AD4000B1002000600B2100DC7C0200000000004C
:10AD500000000600E4874700889FBE008A9FBE006F
:10AD60008C9FBE008E1F780090F79F00206302002A
:10AD700000000000C922A800C902A800CB02A90057
:10AD8000CB22A90062A0A80062C0A8008660A9002A
:10AD9000CBC2BF000000D100B12C20009140780050
:10ADA0006146600061C460000047EB008E46780099
:10ADB0008EF79F00060037000B4678000A447800A3
:10ADC0000047EB00020037000B4678000A44780089
:10ADD00086C0BF000038A3000E003A002E630200B8
:10ADE000000000001A630200000000000004E00000
:10ADF000F7FF3200A06302000000000062A0A9007B
:10AE000062C0A9009FF097000104E00057003200E3
:10AE1000530037008660A900CBC2BF000000D100FC
:10AE2000E104600089457800CBC2BF00614060004A
:10AE3000004578000E04E0002F0032000804E00016
:10AE40002F003A000004E000DFFF3200E7CF560099
:10AE50000B003E000FF097000040400080F79F007D
:10AE60000904E000020032000004A00080F79F0007
:10AE70008D46E8000B4678000A447800D4FF37007E
:10AE80001FF097000004E000050032008FF09700EB
:10AE90000180FB006662020000000000060037002F
:10AEA000C0C5B30078630200000000000FF09700F7
:10AEB00078630200000000000904E000070032008F
:10AEC000D0C2B30078630200000000000B46780097
:10AED0000A4478008046EB00BDFF3700B0C2B300E3
:10AEE00078630200000000000B4678000A447800F6
:10AEF0008046EB00B6FF37000804E000AEFF3200EA
:10AF00000004E000B0FF32000C04E0000A00320050
:10AF10000904E000ACFF3A00B0C5B300786302005A
:10AF2000000000000B4678000A4478001EC0B30001
:10AF300089467800A6FF37000904E000A2FF32002E
:10AF4000D0C5B30078630200000000000B46780013
:10AF50000A4478000047EB008E4678009CFF3700DB
:10AF6000E0C1280040600200000000004F077800A8
:10AF70004F06BE004F05BE004F04BE004F00B1009B
:10AF80000000060070C228002860020000000000D7
:10AF900000000600889FBE008A9FBE008C9FBE00F6
:10AFA0008E1F7800C922A800C902A800CB02A90000
:10AFB000CB22A900C8C2A900A1AF2000114078008F
:10AFC0000034A1000044A0008048780080C0EB005D
:10AFD00020C0B3008267020000000000E9FF070004
:10AFE000CAB02000AEAF2000A06302000000000045
:10AFF00080417800004D78000080FB004400DE00B6
:10B00000B1B0200080487800E14F5000D2003200FB
:10B0100005003900E44F5000F1003200E64F5000C7
:10B02000F6003A00E50037000380FB000100200035
:10B03000EF0F5000E08F5800C3003E000060010099
:10B04000F50037000E0037000F00370014003700FE
:10B0500019003700BC0037001C0037002200370001
:10B06000280037007D003700B7003700B6003700F2
:10B07000B5003700B4003700B3003700AC0037002C
:10B08000C0FF0700D8FF3700F4670200000000008F
:10B0900010C0B300B463020000000000D2FF37000C
:10B0A000286802000000000010C0B300B463020072
:10B0B00000000000CCFF3700EC6802000000000038
:10B0C000B463020000000000C7FF37000040EB003F
:10B0D000526902000000000010C0B300B463020017
:10B0E00000000000C0FF370010C0B300526902002A
:10B0F0000000000010C0B300B463020000000000B4
:10B10000B9FF3700A0630200000000004804DD0022
:10B11000A0630200000000000080FB0080057400B6
:10B12000A0630200000000004804DD00A0630200EC
:10B13000000000000080FB000006740000002100F9
:10B14000808F550002003E00800F5600AF00360091
:10B150000040EB00B463020000000000A2FF3700D3
:10B160008004EB00ED8020001D844400A0630200F9
:10B1700000000000004C78008904E800898F550029
:10B18000F9FF3A00F4670200000000000B00E00045
:10B190000D0032000004EB00704080006840780031
:10B1A0000080FB00A4680200000000002E6902007D
:10B1B00000000000E14F5000E5FF32000804E80005
:10B1C000888F5500F4FF3A008C05E9000C00E00080
:10B1D000120032008004EB00ED8020001D8444004A
:10B1E000EC68020000000000004C78008B8F5400D7
:10B1F000040031000040EB00526902000000000032
:10B200000300370010C0B3005269020000000000C4
:10B210008904E800890F5600F0FF3A002868020010
:10B220000000000010C0B300B46302000000000082
:10B230000C00E0006CFF32000004EB007040800066
:10B2400068407800B4630200000000000804E800D1
:10B25000880F560064FF3200F8FF370010C0B300BB
:10B26000B46302000000000022C2BF000008A30077
:10B27000FDFF32003011800080407800004D7800E2
:10B28000E24F50001700320005003E000004E000CD
:10B290000C003200E14F500008003A000D0037006A
:10B2A000F04F50001600320000C2B30080CF5000B3
:10B2B00017003200E3CF50000E00320010002000D3
:10B2C00018003700F83902000000000010002000CC
:10B2D00014003700DC3902000000000010002000DC
:10B2E00010003700C43902000000000010002000E8
:10B2F0000C003700143A020000000000090037007B
:10B30000C0CFB3001E4F60001000200005003700C2
:10B310001E4078000014A1000004A000004F780037
:10B3200010002000B4630200000000002EFF370070
:10B330000040EB0087FE070010C0B300B4630200BA
:10B340000000000028FF37000040EB00B46302005B
:10B350000000000024FF37006FC06100004DE800CE
:10B3600010C0B300B463020000000000A0B02000D1
:10B370000048EB001A04E0001BFF320000047800D4
:10B38000C9B02000A0630200000000000080FB00A4
:10B39000A4680200000000002E6902000000000006
:10B3A000B4630200000000001840E800004C780080
:10B3B000994F50000CFF3100F2FF3700E3C06100ED
:10B3C000014D780020C0B300826702000000000039
:10B3D00010C0B300B46302000000000002FF370099
:10B3E00003407800968002000000000010C0B30007
:10B3F000B463020000000000FBFE37000040EB00D9
:10B40000B463020000000000F7FE37000B00E0000C
:10B410005CFF320052FF37004F0778004F06BE0036
:10B420004F05BE004F04BE000000060000C0EB0048
:10B43000E27E0200000000000080FB000000060029
:10B44000E27E020000000000001020000000060064
:10B4500010C0B300987E0200000000000080FB00D6
:10B460000000060020B1200010407800987E020005
:10B47000000000000000060020B120001080FB004A
:10B480000000060020B120000048EB00410220002F
:10B49000B0002000DC7C020000000000000006007C
:10B4A00011C0B30020B12000014878004102200003
:10B4B000B0002000DC7C020000000000000006005C
:10B4C000A0AF20001044A00040B220000048EB00D4
:10B4D000C922A800CB22A90000000600889FBE0058
:10B4E0008A1F7800800078000004E9001003200023
:10B4F000800F540030003E0040B220001080FB005E
:10B50000800F54000500390091022000F002200055
:10B51000DC7C0200000000000E013700E10020008A
:10B5200080052000827C0200000000000840E80046
:10B530000462020000000000C0C22800286002006F
:10B54000000000008040EB00E0B1200001487800DE
:10B5500001407800C344DD005AB22000E8B1200069
:10B560000080FB000900400060407D000080FB007F
:10B570007C7B02000000000000C2B300B463020044
:10B58000000000001880FB000900400060407D00C2
:10B59000E27E0200000000001840E800004C780045
:10B5A000E74F5000EEFF3600F0C228004060020076
:10B5B00000000000E700370050052000808F500099
:10B5C000CE00320006003E000100E0000E00320016
:10B5D00030032000808F5000DA003A00A4003700CA
:10B5E000C00E2000808F50004800320064004000F0
:10B5F000808F500045003200C00C2000808F50002A
:10B60000D0003A00C6003700D100200060062000BC
:10B61000DC7C0200000000007101200030072000E7
:10B62000DC7C02000000000040B220001004E000BA
:10B6300005003A0091022000F0022000DC7C0200AC
:10B64000000000002C003700F0B120000048EB00A3
:10B6500080047800E8B120005AB2200000C2B30094
:10B66000B4630200000000001940E8000462020018
:10B670000000000000C32800286002000000000055
:10B680000040EB00004C78000080FB009980FB003C
:10B69000C308DD000100400060407D000080FB0029
:10B6A0007C7B02000000000000C2B300B463020013
:10B6B000000000001840E800004C7800E74F500000
:10B6C000F1FF360061002000A0082000827C02000B
:10B6D000000000001980FB004300DD0060407D0099
:10B6E000C80007009940E800814C780040B2200073
:10B6F00090CF5000D9FF3900310D20000009200003
:10B70000DC7C02000000000092003700A0822000D4
:10B7100001487800C00E2000808F500005003A00DC
:10B720003101200030162000DC7C02000000000007
:10B7300004003700D100200060172000DC7C0200EC
:10B74000000000007101200030072000DC7C0200B6
:10B75000000000000044EB00E0B120000848780041
:10B76000D7000700F1B120008048780041B22000E6
:10B77000884878000004E00038003200EAB1200078
:10B780008004EB0058B7200000C2B300B46302008D
:10B79000000000001A40E8000462020000000000FF
:10B7A00000C328002860020000000000E95888005B
:10B7B0000900780060407C000080FB007C7B020078
:10B7C0000000000000C2B300B463020000000000EB
:10B7D000E05880000000E800E0588800E70F5000C3
:10B7E000F4FF360061002000A0082000827C0200E7
:10B7F0000000000018407800820007009A4278009C
:10B80000E9CF52000F003E00E95888008900780017
:10B8100042B2200054B2200053B720001280FB0037
:10B820004300DD000100400061C3790006707A002A
:10B830008100E800E88F5000F8FF3A00E1588800E6
:10B840001249E800054DE800A7000700F1B120000B
:10B85000804878000004E000CBFF3A00B1022000ED
:10B8600030182000DC7C02000000000039003700A6
:10B870004000070011012000E01A2000827C020035
:10B880000000000030C3B300E27E020000000000B0
:10B890000000EB00E05888000004780039B1200077
:10B8A00000C0EB00E27E02000000000000F47C001B
:10B8B000E058800060C07C000080FB007C7B0200C0
:10B8C0000000000000C2B300B463020000000000EA
:10B8D000E05880000004E800E8588800E70F5400B2
:10B8E000EFFF3600F0C228004060020000000000B8
:10B8F0001940780043000700160037001D000700BC
:10B9000001012000F01B2000DC7C02000000000090
:10B9100050C5B300E27E0200000000000D003700B9
:10B9200014000700F1002000F01C2000DC7C020065
:10B9300000000000C0CCB300E27E02000000000066
:10B940000400370041022000E01D2000DC7C0200E2
:10B95000000000004F0578004F04BE000000060004
:10B9600091002000200A2100DC7C02000000000081
:10B9700000000600881F78005C7E020000000000C6
:10B9800000447800A100200020202000827C0200DA
:10B99000000000000804E00005003A00310020002B
:10B9A00080BB2000DC7C0200000000001300370098
:10B9B00091002000C0202000827C020000000000D6
:10B9C0000808A3000400320051012000502120008B
:10B9D000827C0200000000000818A300040032006E
:10B9E00041012000A0222000827C02000000000013
:10B9F000F0C2280040600200000000004F04780000
:10BA0000000006008040780020C2B30080CF5000C4
:10BA10001700320005003E00E4CF5000190032004C
:10BA2000F0CF500021003A000700370080C2B30079
:10BA300080CF5000090032006540400080CF5000A8
:10BA40001A003A0014003700B1012000E023200062
:10BA5000DC7C02000000000018003700A10120007B
:10BA600090252000DC7C020000000000130037005D
:10BA70005101200030272000DC7C02000000000083
:10BA80000E0037008101200080282000DC7C0200AD
:10BA9000000000000900370001012000002A2000FA
:10BAA000DC7C02000000000004003700E100200000
:10BAB000002B2000827C0200000000000000060035
:10BAC0008040EB00D0B7200001487800F0B720009C
:10BAD00001487800E0B72000014878000500070021
:10BAE0000080FB0000000600020007000080FB0051
:10BAF00000000600889FBE008A9FBE008C9FBE008B
:10BB00000044EB0000B8200008487800F9B7200096
:10BB10001904E00067003A005C7E020000000000AB
:10BB20000004E00007003200D0B720000848780089
:10BB3000884C7800E0B72000084878000000EB004F
:10BB400064003700A082200010407800E27E0200EE
:10BB5000000000001BC0B3008046EB000D457800DC
:10BB60008B4478005CB7200010C0B300987E0200C0
:10BB7000000000000044780010C0B300987E02006E
:10BB800000000000E14F540003003A00E14F500074
:10BB90001D003A0036003700804F5400020032008A
:10BBA0008841780020003700D0B72000104078008E
:10BBB00080CF5500060031000A80FB0060407E0007
:10BBC00080C164000600320013C0B30004003700D7
:10BBD00000C06D000080FB000000E900CF01DE0026
:10BBE0000304E00006003A00E8CF55000C003E00D8
:10BBF000E0B720000B4878008B4678000A00370039
:10BC0000E1CF510008003A008A80FB0061407E00CD
:10BC100000C0740080707E0013C0B30007003700BE
:10BC20008B4678008041EB000A80FB0089C0EA0067
:10BC300060417E0082C0600001707E000340780099
:10BC4000987E0200000000008B45E80089C4440093
:10BC500005003A000A80FB0060407E0057000700A4
:10BC60000A45E80019C0B300E74F5500BEFF360093
:10BC700000C4B30080CF55000E00360000B820008D
:10BC80001004E0000B003A00D0B720000D48780007
:10BC90000D04E00003003A0011C0B300F0B720002B
:10BCA0000148780011C0B30050B720001004E00034
:10BCB00007003A008040EB00D0B720000148780030
:10BCC000F0B7200001487800E0B720000148780074
:10BCD0000180FB004F06BE004F05BE004F04BE00B2
:10BCE000000006000800FA00889FBE008A1F780046
:10BCF0000000EB0051B72000E0C178006E815700D2
:10BD0000037178000000E800E80F5000FAFF3A00E5
:10BD1000D2B7200012457800F1B720009144780096
:10BD2000E0B720001044780000C4B3000049780058
:10BD30008048EB006FFF07000004E0000C003200B9
:10BD40000001EB0053B720006E805700E0407900FF
:10BD500062C0790080CF500005003A000201E8007F
:10BD6000E80F5100F8FF3A0012C0B300010037009D
:10BD70000041EB000000EB0051B72000EE815700BE
:10BD8000E37078000000E800E80F5000FBFF3A0085
:10BD9000D0B720000A487800F0B7200009487800A2
:10BDA000E0B72000084878000280FB004F057800CB
:10BDB0004F04BE000080FA000000060002B8200018
:10BDC000124068000080FB00B182200060C0780053
:10BDD000004978000080FB000000060020C3280016
:10BDE000286002000000000000000600889FBE00DE
:10BDF0008A9FBE008C1F7800C922A800CB22A90010
:10BE0000C8C2A900A1AF2000114078000034A100F1
:10BE10000044A00080487800F0FF07003AB22000FC
:10BE20000CB22000A06302000000000080417800F6
:10BE3000004D78000080FB004400DE0021B22000AD
:10BE400080487800E14F5000530032000300390071
:10BE5000E44F50006E003A0066003700E2CF510018
:10BE60000F00320005003E000304E0006C003200C9
:10BE7000E1CF510044003A0007003700E4CF510001
:10BE80000E0032004000390068C05100E14F500000
:10BE90003D003E000F003700D0FF0700E1FF3700F4
:10BEA0005C7E020000000000004E780010C0B3006D
:10BEB000B463020000000000DAFF370000C0EB00AE
:10BEC000E27E020000000000B463020000000000F7
:10BED000D4FF370010C0B300B463020000000000BC
:10BEE00090C0B3009A4F100004003A00C1CEB300D6
:10BEF000A0822000014878000300370001CFB30082
:10BF0000A082200001487800EDFE0700004E780076
:10BF10000004E0001100320018B220008045EB0060
:10BF200059B720000B4C78000B4078000080FB00D4
:10BF300060C07C00B4630200000000001840E8000C
:10BF4000004C7800E74F5000F8FF3600E6FE07008F
:10BF5000004E78000004E000F2FF3A0010B220002A
:10BF60000048EB000004780000C0EB00B46302005E
:10BF7000000000001840E800004C7800E74F500037
:10BF8000A8FF3E00F8FF37000040EB00B46302005A
:10BF900000000000A3FF37006FC06100004DE80003
:10BFA00010C0B300B46302000000000010B2200013
:10BFB0000048EB001A04E0009AFF32000004780009
:10BFC00039B22000A063020000000000E27E0200FF
:10BFD0000000000010C0B300B463020000000000C5
:10BFE0001840E800004C7800994F50008DFF310058
:10BFF000F4FF370003407800968002000000000044
:10C0000010C0B300B46302000000000085FF3700D9
:10C010000040EB00B46302000000000081FF370025
:10C020004F0678004F05BE004F04BE00000006001A
:10C030000000E0000300320010C3B300CA01070093
:10C040000200370000C3B300C7010700000006006C
:10C05000881F7800B0407800000478000104E000F8
:10C060000500320001407800BF010700B8407800A9
:10C070000104E000FBFF3A004F04780000000600D6
:10C08000881F7800B0407800000478000104E000C8
:10C090000500320001407800B3010700B840780085
:10C0A0000104E000FBFF3A00D0C0B300AE0107007E
:10C0B000A0C0B300AC0107004F04780000000600E8
:10C0C000889FBE008A1F78000045780080BE280047
:10C0D000DFFF070009C8B30088C0B300094065004E
:10C0E0000300320010C3B3009F01070002003700B5
:10C0F00000C3B3009C0107000980FB008004D1004D
:10C100000844E900F5FF3A004F0578004F04BE00EF
:10C1100000000600E4874700889FBE008A9FBE009B
:10C120008C9FBE008E1F78000006BE000040EB0012
:10C1300080F79F000A102E005B5F20008EC0B300C6
:10C140000A01BE000C00BE000C0902000000000045
:10C150000004BE008FF097000104E00003003A00E5
:10C16000E00F5400E08F5C000C00320001C3B3000C
:10C17000014044007C0107000851B8000BC0B90021
:10C180000300400009D2B9008401400002065600B5
:10C1900083865E0010C0B30080F79F00A2002000DD
:10C1A000030020000A00BE000C090200000000008D
:10C1B0000005BE000E47E900E1FF3A0001C3B300ED
:10C1C00001404600680107004F0778004F06BE0097
:10C1D0004F05BE004F04BE004F00B1000000060036
:10C1E000889FBE008A9FBE008C1F78000004BE009E
:10C1F000F0232400F1002000800F5400818F5C00A8
:10C200001700360002242400F30020000800BE00BE
:10C210000C0902000000000056000700C0C2B30075
:10C220005101070002242400F30020000800BE0092
:10C230002C090200000000000004BE001C002000C9
:10C24000703E2000800F5400E08F5C000A003E002A
:10C25000B0BE28007EFF0700100020002B00370032
:10C260000000EB00713E2000810F5400E08F5C0065
:10C27000260036000006EB00823E2000030020006E
:10C280000800BE000C090200000000000005BE000E
:10C2900030062000800F5500E08F5D00030036005F
:10C2A0000A007800330007000F0037000C00E000A0
:10C2B0000B003200E90F5500E08F5D0003003600EF
:10C2C00000C3B300280107000200370000BF2800A8
:10C2D0005FFF07000A007800260007000200370011
:10C2E0000A00780023000700C0C2B3001E01070047
:10C2F000823E2000030020000800BE002C0902003E
:10C30000000000000004BE001000200031062000E4
:10C31000810F5400E08F5C000300360008007800B5
:10C32000140007000F0037000000E0000B0032008F
:10C33000E90F5400E08F5C000300360000C3B30037
:10C34000090107000200370000BF280040FF070076
:10C350000800780007000700020037000800780096
:10C36000040007004F0678004F05BE004F04BE00D2
:10C3700000000600889FBE008A9FBE008C1F7800C8
:10C38000800478008040EB000A7122004BC0B300AB
:10C39000AC002000811F7800110009008A84D800B9
:10C3A00000047800CF0078000104E00002003A00A9
:10C3B0000800E0000600320001C3B3000140440061
:10C3C000E90007000AC0B9008084540011C0B3001E
:10C3D000811F7800110009000C85D8000005780045
:10C3E000CF0078008B45E900EAFF3A0001C3B300B3
:10C3F00001C04400DC0007004F0678004F05BE0076
:10C400004F04BE0000000600889FBE008A9FBE0049
:10C41000804478008041EB004AC6B3002BC0B300D3
:10C420000980FB000A81FB00110009000280D8008E
:10C430008000FD00014478000304E00002003A009F
:10C440000104E0000600320001C3B30001404400D3
:10C45000C50007000AC0B90080C4540013C0B3006F
:10C460000A80FB00A2002000110009000280D80011
:10C47000004578008B45E900E9FF3A0001C3B300AD
:10C4800001C04400B80007004F05BE004F04BE00C5
:10C4900000000600889FBE008004780030C028009D
:10C4A000EBFE07004448DE006F00600038BF280044
:10C4B00060407C00AC0007006F80640060407C003E
:10C4C000A90007004F04BE0000000600889FBE00C0
:10C4D0008004780000C3B3008500070080C7B30064
:10C4E000830007004448DE006F00600038BF28006A
:10C4F00060407C007E0007006F80640060407C002C
:10C500007B0007004F04BE0000000600889FBE00AD
:10C510008004780030C02800CDFE07004C48DE00C3
:10C5200038BF280060407C008F0007004848DE00CC
:10C530006F00600060407C008B0007004448DE0014
:10C540006F00600060407C00870007006F8064001F
:10C5500060407C00840007004F04BE00000006001D
:10C56000881F78007D00B900D20220001100090068
:10C570000280D8008000FD00420620001100090062
:10C580008280D800010478009FFF0700E0C2B3005A
:10C5900075000700E94F540002003E0000C3B300DD
:10C5A000710007000840780097FF07004F047800EB
:10C5B00000000600220320001241780032E0B7009C
:10C5C0001180BA009100BA000001FD0032E0B7000E
:10C5D0000001FD004800DD000100700000000600C1
:10C5E0000081200010407800E94F50000500320023
:10C5F0000080FB0000004000C1AA2000E08078001D
:10C60000411188000000EB00001188002062A800A2
:10C610001011880021E2A8002342A8008560A9002B
:10C620000000060023C2BF000000D10061006000CE
:10C630000000060022C2BF0061006000000006008A
:10C640000000EB00906A880010002000806A8800DB
:10C65000A081200010A0A1000000060023C2BF009E
:10C660000018A3000E003A00906A80008000E800E5
:10C6700000002100808F500001003A008000EB0094
:10C68000806A8000808F500005003200916A880027
:10C6900070408000614078000080FB00201188001D
:10C6A00000000600826A80007440800003002100C0
:10C6B000906A80008000E800838F500001003A00FB
:10C6C0008000EB00828F50000800320023C2BF00C0
:10C6D0000018A300F6FF3A00916A880061407A00D2
:10C6E0000080FB0020118800F1FF370000000600E9
:10C6F00000417800816A8000906A8000808F50003D
:10C7000004003A00C222A900A081200010A0A000CD
:10C710000A0037007040800082707800806A8000D4
:10C720000000E800806A880001002100810F5000AD
:10C7300002003A000000EB00806A8800000006005A
:10C7400022C2BF000008A300FDFF320030118000AC
:10C750000080FB000000060023C2BF000008A30009
:10C76000FDFF32000000060000417800A18120009A
:10C77000001020001100600005003A0023C2BF0035
:10C780000018A300FDFF3A000200FB002011880002
:10C79000000006000080FB00401188000000060039
:10C7A00022C2BF000000D10061006000000006004E
:10C7B0002222A9000000060095C0BF000048A30087
:10C7C0000D003A004140800050408000810F500031
:10C7D0000900320023C2BF000018A300FDFF3A0089
:10C7E0008580A9009580A8003040800061407800D5
:10C7F0000080FB002011880000000600809FBE0022
:10C80000821F7800321180002140800000408000AB
:10C8100082707800204080000000E80020408800FE
:10C8200011408000810F500001003A009560A9007E
:10C830008560A9004F0178004F00BE00004006004F
:10C84000809FBE00404080008000E800414088009A
:10C8500050408000808F500002003A009580A9006F
:10C860000400370030408000614078000080FB0009
:10C87000201188008580A9004F00BE0000400600FE
:10C88000A0C428002860020000000000000006008C
:10C89000889FBE00C222A800D8000700F8FF07004A
:10C8A000D20007008040780080D620000148780040
:10C8B0000104E000C800350002003A00F0FF070064
:10C8C000F7FF3700E1CF500006003A00CB00070029
:10C8D000F440020000000000C8000700E8FF070065
:10C8E000EFFF3700E2CF500006003A00C300070018
:10C8F000CA57020000000000C0000700E0FF070068
:10C90000E7FF3700E3CF500006003A00BB00070006
:10C91000C649020000000000B8000700D8FF070069
:10C92000DFFF3700E4CF500006003A00B3000700F5
:10C93000F65E020000000000B0000700D0FF070014
:10C94000D7FF3700E5CF500006003A00AB000700E4
:10C950001C4C020000000000A8000700C8FF0700F0
:10C96000CFFF3700E6CF500006003A00A3000700D3
:10C970008676020000000000A0000700C0FF07004C
:10C98000C7FF3700E7CF500004003A009B000700C4
:10C990009A000700BAFF0700C1FF3700EFCF500031
:10C9A00008003A0010C0B300B463020000000000A9
:10C9B000C222A900AC630200000000000000FE00DB
:10C9C000B7FF3700F0CF500003003A000040EB0003
:10C9D00019010700B2FF3700F1CF500003003A0001
:10C9E00010C0B30014010700ADFF3700F2CF5000B4
:10C9F00025003A000000EB0080088800F00888005D
:10CA0000E00C8800CAC6BF0001CEB3000140600040
:10CA10006041B300CAE6B700740007000080FB0065
:10CA20000018A3000100320010A1A8000008A30014
:10CA3000010032001081A8006C0007004804DD00EE
:10CA40006A0007000080FB0000007400D00C880022
:10CA5000C00C880060002000E00C88006300070024
:10CA60004804DD00610007000080FB000000740046
:10CA70006008880011E1A80010C0B300B463020090
:10CA80000000000086FF3700F3CF50000B003A0093
:10CA90000000EB0080088800E00C8800CAC6BF00D8
:10CAA00001CEB30001406000CAE6B70010C0B30079
:10CAB000B46302000000000079FF3700F4CF50009B
:10CAC0000D003A0021E3A800C0C0B300FE7A0200C6
:10CAD000000000000004780021E3A9004800DE0007
:10CAE000B46302000000000008407800B463020054
:10CAF000000000006AFF3700F5CF500015003A0033
:10CB000021E3A800C0C0B300FE7A020000000000CC
:10CB100000047800AC630200000000004840DE0022
:10CB2000B46302000000000008407800B463020013
:10CB3000000000001A63020000000000E14F5000F6
:10CB4000F0FF3A00A06302000000000021E3A9000A
:10CB500053FF3700F6CF500014003A005E38020051
:10CB6000000000000004BE004808DE00B4630200BC
:10CB7000000000004048DE0001002000B463020015
:10CB8000000000004849DD004840DE000000710060
:10CB9000C848DE00B46302000000000008407800CE
:10CBA000B4630200000000003DFF37000168A300ED
:10CBB000050032000140780015000700B463020050
:10CBC0000000000036FF37000040EB00B4630200B5
:10CBD0000000000032FF3700014078004A000700E3
:10CBE000B4630200000000002DFF3700A0630200C4
:10CBF000000000000080FB000000060000C0EB0009
:10CC0000030007000040EB003F00070000000600A3
:10CC1000881F7800004478000081FB00C410DE000B
:10CC2000E1C06000C208DD00C9C2BF000024A1004D
:10CC300001407000C9E2B700C310DE00E1C060002F
:10CC400081C04000C9C2BF000014A10001407000B3
:10CC5000C9E2B700C210DE00E1C06000C9C2BF0077
:10CC60000004A10001407000C9E2B7000201D10038
:10CC70004711DD00C8C2BF000074A100024070006F
:10CC8000C8E2B700E1406400C608DD00C8C2BF00CA
:10CC90000064A10001407000C8E2B700500020000D
:10CCA0002C7C02000000000000CEB3008040640035
:10CCB000CBC2BF000028A300010032000144A00045
:10CCC000CBC2BF000018A300010032000134A00055
:10CCD000CBC2BF000008A300010032000124A00065
:10CCE000CA42E20001003D000114A000CAC2BF0018
:10CCF0000068A300010032000104A0000180FB00D5
:10CD00004F04780000000600881F78000044780077
:10CD10000081FB000268A30003003200C002A900EA
:10CD2000C202A80002003700C002A900C202A90086
:10CD30000258A30003003200C962A800CB62A90018
:10CD400002003700CB62A900C962A900C410DE004E
:10CD5000E1C06000C208DD00CBC2BF000024A1001A
:10CD600001407000CBE2B700C310DE00E1C06000FC
:10CD700081C04000CBC2BF000014A1000140700080
:10CD8000CBE2B700C210DE00E1C06000CBC2BF0042
:10CD90000004A10001407000CBE2B7008200D10086
:10CDA000C708DD00CAC2BF000074A10001407000C6
:10CDB000CAE2B700E1406400C608DD00CAC2BF0095
:10CDC0000064A10001407000CAE2B70050002000DA
:10CDD0002C7C02000000000000CEB3008040640004
:10CDE000CBC2BF000028A300010032000144A00014
:10CDF000CBC2BF000018A300010032000134A00024
:10CE0000CBC2BF000008A300010032000124A00033
:10CE1000CA42E20001003D000114A000CAC2BF00E6
:10CE20000068A300010032000104A0000180FB00A3
:10CE30004F04780000000600881F780080407800CA
:10CE40000040EB0032740200000000000044780053
:10CE50000004E00001003200C222A800084078006F
:10CE6000B4630200000000001A630200000000002A
:10CE70000004E0000D003200A0630200000000008A
:10CE8000E14F40000400320000404400B46302005F
:10CE9000000000000500370010C0B300B4630200BA
:10CEA000000000004F047800000006000804E000C5
:10CEB000EDFF3A00506B80000000E0000D003A00EA
:10CEC0000080EB00506B8800C2C2BF000000D100A0
:10CED000610060000004A20000404000212C2000FE
:10CEE000914078000114A10080C07000010078001A
:10CEF000C2E2B700506B80000000E900506B880070
:10CF0000D9FF370001417800E1D520008048780042
:10CF1000E34F500005003A0000202000006B88001D
:10CF200000082000106B880003003700002020005C
:10CF3000006B8800106B8800E14F51000E0032003A
:10CF400003003900E24F51001F003A00140037007F
:10CF500041C1B30040D620000148780041C6B3006B
:10CF600050D620000148780021C3B30060D62000CD
:10CF7000014878001B00370021C0B30040D62000D4
:10CF800001487800A1C0B30050D6200001487800C5
:10CF900051C0B30060D6200001487800110037006E
:10CFA00011C0B30040D620000148780051C0B30042
:10CFB00050D620000148780021C0B30060D6200080
:10CFC00001487800070037008040EB0040D6200081
:10CFD0000148780050D620000148780060D6200033
:10CFE0000148780000000600889FBE0050D620004F
:10CFF0009040780000302000E2000700CBC2BF0064
:10D000000008A30004003200CBC2BF008004EB0084
:10D010000018A30001003A001900200058D6200093
:10D020009840780000202000E60007009840780033
:10D0300000102000E3000700984078000020200046
:10D04000D0000700090078004F04BE000000060071
:10D05000881F780058D620009840780000302000C3
:10D06000D80007009840780000102000C500070095
:10D070009840780000202000C20007000000EB006C
:10D080004F04780000000600889FBE008A9FBE0003
:10D090008C9FBE008E1F78008001780090AE20002B
:10D0A000104178000280FB000000E9001100200020
:10D0B000800EDD008005EB000204E0001C00320061
:10D0C000830478000005EB008A0578004ED6200026
:10D0D0005CD620000D8064001E41780001202000F5
:10D0E000BF0007009C40780000102000A50007004A
:10D0F00000082000CF000700004478009C40780022
:10D1000000102000AF000700898444008B85450093
:10D110000804E000010032008B05E8000A05E80081
:10D1200090AE20001080FB008A0F5000E9FF3E0007
:10D130000B0078004F0778004F06BE004F05BE0079
:10D140004F04BE0000000600889FBE008A9FBE00FC
:10D150008C1F78008001780090AE2000104178008C
:10D160000280FB000000E90011002000800DDD00BE
:10D170000204E00014003200030478008004EB0095
:10D180004CD620005AD620000B0064001C417800C9
:10D1900001202000920007009A4078000010200033
:10D1A000780007009A4078000010200085000700F2
:10D1B000080444008904E80090AE20001080FB00C1
:10D1C000808F5400F0FF39004F0678004F05BE00F5
:10D1D0004F04BE0000000600889FBE008A9FBE006C
:10D1E00000202000930007000005EB0090AE200017
:10D1F0001004E000150032008004EB0009057800FF
:10D200005BD620009B407800001020005D000700E6
:10D210000020200087000700004478009B40780031
:10D2200000102000670007000A0545000804E00020
:10D23000010032000A05E8008904E80090AE2000F1
:10D240001080FB00890F5000EEFF3E000A007800BE
:10D250004F05BE004F04BE0000000600889FBE00C0
:10D2600028D62000180078007200070059D6200048
:10D270009940780000102000420007001800780054
:10D280006C000700004478009940780000102000EE
:10D290004C0007000884FB00080078004F04BE0023
:10D2A00000000600881F78000080FB0041D62000A7
:10D2B00011417800016B80004900070058D620001A
:10D2C00098407800001020002E0007009840780059
:10D2D000001020003B0007004F047800000006000B
:10D2E000889FBE008A1F7800804478000004E00018
:10D2F0000B0032000044EB005AD620009A40780020
:10D30000001020001F0007009A4078000010200045
:10D310002C0007000844E80088CF5400F7FF3A00CB
:10D320004F0578004F04BE00000006000080FB009F
:10D3300041D6200011417800016B800028000700D1
:10D34000000006000080FB0041D62000114178005B
:10D350000110200022000700000006000080FB00F2
:10D3600041D6200011417800010420001C00070074
:10D3700000000600106B80002E0007000080FB00FC
:10D380000000060000017800A0AF200010407800E7
:10D390007040600005003A0002007800CC22B7001F
:10D3A0000280EA00C822B6000200370002007800BE
:10D3B000C822B7000180FB002C7C020000000000A6
:10D3C000000006000080EA00CC22B600C822B600A9
:10D3D0000180FB002C7C0200000000000000060021
:10D3E0000000E00004003A000180EA00CC22B60010
:10D3F000C822B6000B003700A0AF20001040780014
:10D400007040600005003A0001007800CC22B700AF
:10D410000180EA00C822B60002003700010078004F
:10D42000C822B7000280FB002C7C02000000000034
:10D4300000000600C822B700000000000000000045
:10D44000000000008000EB00CA02B60001003200BC
:10D45000110020000100780000000600EC680200C6
:10D460000000000000000600A468020000000000A8
:10D470000010200000000600F46702000000000019
:10D480008100200000932000827C02000000000048
:10D49000D1002000A0412000DC7C02000000000040
:10D4A0000000060028680200000000006100200063
:10D4B00080932000827C020000000000C100200058
:10D4C00070422000DC7C020000000000000006002A
:10D4D0002E690200000000000080FB000000060032
:10D4E000BA690200000000000080FB000000060096
:10D4F0000040EB00A26902000000000000000600EE
:10D5000010C0B300A2690200000000000000060085
:10D5100010C0B300706902000000000000000600A7
:10D520000040EB00966902000000000000000600C9
:10D5300010C0B30096690200000000000000060061
:10D5400001012000D0982000827C02000000000031
:10D5500080AE20001040780004620200000000004D
:10D5600000C2B300B463020000000000A0AF2000BE
:10D570001080FB004400DE00614060000462020095
:10D580000000000000C2B300B4630200000000000D
:10D590003100200020AE2000827C0200000000004C
:10D5A00000000600881F7800D61D02000000000061
:10D5B0000E1C02000000000000047800D61D0200CE
:10D5C000000000000E1C0200000000008000780037
:10D5D0000800E900E30F5000020036000004EB00F1
:10D5E0000200370080AE20000848E9000100E90091
:10D5F000E10F500008003E00A0AF2000E1C0600035
:10D60000C408DD00104178000244A1000148710007
:10D610000800E0001F003A000004EB006865880085
:10D62000B103200080452000DC7C020000000000E7
:10D630008801780042002000110020001000200026
:10D64000DC1E02000000000081AE20008048E900DE
:10D65000F1042000E0932000DC7C020000000000C8
:10D660008801780022002000110020001000200016
:10D67000DC1E020000000000A2AF2000614060003C
:10D680004400DD00924078000144A10000C9700010
:10D6900001003700AAFF07004F04780000000600D1
:10D6A000CB02A900CB22A900C922A800C902A90067
:10D6B00080AE20009040780020C0B3008267020056
:10D6C0000000000000000600E10F500009003200D9
:10D6D00003003900E20F500009003A00060037004D
:10D6E00081032000D0992000827C0200000000000D
:10D6F000070037000C0007001F0007000400370078
:10D7000041022000E01D2000DC7C0200000000003F
:10D7100000000600B1002000600B2100DC7C02004C
:10D720000000000000000600F1032000509D2000D2
:10D73000DC7C0200000000000040EB00AE6902004B
:10D7400000000000F00F20002C7C02000000000010
:10D7500010C0B300AE6902000000000010C0B300AA
:10D7600070690200000000000040EB00AE6902009A
:10D7700000000000000006000400FA00889FBE00C0
:10D78000D102200040A12000827C020000000000A5
:10D7900068845700E4845700EC6802000000000031
:10D7A000005C78000080FB004A620200000000007C
:10D7B00000C2B300B463020000000000888F540070
:10D7C000F5FF3A00E0C528004060020000000000BC
:10D7D000A100200010A42000827C020000000000B4
:10D7E0008FF897000180FB004400DE00E94F5000F5
:10D7F0000E00320003003E00E84F50001A003A00CD
:10D8000005003700EA4F50000D003200EF4F500086
:10D8100015003A000F00370061002000B0A420007E
:10D82000827C02000000000013003700610020002D
:10D8300010A52000827C0200000000000E003700CE
:10D840006100200070A52000827C02000000000022
:10D850000900370031002000D0A52000827C0200A2
:10D8600000000000040037007100200000A6200026
:10D87000827C020000000000E0C528004060020039
:10D8800000000000B100200070A62000827C020091
:10D89000000000001FFC97000878A30005003A0074
:10D8A0006100200020A72000827C02000000000010
:10D8B00004003700F100200080A72000827C0200D5
:10D8C00000000000E0C528004060020000000000E9
:10D8D000C100200070A82000827C0200000000002F
:10D8E000080078008007B2004380DE000041780025
:10D8F0000004E00005003A00D100200030A920001B
:10D90000827C0200000000001000370000042000AC
:10D910008040EB00EF4F510005003A00310020003D
:10D92000D0A52000827C0200000000000700370024
:10D93000000040008140E800814F5100FCFF3A00A8
:10D9400082FF9F00BA61020000000000E0C52800CD
:10D9500040600200000000009101200000AA2000A9
:10D96000827C0200000000001FF897006741600001
:10D9700010002000060032008040EB001000200064
:10D98000000040008140E800814F5100FCFF3A0058
:10D990000462020000000000E0C5280040600200B0
:10D9A000000000004F04BE000080FA0000000600E6
:10D9B0000C080000120000000200000000009400AB
:10D9C0000D0000000000000000000000000000004A
:10D9D00000000000E80A00001A000000000000003B
:10D9E000940D00000010000000000000020B000079
:10D9F00002000000000000001E0800000C000000F3
:10DA00000200000000181C001D0018001C1D03006F
:10DA10000B131B00040B00000600000000000000B8
:10DA20000A0B000008000000000000002A080000A7
:10DA30000201000002000000F0005E00BCE2610094
:10DA40003FDD8300C29C7E0020A3FD001F419D009E
:10DA5000C3217F00FCA240001E5F0100E3BD3E0029
:10DA60006082DC00237D9F00C1421C00FEA0E1001B
:10DA7000BF5D030080DE3C0062BEE000025CDF00B0
:10DA800081633D007C22C0009E1D4300A1FF460033
:10DA900018FAA40027799B00C584DA003866E500EF
:10DAA000BB590700DB85670039BAE4000658190046
:10DAB00047A5FB007826C4009A653B00D98704007F
:10DAC0005AB8E600A7F91B0045C698007A24F8006A
:10DAD000A6441A0099C725007B3A640086D85B00EB
:10DAE00005E7B9008CD230006EEDB300510F4E0047
:10DAF00010F2AC002F719300CD114F00ADF3700008
:10DB00002ECC9200D38D6F0031B2EC000E50AF00DE
:10DB1000F1134D00CE9072002C6D3300D18F0C00AC
:10DB200052B0EE00326C8E00D0530D00EFB1F00019
:10DB3000AE4C120091CF2D0073CA94007628AB0032
:10DB4000F51749000856B400EA693700D58B57002D
:10DB500009EBB50036688A00D495CB002977F4002C
:10DB6000AA481600E9B755000B88D600346A2B0086
:10DB70007597C9004A14F600A8742A00C8961500C3
:10DB80004BA9F700B6E80A0054D789006B350000AE
:10DB9000120B00007000000000000000820B00006B
:10DBA00026000000000000002C0900008001000099
:10DBB00002000000308030008030800030803E0065
:10DBC000804E8000308030008030800030804E00F9
:10DBD000803080004E804E00805E80006C806C0043
:10DBE0008078800084808E00804869005A000000A0
:10DBF00000000000BA5CBA005C3080003080200079
:10DC00005A165A003080300080505A00425A3C0068
:10DC10005A325A00285A4E00806E5A00605A6000EC
:10DC20005A788000B05C8E0080312D005749520038
:10DC300045000000C647C60047DA4700DA4724001F
:10DC400044D64300308030008030800030804E0069
:10DC5000803080004E80EC0047B64600B8443E005D
:10DC600046B0460058482C0044554100525400002C
:10DC7000000000007A547A0054CC5400CC541800B0
:10DC800054DA5300308030008030800030804E0005
:10DC9000803080004E804E0080B255002E558A00A4
:10DCA00055A45500A0560400554932004300000019
:10DCB00000000000563B34003B783B0030809E0063
:10DCC0003B963B00308030008030800030804E003A
:10DCD000803080004E804E0080CE3D00283CA80061
:10DCE0003DCA3D008E3EB2003B535000490000004B
:10DCF000000000003C6A3C006A526A00526A34002C
:10DD00006A2E6A00806A78006A986A00906A7000D9
:10DD10006A886A00686A4E0080646B00D26A5000AC
:10DD20006B7880008A6BA0006A3257004952450028
:10DD300000000000F078BE00782279002279AA0065
:10DD400078A278006C797400797C790084795C0021
:10DD50007964790054794E00805E8000CC798C0023
:10DD60007A788000A87A8C007933570049524500B0
:10DD700000000000DC71DC0071EA7100EA71CA0089
:10DD8000714E8000308030008030800030804E0046
:10DD9000803080004E804E00803C7200F871FE00A2
:10DDA00071123F0072738E00804C430044000000EB
:10DDB00000000000A80B0000A80100000000000007
:10DDC000AC0A00001200000002000000143404003D
:10DDD0000D8206004003A00001CF00006700440050
:10DDE00000220000500D00000400000000000000B0
:10DDF000000800000C00000000000000BE0A000047
:10DE00002800000002000000143404000D82060007
:10DE10004003A00001CF0000670044000022000082
:10DE20007F00140034040D008206400003A00100AE
:10DE3000CF007F00006700004400220000000000C7
:10DE4000540D000008000000000000005C0D000000
:10DE500002000000000000005E0D00000A0000004B
:10DE600000000000680D0000040000000000000039
:10DE7000E60A0000020000000200000003000000AB
:10DE80006C0D00000E000000000000007A0D000084
:10DE900002000000000000007C0D000002000000F5
:10DEA000000000007E0D00001600000000000000D1
:10DEB00000000000007C2000C822B7000F0007000F
:10DEC00020C0B300210007001A6302000000000018
:10DED0000004E00005003200A06302000000000022
:10DEE0001A0007000004E00003003A00F8000700F1
:10DEF0000004E000F4FF320000000600C222A90086
:10DF00000001EB00420388005203880002038800EE
:10DF100012038800F2088800ADC0BF00F1C8B3004A
:10DF200001406000ADE0B700E20888000064200016
:10DF3000D008880000002100906C880000D92000E3
:10DF400002487800F26B88000000060080417800EB
:10DF5000406C8000E10F5000700032000300390077
:10DF6000E20F5000D8003A0076003700E2CF5100AF
:10DF70001000320005003E000304E0000A003200F9
:10DF8000E1CF51005A003A000F003700F1CF5100A5
:10DF9000CD003200F3CF5100CB003200E4CF51006E
:10DFA00053003A001A003700D4FF07001000200089
:10DFB000C600370080C3280028600200000000006F
:10DFC0000000EB00C1003700C222A8000001EB00F6
:10DFD000F2088800B2088800A208880080002000AB
:10DFE000F00888008660A9009660A900ADC0BF0057
:10DFF000F1C8B300014060000044A000ADE0B700EC
:10E0000010002000F06B880002007800AF0037009D
:10E0100010C0B300B463020000000000D0C32800A9
:10E0200028600200000000000040EB00B463020022
:10E030000000000010C2B300B46302000000000042
:10E040000040EB00B4630200000000000040EB0061
:10E05000B46302000000000000C1B300B46302001A
:10E06000000000000040EB00B4630200000000006C
:10E0700030C2B300B4630200000000000040EB00B7
:10E08000B463020000000000F0C0B300B4630200FB
:10E090000000000020C4B300B463020000000000D0
:10E0A00000C4B300B46302000000000000C4B30069
:10E0B000B46302000000000050C0B300B46302006B
:10E0C0000000000010C4B300B463020000000000B0
:10E0D00020C0B300B4630200000000000040EB0069
:10E0E000B4630200000000000000EB00770037007E
:10E0F00000D820000348780041C0B30050D8200069
:10E100000148780060D820000048EB001000200093
:10E11000406C88000000EB006C00370062D82000E3
:10E120001240E800004978000080FB0001D8200080
:10E1300003F0780050D8200012417800904F510031
:10E140006100390000D820009040780010C8B3006A
:10E1500080CF50001900320000CCB30080CF5000B7
:10E160000400320000C8B30080CF500053003A00D2
:10E170002000370010D82000104078008080FB007D
:10E180000148A300010032006200A8000138A3008A
:10E190000100320062A0A8000128A30001003200A3
:10E1A00062C0A8000118A3000100320062E0A800CC
:10E1B0000008A300010032006300A80020D820005E
:10E1C0001080FB004800DD0011D820009180FB008A
:10E1D000010070004200DD0064004000906C880087
:10E1E00001002100810F500034003600916C88003E
:10E1F0003200370030D82000104078004800DD00A1
:10E200000100200022D82000124178000281FB008A
:10E21000030020000200700083807000C808DD0049
:10E220000080FD00804078000040EB0012D8200004
:10E23000124178000281FB00030020000200700000
:10E24000838070004209DD00CE00DE008100710095
:10E250004200DD0064004000E080480092012000A0
:10E26000030020000C09020000000000506C880030
:10E27000616C8800F00F5000E08F580005003600F8
:10E2800070005000E0805800506C8800616C88007D
:10E29000040037001000200001002000506C8800AE
:10E2A000616C8800526C8000636C80004018DE0056
:10E2B00001002000E0088800D20888000000EB0080
:10E2C000406C8800010037000000EB0000000600F1
:10E2D000F06B8000E10F50002C003A0086C0BF00B8
:10E2E0000038A30002003A006200E20027003A0072
:10E2F0001FE1A8008780A9000000EB00706C880077
:10E30000916C80000100E0000E00320000017800F6
:10E31000501680004600DE007140800000F1780059
:10E3200087C0BF000048A300FDFF32008780A9001E
:10E330000201E800916C8000810F5100F4FF390068
:10E34000726C88000000EB0010038800F008880061
:10E35000716C88000100E00009003200704080000C
:10E360000100400070F89700B46302000000000054
:10E37000706C80008000E900716C8800F7FF3A0043
:10E38000DEFE070010002000010037000000EB0057
:10E3900000000600A1D720009180FB008100D10081
:10E3A00061C1600080407800024078000A010700E7
:10E3B0000010200000000600A0D720001014A100CB
:10E3C0004101200050EE2000DC7C02000000000033
:10E3D00000000600A0D720001014A000210120009A
:10E3E00090EF2000DC7C020000000000000006002E
:10E3F000A0AF20001044A00000000600A0D720001D
:10E400001014A000A8C6BF0001CEB30001406000F8
:10E410007040B300A8E6B700C9C6BF000140600065
:10E420007040B300C9E6B700C8C6BF000140600035
:10E430000034A000C8E6B700CAC2A900C8C2A9003B
:10E44000C902A900C8E2A800C922A900D01320006F
:10E45000101288000000EB002012880000128800D3
:10E4600041E2A800D1012000E0F12000DC7C0200A4
:10E470000000000000000600889FBE008A1F780090
:10E4800000047800506580000000E8000080FB0078
:10E4900050658800D61D0200000000000E1C02001E
:10E4A00000000000800478000000EB006065880038
:10E4B000E30F54003000320003003E000800E0008B
:10E4C000080032000C003700E60F54003E00320016
:10E4D000E70F54005C003200E40F54007A003A0069
:10E4E000300037008109200000F82000DC7C0200A9
:10E4F000000000007800370051002000506020002C
:10E50000DC7C02000000000095000700E10F5400D1
:10E51000710032000900E900E10F500011003600DF
:10E520004102200080012100DC7C0200000000008C
:10E530008001EB00220020001100200020002000BC
:10E54000DC1E020000000000E10F500003003A0052
:10E550000040EB00680007000200370080C0B300F5
:10E560006500070041002000C0032100DC7C0200A0
:10E57000000000005800370011C0B3000040EB005D
:10E5800095000700F0002000087C02000000000059
:10E590005100200000042100DC7C0200000000008B
:10E5A0004D003700894078000174A0000040EB0066
:10E5B00089000700A100200050042100DC7C02003B
:10E5C000000000004400370011C0B3000040EB0021
:10E5D00081000700F0002000087C0200000000001D
:10E5E0000900E00004003A00080320000905780053
:10E5F0000905200009003700080320000005EB0092
:10E600000900E00005003C003300370090032000C3
:10E61000800F540001003600080320008840780075
:10E6200010C0B3006C00070008407800B46302001B
:10E63000000000000804E8000A05E8008A8F540082
:10E64000F2FF3A002400370011C0B3000040EB0095
:10E6500061000700F0002000087C020000000000BC
:10E660000900E00004003A001802200009057800C3
:10E670000905200009003700180220000005EB0002
:10E680000900E00005003C0013003700F0072000FF
:10E69000800F5400010036001802200088407800E6
:10E6A00010C0B3004C00070008407800B4630200BB
:10E6B000000000000804E8000A05E8008A8F540002
:10E6C000F2FF3A000400370041022000E01D200064
:10E6D000DC7C0200000000004F0578004F04BE0003
:10E6E00000000600B1002000600B2100DC7C02006D
:10E6F000000000000000060002C2B300824040009B
:10E700000040EB0034000700F0002000087C02000D
:10E710000000000081C0B3000040EB002E000700A5
:10E72000F0002000087C02000000000011C0B300CF
:10E730000040EB0028000700F0002000087C0200E9
:10E7400000000000E1C0B3000040EB002200070021
:10E75000F0002000087C020000000000000006001D
:10E760000040EB003A000700F0002000087C0200A7
:10E770000000000031C0B3000040EB0022000700A1
:10E7800050002000087C02000000000031C0B300EF
:10E790000040EB001C000700000A20002C7C020057
:10E7A0000000000031C0B3000040EB00160007007D
:10E7B000000A20002C7C02000000000021C0B300F1
:10E7C0000040EB0010000700000A20002C7C020033
:10E7D0000000000000000600889FBE008044780012
:10E7E000014478008180FB00C408DE0006000700B9
:10E7F0006F446400884078000940780002000700F8
:10E800004F04BE0000000600881F7800C408DD0029
:10E81000014478000804A000E14F500002003A00D3
:10E82000014478003840B300084078000800070031
:10E830000834A00008407800050007000840780070
:10E840000034A100020007004F0478000000060019
:10E850002E3F020000000000CAC2A800CAC2A900E0
:10E8600000000600889FBE008A1F780000457800DF
:10E8700081447800C0D520000048EB000A04E00085
:10E8800003003A00A08120001080A0000C00370097
:10E890000104E0000A003200F103200050AE200025
:10E8A000DC7C02000000000011012000A019210002
:10E8B000DC7C020000000000A063020000000000F9
:10E8C0004100200040B22000DC7C0200000000007B
:10E8D000CB42A800C942A9003100200080B220002C
:10E8E000827C020000000000CBC2BF004200DE00BC
:10E8F0006100600011C0B300F2000700CB42A90024
:10E90000C942A800C222A800C022A900810020009C
:10E91000B0B22000827C020000000000C2C2BF0032
:10E920000000D1006100600011C0B300E5000700E5
:10E93000C222A900C962A800CB62A9008100200000
:10E9400030B32000827C020000000000CBC2BF0078
:10E950004300DE006100600011C0B300D900070071
:10E96000CB62A900C962A90081002000B0B32000D9
:10E97000827C020000000000CBC2BF004300DE002A
:10E98000610060008040EB00CE000700C002A900DB
:10E99000C202A80020002000087C02000000000045
:10E9A0004100200030B42000827C02000000000002
:10E9B000C2C2BF006140600011C0B300C1000700C7
:10E9C000E100200070B42000DC7C020000000000A8
:10E9D00021E3A8002100200050B52000827C020025
:10E9E0000000000072352000712B200090C0B300A1
:10E9F000710007000904E000080032003100200027
:10EA000070B52000827C02000000000072352000FA
:10EA1000712B2000B0C0B300670007004100200048
:10EA2000A0B52000827C020000000000022520002A
:10EA3000011B2000A0C0B3005F0007000904E00034
:10EA40000800320031002000E0B52000827C020086
:10EA50000000000002252000011B2000C0C0B30000
:10EA60005500070021E3A9008100200010B6200016
:10EA7000DC7C020000000000F8C32F000004FD0051
:10EA8000C822B6000004FD00003C2000CC22B700E4
:10EA900040062000087C02000000000010C0B30007
:10EAA00061000700A100200090B62000DC7C02007D
:10EAB000000000000004FD00CC22B6000004FD00B0
:10EAC0000904E00002003200C962A800CB62A9007C
:10EAD00040062000087C0200000000000040EB001F
:10EAE000510007000904E0000B003200A1002000E3
:10EAF00030B72000DC7C020000000000003C200059
:10EB0000C822B70040062000087C02000000000078
:10EB100010C0B300440007000A04E00012003200F5
:10EB20000904E00010003200C002A900C202A800DF
:10EB3000C422A80001022000D0B72000DC7C020023
:10EB400000000000F1002000B0182100DC7C020071
:10EB500000000000A063020000000000C422A90021
:10EB6000C002A900C202A900C07A02000000000091
:10EB700061002000D0B92000827C0200000000006B
:10EB8000C8D5200018407800046202000000000090
:10EB90008100200030BA2000DC7C02000000000070
:10EBA000A08120001080A1001880FB004F05780094
:10EBB0004F04BE0000000600889FBE008A1F780038
:10EBC00000447800810478000205780080C2B30018
:10EBD000B46302000000000008407800FE7A0200E2
:10EBE0000000000000047800B06202000000000095
:10EBF00090C2B300B463020000000000890F54000B
:10EC000003003600100020008A0F54000100390074
:10EC10000000EB0011C0B3002A0007004F05780088
:10EC20004F04BE0000000600881F780000447800F2
:10EC300041002000B0BA2000827C020000000000E9
:10EC4000CBC2BF000000D1006100600088407800A6
:10EC50001C00070031002000F0BA2000827C020076
:10EC600000000000CBC2BF00614060008840780017
:10EC7000140007004100200020BB2000827C02001D
:10EC800000000000CAC2BF000080FB004700DE0099
:10EC9000884078000B0007002100200060BB2000A6
:10ECA000827C020000000000CAC2BF004600DE00F5
:10ECB0006100600088407800020007004F0478007F
:10ECC00000000600814F500005003A00310020008E
:10ECD00080BB2000DC7C0200000000000600370042
:10ECE00051002000B0BB2000DC7C020000000000CE
:10ECF000C0D520001048E8000000060060C52800CC
:10ED0000286002000000000000000600889FBE008E
:10ED10008A9FBE007940800010002000E06B8800D0
:10ED2000F6FF07008005EB00A06302000000000072
:10ED3000E34F50001200320004003E00E14F50004B
:10ED40003100320034003E0096003700E64F50009C
:10ED50000900320003003E00E54F50008B003A00EE
:10ED600063003700E74F50003E003200E84F50008C
:10ED700086003A0031003700E0FF0700EAFF370065
:10ED800030C0B300804C780080C0B300904498003D
:10ED900021E3A800C0C0B300FE7A0200000000001A
:10EDA000C800DE00A1449800B0449800B0C0B30091
:10EDB000FE7A020000000000C800DE00C144980096
:10EDC000D0449800A0C0B300FE7A0200000000000A
:10EDD000C800DE00E1449800F044980090C0B30001
:10EDE000FE7A020000000000C800DE00814C98009E
:10EDF000904C980021E3A900A100200009007800B0
:10EE00008E000700C8FF3700A0630200000000006A
:10EE100067000700C4FF3700A06302000000000085
:10EE200000447800A06302000000000080407800E9
:10EE30000840780091000700BBFF3700A063020084
:10EE40000000000000447800A06302000000000001
:10EE5000C840DD000080FB0000807000E06B88008F
:10EE6000B1FF3700A0630200000000000085FB0036
:10EE7000E14F500004003A0030C0B300CA63020002
:10EE8000000000000300370020C2B300CA63020084
:10EE900000000000A06302000000000000447800B1
:10EEA000A06302000000000080407800A0CAB30008
:10EEB000804F540003003A0050C5B30080CF50008B
:10EEC0000400320020C2B300CA6302000000000048
:10EED0000005EB0070C0B300804C78009A449800A5
:10EEE0002100200009007800540007008EFF370041
:10EEF000A06302000000000000457800A06302004B
:10EF000000000000004178008560A900C850DD00C5
:10EF10000080FB000084700000002200800F54007D
:10EF2000010036000004780050C0B300804C780027
:10EF30009A449800A244980031002000090078000B
:10EF40003E0007007040800000408800E700440059
:10EF5000C308DE0081804000114088002B408800FB
:10EF60004183200081004000314088004B408800F0
:10EF70005B4088009560A800E36B80000801780082
:10EF8000AC7F02000000000067FF37008B4C780068
:10EF90009B4498001100200009007800270007001A
:10EFA00061FF37004F05BE004F04BE0000000600A1
:10EFB000CAC2A900CB22A900CB02A900CB42A9005A
:10EFC000CA02A900E24F500006003A00CAC2A800D7
:10EFD000CB02A800CB22A800CB42A800CA02A800FE
:10EFE00005003700CAC2A900CB02A900CB22A900A4
:10EFF000CB42A900CA02A9000040E900E14F50003D
:10F0000007003E00C8C2A900C922A900C902A90080
:10F01000C942A900C802A900C8E2A800060037003A
:10F02000C8C2A800C922A800C902A800C942A800F5
:10F03000C802A800C8E2A80000000600889FBE0021
:10F040008A1F780000057800810478000100E00044
:10F05000070032000004EB0068407D00B46302004A
:10F06000000000000804E800888F5400FAFF3A000E
:10F070004F0578004F04BE0000000600E44F50002A
:10F080002300320005003E00E14F5000080032002E
:10F09000E24F50002A003A000D003700E84F5000C0
:10F0A00021003200F04F500025003A0010003700D8
:10F0B000C022A900E1C0600081C04000C2C2BF0000
:10F0C0000014A10001407000C2E2B7001C0037002C
:10F0D0000104E00003003200C002A900C202A8003F
:10F0E00017003700C002A900C202A90014003700AF
:10F0F0000104E00003003200C962A800CB62A9004D
:10F100000F003700CB62A900C962A9000C003700CC
:10F11000E1C06000CAC2BF000004A100014070004D
:10F12000CAE2B70006003700E1C06000C208DD0097
:10F13000CBC2BF000024A10001407000CBE2B700A9
:10F1400000000600F00F20004468020000000000EC
:10F150000000060044680200000000008000780003
:10F16000A0AF200002C4B3001040610001003A00CB
:10F170008000EB000100780000000600A0AF200036
:10F180001064A00020B020001040780061406000B2
:10F19000040032000040EB00AE69020000000000F5
:10F1A0000300370010C0B300AE6902000000000089
:10F1B00020B0200010407800614060000300320061
:10F1C000F0C2B300B463020000000000A100200000
:10F1D00090AB2000DC7C0200000000000000060074
:10F1E000A0AF20001064A10020B0200010407800E3
:10F1F00061406000040032000040EB00AE69020094
:10F20000000000000300370010C0B300AE69020028
:10F210000000000020B02000104078006140600035
:10F2200003003200F0C2B300B4630200000000002B
:10F23000A100200090AB2000DC7C02000000000058
:10F2400000000600A0AF20001064A10020B0200044
:10F2500010407800614060000400320010C0B3002C
:10F26000AE69020000000000030037000040EB0020
:10F27000AE6902000000000020B0200010407800BD
:10F280006140600003003200F0C2B300B4630200CA
:10F2900000000000B100200030AC2000DC7C020047
:10F2A00000000000000006002E69020000000000BF
:10F2B0000080FB0000000600BA69020000000000A8
:10F2C0000080FB000000060010C0B300706902005F
:10F2D000000000000000060010C0B300A269020098
:10F2E00000000000000006000040EB00A2690200E0
:10F2F000000000000000060010C0B3009669020084
:10F3000000000000000006000040EB0096690200CB
:10F31000000000000000060041012000E0AC2000D9
:10F32000827C02000000000080AE200010407800C7
:10F33000046202000000000000C2B300B4630200D7
:10F340000000000020B02000104078006140600004
:10F35000046202000000000000C2B300B4630200B7
:10F3600000000000A0AF20001080FB004400DE0081
:10F3700061406000046202000000000000C2B300AF
:10F38000B46302000000000000C6280040600200D4
:10F390000000000000000600889FBE00D61D02008D
:10F3A000000000000E1C02000000000000047800B5
:10F3B000D61D0200000000000E1C0200000000002C
:10F3C00080047800D61D0200000000000E1C020020
:10F3D00000000000000178000800E900E30F500081
:10F3E000020036000004EB000200370080AE20006F
:10F3F0000848E9000900E900E10F5000020036006A
:10F400000004EB000500370021B020000940E900AE
:10F41000614060001104A100914870000200E90001
:10F42000E10F500008003E00A0AF2000E140610065
:10F43000C408DD00104178000244A10001487100B9
:10F440000800E0002E003A00B103200080452000B3
:10F45000DC7C0200000000008001EB004200200084
:10F460001100200010002000DC1E0200000000003F
:10F4700081AE20008048E900D1012000601C2100FD
:10F48000DC7C0200000000008001EB002200200074
:10F490001100200020002000DC1E020000000000FF
:10F4A00021B020000040E900614060001104A1008B
:10F4B00091487000F1042000E0932000DC7C020001
:10F4C000000000008001EB0022002000110020005D
:10F4D00010002000DC1E020000000000A2AF20008F
:10F4E000614060004400DD00924078000144A100CA
:10F4F00000C970000000EB00606588000100370063
:10F5000085FF0700A1AF2000F0C9B300914860005B
:10F510004F04BE000000060080AE2000904078003E
:10F5200030C0B3008267020000000000C922A900B9
:10F53000C902A900C8E2A80020B02000104078004D
:10F5400061406000AE69020000000000000006009B
:10F550000101200040062100DC7C020000000000C8
:10F5600000000600A1AF20001141780080AE20000D
:10F570000048EB0000CEB3008048610000000600A8
:10F58000889FBE00C922A800C902A800C8E2A8003E
:10F59000C8C2A800C942A800C222A900C022A9006E
:10F5A000CAC6BF0009CEB30009406000CAE6B70072
:10F5B0000004EB00A8408800EAFF0700CB62A90026
:10F5C000C962A900C002A900C202A9002D83A90036
:10F5D0002D43A9002D23A9002D63A900094078001F
:10F5E0002063B7008819880020F0210020198800C6
:10F5F000181988004F04BE00000006000080FB00C0
:10F60000401988002023A8002003A90020C3BF00C0
:10F610000008A300FDFF3200001880000000060073
:10F6200021E3A800C0C0B300F4FF0700B0620200ED
:10F630000000000021E3A90000000600881F7800F8
:10F64000E1002000E0352000DC7C0200000000002A
:10F65000F1002000B0182100DC7C02000000000056
:10F66000F1002000C0362000827C02000000000073
:10F670000000EB00B062020000000000110020005A
:10F68000B0372000827C0200000000000F0037002D
:10F6900021E3A800C0C0B300D8FF07000004780031
:10F6A00021E3A90020C42800286002000000000017
:10F6B00008007800B0620200000000001100200085
:10F6C000B0372000827C0200000000001A630200B4
:10F6D000000000000004E000EDFF3200A063020023
:10F6E0000000000080C4280040600200000000000C
:10F6F0004F04780000000600881F7800000478009E
:10F7000090AE200010407800EF4F500005003E0002
:10F710008080FB00EF801000F0FF27000180DE00FA
:10F720000004640090408000E10F5000120032009D
:10F7300005003900E20F50001B003200E30F5000BB
:10F7400031003A0026003700A0AF200001C2B3000C
:10F7500010C06000040032000800780086620200D9
:10F760000000000028003700080078004A6202000C
:10F770000000000024003700A0AF200001C2B30049
:10F7800010C060000400320008007800BA61020076
:10F79000000000001C0037000840780004620200EE
:10F7A0000000000018003700A0AF200001C2B30025
:10F7B00010C060000600320008407800606002005F
:10F7C0000000000000C2B300B463020000000000AB
:10F7D0000840780060600200000000000A00370066
:10F7E000A0AF200001C2B30010C0600003003200CF
:10F7F0004840DE00B46302000000000008407800CA
:10F80000B4630200000000004F047800000006000E
:10F81000889FBE008A1F7800000578000000E00085
:10F820000A0034008004EB000004EB00A00F20006D
:10F83000090007000804E800E40F5400FBFF3A0049
:10F840008904E800890F5500F7FF3A004F0578005A
:10F850004F04BE00000006000000E0001400340069
:10F860008000EB000000000000000000000000002D
:10F870000000000000000000000000000000000088
:10F880000000000000000000000000000000000078
:10F890000000000000000000000000000000000068
:10F8A000000000008100E800810F5000EDFF3A00E9
:10F8B00000000600000278008001EB00110020002B
:10F8C000020120008381410001006200010032003A
:10F8D0000300A000818040000201E900F9FF3A0026
:10F8E00090AE200010407800F04F5000030032002E
:10F8F0000080FB00700010008019DE00030078001B
:10F9000000000600889FBE008A9FBE008100400064
:10F91000810F500025003D000004780039002000D0
:10F92000EB3B220001057800110009000904D80012
:10F930000100E00006003A00000040000B0040001B
:10F940001000BA00B4630200000000001400370089
:10F95000E18F500009003A00110009000904D800A5
:10F96000000040000B0040001000BA004800DE001C
:10F97000B46302000000000009003700E28F50006D
:10F9800007003A00110009000904D80000004000F7
:10F990000B0040001080BA00B463020000000000B9
:10F9A0000804E800880F5500DFFF3A004F05BE004D
:10F9B0004F04BE0000000600D2FF070040C628002A
:10F9C000406002000000000000000600110220005C
:10F9D00040272100F8FF0700C10420005029210022
:10F9E000F5FF070061022000102E2100F2FF070042
:10F9F0008102200070302100EFFF0700510120003C
:10FA0000F0322100ECFF0700B1012000403421005A
:10FA1000E9FF070081022000F0352100E6FF070022
:10FA2000B101200070382100E3FF0700E10220004F
:10FA3000203A2100E0FF070051012000003D210095
:10FA4000DDFF070031022000503E2100DAFF0700F1
:10FA5000E102200080402100D7FF0700C101200003
:10FA600060432100D4FF070011022000204521003F
:10FA7000D1FF0700C101200030472100CEFF070061
:10FA800051022000F0482100CBFF070011022000A6
:10FA9000404B2100C8FF070091012000504D21007C
:10FAA000C5FF0700F1012000E04E2100C2FF070062
:10FAB00091022000D0502100BFFF0700510220001A
:10FAC00060532100BCFF070061032000B0552100F6
:10FAD000B9FF0700E103200010592100B6FF07001D
:10FAE00000000600881F7800E100200070912000CF
:10FAF00084FF0700A06302000000000000447800BB
:10FB0000B46302000000000040C62800406002000C
:10FB10000000000090C7B300804F54000400320082
:10FB20008000EB0090C5B300804F540001003A0004
:10FB300011002000010078004F047800000006004A
:10FB400004000700660C0200000000000000EB004B
:10FB5000000006000400FA00881F7800F0FF2F0064
:10FB600001002000D0BF9F00E1BF9F004507A90012
:10FB70002CA3EF004227A9000080EB008080EB005F
:10FB80005FB99700EFB9970061015100E08159001A
:10FB9000D2BF9F00E3BF9F005FB99700EFB9970006
:10FBA000800F5100818F5900F5FF3A00A4C6BF00B5
:10FBB00001CEB300014060005040B300A4E6B7009E
:10FBC000C4C6BF00014060003040B300C4E6B700C7
:10FBD00081C0B30000812000014878000004EB00E0
:10FBE00098408800C07A020000000000F062020025
:10FBF0000000000068C0A80068E0A8008800780045
:10FC0000F00F2000DA62020000000000B04088001F
:10FC100021002000F00F2000DA6202000000000046
:10FC2000C0408800501680000080FB004200DE00CB
:10FC300063406000E34F500004003A0011C6B30077
:10FC4000A0812000014878000B003700E24F5000EF
:10FC500004003A0021C6B300A081200001487800CA
:10FC6000050037000004E00003003A0051C3B30070
:10FC7000A08120000148780068C0A90068E0A900C0
:10FC8000A08120001080A10081C0B30090AE2000B0
:10FC9000014878003260EF00C0C5280040600200D3
:10FCA00000000000FA1F0200000000004F0478006E
:10FCB0000080FA0000000600889FBE00C922A8004C
:10FCC000CB22A900C922A90028022000A000200000
:10FCD0002C7C0200000000000804E900FBFF3A0051
:10FCE000C922A800100420002C7C020000000000A3
:10FCF000CBC2BF00E204600038022000A000200058
:10FD00002C7C0200000000000804E900FBFF3A0020
:10FD1000CBC2BF00110020000018A3000100320078
:10FD20008980FB00010078004F04BE00000006003F
:10FD3000881F780000447800C922A800CB22A900BF
:10FD4000C922A900400020002C7C02000000000015
:10FD50000804E00001003200C922A8008000200051
:10FD60002C7C0200000000000804E00007003200C4
:10FD7000CBC2BF000000D10061446000000220003F
:10FD80002C7C0200000000000800370090012000D9
:10FD90002C7C020000000000C922A8007000200096
:10FDA0002C7C0200000000000044EB00500020000A
:10FDB0002C7C0200000000000880FB004F0478004B
:10FDC00000000600889FBE000044780089C0B30090
:10FDD00061406400D6FF07008880FB000104D10069
:10FDE0000004E000010032000874A0008944E9002A
:10FDF000F7FF3A00800020002C7C02000000000089
:10FE00000880FB004F04BE0000000600E1C0600057
:10FE100081C04000F52C2000954278000514A10017
:10FE200081C272008002FD00CFE2B7008002FD00B7
:10FE3000616A20009140780005CEB30085C0600063
:10FE40007140B3008000FD00A6E6B7008000FD0011
:10FE5000916C20009140780085C060005140B30053
:10FE60008000FD00C9E6B7008000FD00C0118800D9
:10FE70008002EB00851188003062A80061416100BA
:10FE8000C410DD0030C2BF000044A100014070007A
:10FE900030E2B700E3C1610083C1410030C2BF005E
:10FEA00091CFB300014060000340700030E2B70022
:10FEB0006142620030C2BF000004A1000440700033
:10FEC00030E2B700951188004611DD0033C2BF0053
:10FED0000064A1000240700033E2B7000000060099
:10FEE00031E2A8003342A80087C0A900C922A900B6
:10FEF0000000060031E2A9003342A900F0C1B300BE
:10FF0000A666B700C9C6BF0001CEB30001406000BD
:10FF1000C9E6B700CF22A900C922A8000000060048
:10FF20008000780033C2BF000018A300FDFF3A0034
:10FF3000A11188000000060032C2BF000008A30023
:10FF4000FDFF3200B01180000000060032C2BF0089
:10FF50006100600000000600889FBE008A9FBE000E
:10FF60008C1F78008002EB000203E9008003780018
:10FF70000104780003067800A92C20009A002000D4
:10FF80006B00200010408000E48242000028E60060
:10FF9000050078000408E300FEFF35003701780013
:10FFA000B70178000280FD0003026900F40FB2007F
:10FFB00004016900848169000280FD00F0002000D6
:10FFC0000030E60006007800800078000C80090010
:10FFD000000000001980A1000281D3001950AD007B
:10FFE0008381D3001958AD000C8009000000000087
:10FFF0001980A0001970A3000482D3008100E900D9
:020000040001F9
:10000000F2FF3100EF0010000122DE00041C780036
:100010004300DE000000E8000A28B4009580AB0031
:1000200008003200404080000A08E300050032006A
:100030008580A9009580A8000608B400100078000B
:100040002011880070035300CEFF31004F06780066
:100050004F05BE004F04BE00DC630400000000003A
:1000600011022000203F2000DC7C02000000000084
:1000700010002000606588000000060011022000CA
:10008000203F2000DC7C0200000000001000200067
:1000900060658800001020000000060011022000AA
:1000A000203F2000DC7C0200000000001000200047
:1000B000606588000000EB000000060011022000CF
:1000C000203F2000DC7C0200000000001000200027
:1000D000606588000000060081C0B30090AE20007B
:1000E00001487800A0AF20001054A10000000600D5
:1000F00081C0B30090AE200001487800A0AF20007E
:100100001054A1000000060001012000400621005B
:10011000DC7C0200000000000000060020C6280071
:100120004060020000000000000006008080FB002C
:100130000138A30003003200C002A900C202A800D7
:1001400002003700C002A900C202A9000128A300D2
:1001500003003200C962A800CB62A9000200370088
:10016000CB62A900C962A9000118A30003003200F4
:10017000C942A900CB42A80002003700C942A90029
:10018000CB42A9000008A30009003200A0AF200064
:10019000104078007040600002003200C8C2A80021
:1001A00006003700CCC2A800C8C2A900030037006F
:1001B000F0FB2F00CC22B600C822B60000000600DB
:1001C0000040DA000000FE00FFFFFF00FFFFFF001D
:1001D000FFFFFF00FFFFFF00FFFFFF00FFFFFF002B
:1001E000FFFFFF00FFFFFF00FFFFFF00FFFFFF001B
:1001F000FFFFFF00FFFFFF00FFFFFF00FFFFFF000B
:10020000FFFFFF00FFFFFF00FFFFFF00FFFFFF00FA
:00000001FF
